:104632004C45442D4465627567004C45442D5075C8
:104642006C7365720044696E203556004F70744970
:104652006E0043504C4400446F75742035562F321F
:1046620034560052656C616973004F70744F7574F3
:1046720000446F757420332E335600446F757420D6
:10468200352E305600446F75742032345600556909
:104692006E20302D322E35560055696E202B2D316D
:1046A20030560049696E20302D322E356D41004959
:1046B200696E20302D32356D410055696E20302DE6
:1046C200322E3556204673740055696E202B2D31DB
:1046D200305620466173740049696E20302D322EA7
:1046E200356D41204673740049696E20302D323594
:1046F2006D41204673740055696E202B2D31305662
:1047020020446966660055696E202B2D3130562093
:10471200466C740043696E20302D31306E46004382
:10472200696E20302D3175460050543130302D38AD
:10473200005054313030302D38004144353930008A
:1047420050543130302D32005054313030302D320F
:10475200004345524E4F582D3200554F757420304C
:104762002D322E355600554F7574202B2D31305673
:1047720000494F757420302D322E356D4100494F5E
:10478200757420302D32356D41004C69712E4865AB
:10479200206C6576656C00554F757420323030564A
:1047A20000554F7574203330305600554F757420C4
:1047B2003130562F3235306D410024526576240057
:1047C200013400000050254F757400000001000103
:1047D2000000000000437F00003F80000000000056
:1047E2000418000001502555696E230000010008DD
:1047F20004000000000000000000000000000000B3
:104802000418000001502555696E230000010004C0
:104812000400000000000000000000000000000092
:104822000418000001502555696E230000010002A2
:104832000400000000000000000000000000000072
:104842000418000001502555696E2300000100087C
:104852000400000000000000000000000000000052
:104862000134000008502552616E676500010000A6
:104872000000000000000000000000000000000036
:1048820004180000015025556F75742300010008BB
:104892000200000000402000003DCCCCCD00000012
:1048A20004180000015025556F757423000100089B
:1048B20002C1200000412000003F00000000000073
:1048C2000406FD0001502549696E2300000100081D
:1048D20004000000000000000000000000000000D2
:1048E200041DF70001502543696E230000010004F6
:1048F20004000000000000000000000000000000B2
:1049020004080000015025542300000000010008A3
:104912000200000000000000000000000000000093
:104922000406FD0009502545786369740001000002
:104932000100000000000000000000000000000074
:104942000408000001502554230000000001000863
:104952000200000000000000000000000000000053
:104962000408000001502554230000000001000249
:104972000200000000000000000000000000000033
:10498200040700000150255423000000000100022A
:104992000200000000000000000000000000000013
:1049A2000406FD00015025496F75742300010008BB
:1049B200020000000041A000003DCCCCCD00000070
:1049C20004180000015025556F7574230001000181
:1049D20002C1200000412000003DCCCCCD000000EF
:1049E2000406FD0009502545786369740001000042
:1049F200010000000042C800003F800000000000EB
:104A0200045A00000950254C4F6673000001000053
:104A12000200000000000000000000000000000092
:104A2200045D00000950254C4761696E00010000D9
:104A32000200000000000000000000000000000072
:104A420002030000085025546F6666000001000052
:104A52000000000000000000000000000000000054
:104A620002030000085025546F6E00000001000090
:104A72000000000000000000000000000000000034
:104A8200045A00000150254C696E0000000100002C
:104A92000100000000000000000000000000000013
:104AA2000132000000502544696E23000001000815
:104AB20001000000000000000000000000000000F3
:104AC2000132000000502544696E230000010004F9
:104AD20001000000000000000000000000000000D3
:104AE20001320000005025446F7574230001000854
:104AF20001000000003F8000003F80000000000035
:104B02000132000000502552656C230000010004B0
:104B120001000000003F8000003F80000000000014
:104B2200013200000050254F75742300000100047B
:104B320001000000003F8000003F800000000000F4
:104B4200041800000150255544230000000100080C
:104B52000300000000434800003F80000000000006
:104B62000418000001502555230000000001000830
:104B72000300000000000000000000000000000030
:104B82000406FA0001502549230000000001000834
:104B92000300000000000000000000000000000010
:104BA20001FF4632FF47C201FFBFE902FF463C0058
:104BB20000000100000020FF4647FF4AA201FFA7B4
:104BC2000321FF464EFF4AC201FFA70322FF4654BC
:104BD200FF4AA201FFA70340FF4659FF4AE201FF35
:104BE20095A141FF4665FF4B0201FF95A142FF4699
:104BF2006CFF4B2201FF95A143FF4673FF4AE2017E
:104C0200FF95A144FF467DFF4AE201FF95A145FFC2
:104C12004687FF4AE201FF95A160FF4690FF47E207
:104C220001FF6DF261FF469BFF47E201FF6DF262F9
:104C3200FF46A5FF48C201FF6DF263FF46B1FF4880
:104C4200C201FF6DF264FF46BCFF47E201FF719DA6
:104C520065FF46CBFF47E201FF719D66FF46DAFF23
:104C620048C201FF719D67FF46EAFF48C201FF711A
:104C72009D68FF46F9FF480201FF6DF269FF470890
:104C8200FF482201FF863770FF4716FF48E201FF07
:104C9200838B71FF4721FF48E201FF838B72FF473D
:104CA2002BFF490202FF64C673FF4733FF4902022A
:104CB200FF64C674FF473CFF494201FF785075FF0D
:104CC2004742FF496201FF549676FF474AFF496215
:104CD20001FF549677FF4753FF498201FF549680A4
:104CE200FF475CFF488201FF8D3A81FF4768FF481A
:104CF200A201FF5A0782FF4773FF49A201FF8D3AC3
:104D020083FF4780FF49A201FF8D3A84FF478CFF52
:104D120049E206FF22C685FF4799FF4B4203FF3552
:104D22003C86FF47A3FF4B4203FF353C87FF47AD5D
:104D3200FF49C201FF8D3A000000000000000000A0
:104D420000003CA3D70A3D23D70A3DA3D70A3E233E
:104D5200D70A3EA3D70A3F23D70A3FA3D70A402345
:104D6200D70A05040302010006070602070300042E
:024D7200050139
:06C24300041400000000DD
:10942400E5732412F8E6FFE5732413F8E6FD75519D
:03943400017B06B3
:10943700D2B1C2B0C2B2E49011A0F09011A0E0FE88
:10944700C39404504CEFC8EEC8088002C333D8FC5D
:109457005408D394004003D38001C392B3000000A3
:1094670000000000000000000000000000000000F5
:1094770000D2B00000000000000000000000000063
:1094870000000000000000C2B09011A0E004F080CE
:10949700AAE49011A0F09011A0E0FFC39403504CF0
:1094A700EDC8EFC8088002C333D8FC5404D3940036
:1094B7004003D38001C392B3000000000000000006
:1094C700000000000000000000000000D2B0000013
:1094D7000000000000000000000000000000000085
:1094E7000000C2B09011A0E004F080AAE49011A09F
:1094F700F09011A0E0FFC39404504CEBC8EFC808EC
:109507008002C333D8FC5408D394004003D38001AE
:10951700C392B3000000000000000000000000003C
:1095270000000000000000D2B000000000000000B2
:1095370000000000000000000000000000C2B09022
:1095470011A0E004F080AAD2B200000000000000E1
:1095570000000000000000000000000000D2B00082
:1095670000000000000000000000000000000000F4
:10957700000000C2B0C2B2C2B3E55124FF92B0D21C
:10958700B2C2B100000000000000000000000000AF
:0995970000000000000000C2B257
:0195A00022A8
:10C94500E5732409F8E6FFE573240AF8E6FD7B069E
:06C95500E4F551029437E5
:05B9F900F8E6FD7BFFF4
:03B9FE00CCEBCCC3
:10BA01007B0312C955E4901189F0EC5480D3940062
:10BA11004003D38001C392B3000000000000000086
:10BA2100000000000000000000000000D2B0000093
:10BA31000000000000000000000000000000000005
:10BA41000000C2B0EC25E0FC901189E004F0E0B404
:10BA510008B8C2B3D2B2000000000000000000002C
:10BA610000000000000000000000D2B00000000053
:10BA710000000000000000000000000000000000C5
:04BA8100C2B0C2B2DB
:01BA8500229E
:10B2D100E5732405F8EFF6E5732412F8E6FFE5734C
:0CB2E1002413F8E6FDE5732405F8E6FBF5
:03B2ED00CCEBCCDB
:10B2F0007B0212C955E4901189F0EC5480D394007C
:10B300004003D38001C392B300000000000000009E
:10B31000000000000000000000000000D2B00000AB
:10B32000000000000000000000000000000000001D
:10B330000000C2B0EC25E0FC901189E004F0E0B41C
:10B3400008B8C2B3D2B20000000000000000000044
:10B3500000000000000000000000D2B0000000006B
:10B3600000000000000000000000000000000000DD
:04B37000C2B0C2B2F3
:01B3740022B6
:0CB41800F8E6FD7B00E5732408F97A00DB
:06B424008B448A458946B5
:10B42A00E4FB12C955D2B20000000000000000007F
:10B43A000000000000000000000000D2B000000080
:10B44A0000000000000000000000000000000000F2
:10B45A0000C2B0C2B2E4901189F0000000000000FE
:10B46A000000000000000000000000000000D2B050
:10B47A0000000000000000000000000000000000C2
:10B48A0000000000C2B090118AE025E0FFA2B4E4F7
:10B49A00334FF0901189E004F0E0B408BD90118AAE
:0AB4AA00E0AB44AA45A9460207D210
:06B8D9008B448A458946FC
:10B8DF007B0112C955D2B200000000000000000029
:10B8EF000000000000000000000000D2B0000000C7
:10B8FF000000000000000000000000000000000039
:10B90F0000C2B0C2B2E4901189F000000000000044
:10B91F000000000000000000000000000000D2B096
:10B92F000000000000000000000000000000000008
:10B93F0000000000C2B090118AE025E0FFA2B4E43D
:10B94F00334FF0901189E004F0E0B408BD90118AF4
:0AB95F00E0AB44AA45A9460207D256
:03BB9E00CCEDCC1F
:10BBA1007B05E4FD12C955E490121BF0EC5480D3DF
:10BBB10094004003D38001C392B300000000000051
:10BBC1000000000000000000000000000000D2B0F2
:10BBD1000000000000000000000000000000000064
:10BBE10000000000C2B0EC25E0FC90121BE004F064
:10BBF100E0B408B8C2B3D2B20000000000000000F7
:10BC0100000000000000000000000000D2B00000B1
:10BC11000000000000000000000000000000000023
:06BC21000000C2B0C2B237
:01BC270022FA
:06B7B6008B3F8A4089412F
:10B7BC007B04E4FD12C955D2B20000000000000069
:10B7CC0000000000000000000000000000D2B000EB
:10B7DC00000000000000000000000000000000005D
:10B7EC00000000C2B0C2B2E490119EF00000000054
:10B7FC00000000000000000000000000000000003D
:10B80C00D2B00000000000000000000000000000AA
:10B81C00000000000000C2B090119FE025E0FFA2E4
:10B82C00B4E4334FF090119EE004F0E0B408BD9006
:0CB83C00119FE0AB3FAA40A9410207D2D7
:10C8E3007B017A117968129C7B901168E0D39400E4
:08C8F30040047F0180027F0078
:01C8FB00221A
:069C7B008B448A45894676
:109C81007B0712C955D2B30000000000000000009C
:109C91000000000000000000000000D2B000000041
:109CA10000000000000000000000000000000000B3
:109CB10000C2B0D2B30000000000000000000000AC
:109CC100000000000000000000D2B0000000000011
:109CD100000000000000000000000000000000C2C1
:109CE100B0C2B3000000000000000000000000004E
:109CF10000000000000000D2B000000000000000E1
:109D010000000000000000000000000000C2B0E4FC
:109D1100901169F0C2B300000000000000000000D3
:109D210000000000000000000000D2B000000000B0
:109D31000000000000000000000000000000000022
:109D4100C2B0901169E004F0E0B406C830B409ABC8
:109D510044AA45A946E4805FE4901169F00000003F
:109D610000000000000000000000000000000000F2
:109D710000D2B00000000000000000000000000060
:109D810000000000000000C2B090116BE025E0FF70
:109D910090116AE033FEA2B4E433FDEF4DFFEEF023
:109DA100A3EFF0901169E004F0E0B410B090116AF3
:0A9DB100E0AB44AA45A9461207D210
:019DBB002285
:10C5BF00901165EFF0A3EDF0A3EBF012C8E3EF706D
:10C5CF0002FF22901165E0FFA3E0FD7B017A117954
:10C5DF0064129C7B901167E0FF901164E06F700410
:06C5EF007F0180027F00C5
:01C5F5002223
:0388D900CCEBCC19
:1088DC007B0712C955D2B300000000000000000055
:1088EC000000000000000000000000D2B0000000FA
:1088FC00000000000000000000000000000000006C
:10890C0000C2B0C2B3000000000000000000000074
:10891C00000000000000000000D2B00000000000C9
:10892C00000000000000000000000000000000C279
:10893C00B0C2B30000000000000000000000000006
:10894C0000000000000000D2B00000000000000099
:10895C0000000000000000000000000000C2B0E4B5
:10896C00901218F0D2B300000000000000000000CC
:10897C0000000000000000000000D2B00000000069
:10898C0000000000000000000000000000000000DB
:10899C00C2B0901218E004F0E0B406C8D2B20000E5
:1089AC0000000000000000000000000000000000BB
:1089BC000000C2B2D2B300000000000000000000B2
:1089CC0000000000000000000000D2B00000000019
:1089DC00000000000000000000000000000000008B
:1089EC00C2B0C2B300000000000000000000000094
:1089FC000000000000000000D2B0000000000000E9
:108A0C000000000000000000000000000000C2B0E8
:108A1C00D2B30000000000000000000000000000C5
:108A2C00000000000000D2B00000000000000000B8
:108A3C00000000000000000000000000C2B0E49044
:108A4C001218F0C2B300000000000000000000008B
:108A5C00000000000000000000D2B0000000000088
:108A6C00000000000000000000000000000000C238
:108A7C00B0901218E004F0E0B406C8E4901218F0BC
:108A8C00EC5480D394004003D38001C392B3000014
:108A9C0000000000000000000000000000000000CA
:108AAC000000D2B000000000000000000000000038
:108ABC000000000000000000C2B0EC25E0FC9012A9
:108ACC0018E004F0E0B410B8D2B2000000000000CE
:108ADC000000000000000000000000000000C2B216
:0A8AEC00E4901219F0A3F020B42763
:0D8AF600751E01751F0300D51FFCD51EF66F
:108B030090121AE004F07006901219E004F090122B
:0A8B130019E0B427DBA3E0B410D68C
:018B1D002235
:1095A1001573A873EBF61573A873EDF61573A8730D
:0495B100EFF6157349
:1095B500A8730808E664016003029643E573240472
:1095C500F8E6FEE5732403F8E6FF75F008A42EF52A
:1095D50082E435F0F583E5822419F582E583340CC0
:1095E500F583E4F0F584E5EF20E119E5732404F84B
:1095F500E6FDEF75F008A42D2419F9E4340CFA7B87
:109605000112B8D9E5732403F8E6FFE5732404F8DD
:10961500E6FD75F008EFA42DF582E435F0F583E558
:10962500822419F582E583340CF583E0FB12B2ED53
:10963500E5732403F8E6FFE573240412B9F9A8736A
:109645000808E66402600302970CE5732406F8CB6C
:10965500E6CB08E6FA08E6F912078CA873F6603E31
:10966500E5732404F8E6FFE5732403F8E675F008CE
:10967500A42FF582E435F0F583E5822419F582E51A
:1096850083340CF583E0FFE5732405F8E6FE7401E9
:10969500C8EEC8088002C333D8FC4FF0803DE5739F
:1096A5002404F8E6FFE5732403F8E675F008A42F13
:1096B500F582E435F0F583E5822419F582E58334F6
:1096C5000CF583E0FFE5732405F8E6FE7401C8EEAA
:1096D500C8088002C333D8FCF45FF0E5732403F8AF
:1096E500E6FFE5732404F8E6FD75F008EFA42DF513
:1096F50082E435F0F583E5822419F582E583340C9F
:09970500F583E0FB12B2ED7F00D8
:07970E00E5732409F5732245
:10A703001573A873EBF61573A873EDF61573A87399
:04A71300EFF61573D5
:10A71700A8730808E66403600302A80AE573240621
:10A72700F8CBE6CB08E6FA08E6F912078C603EE5B7
:10A73700732404F8E6FFE5732403F8E675F008A42C
:10A747002FF582E435F0F583E5822419F582E58358
:10A75700340CF583E0FFE5732405F8E6FE7401C8C1
:10A76700EEC8088002C333D8FC4FF0803DE5732460
:10A7770004F8E6FFE5732403F8E675F008A42FF55F
:10A7870082E435F0F583E5822419F582E583340CFC
:10A79700F583E0FFE5732405F8E6FE7401C8EEC80B
:10A7A700088002C333D8FCF45FF0E5732403F8E6AE
:10A7B700FFE5732404F8E6FD7B00A9737A0012B461
:10A7C70024E5732405F974017E00C8E7C8088005ED
:10A7D700C333CE33CED8F9FFA873E6FDEF5DD3942C
:10A7E700007480948040047F0180027F00E5732419
:10A7F70006F8CBE6CB08E6FA08E6F9EF1207D27FB0
:05A807000180027F004A
:07A80C00E5732409F5732236
:10BFE9001573A873EBF61573A873EDF61573A8739B
:10BFF900EFF6A87308E6B4010DA8730808E6FFE593
:10C0090073240312B9F9A87308E6B40222A87308C5
:10C0190008E6FFE5732403F8E6FDE5732405F8CB8C
:10C02900E6CB08E6FA08E6F912078CFB12B2ED7FB7
:08C0390000E5732408F57322F1
:108D3A001573A873EBF61573A873EDF61573A8737C
:088D4A00EFF6E57324F9F5735F
:108D52002408F8E664026003028F41E573240CF8EC
:108D6200CBE6CB08E6FA08E6F9120983A873120AE1
:108D72006EE5732407F8E6B40209E4FBFA79C878D1
:108D8200428022E5732407F8E6B48209E4FBFA790B
:108D92002078408010E5732407F8E6B4832FE4FBC3
:108DA200FA79C87841E8C0E0A8731209EDD0E0F87A
:108DB2001202A77B007AFF797F784712019E120385
:108DC200FBE5732404F8EEF608EFF68046E573241B
:108DD20007F8E6B4873DE4FBFA79A07841E8C0E001
:108DE200A8731209EDD0E0F81202A7E4FBFAF978B1
:108DF2003F1200AD7B007AFF797F784712019E1205
:108E020003FBE5732404F8EEF608EFF6E573240B92
:108E1200F8760112C945E5732406F8E4F6E57324F1
:108E220006F8E6FFC39404503FEF94014003D38059
:108E320001C392B300000000000000000000000027
:108E42000000000000000000D2B00000000000009E
:108E52000000000000000000000000000000C2B09E
:108E6200E5732406F80680B5E5732406F8E4F6E512
:108E7200732406F8E6C394045051E573240BF8E614
:108E8200FF5408D394004003D38001C392B300007F
:108E920000000000000000000000000000000000D0
:108EA2000000D2B00000000000000000000000003E
:108EB2000000000000000000C2B0E573240BF8EFD0
:108EC20025E0F6E5732406F80680A4E5732406F887
:108ED200E4F6E5732406F8E6C394105060E57324C3
:108EE20004F8E6FE08E6FFEE5480FCD3E49400ECBE
:108EF20094004003D38001C392B30000000000003D
:108F02000000000000000000000000000000D2B0DD
:108F1200000000000000000000000000000000004F
:108F220000000000C2B0E5732404F8EF25E0FFEE74
:108F320033F608EFF6E5732406F8068095D2B17F82
:018F4200002E
:078F4300E573240FF5732212
:105A07001573A873EBF61573A873EDF61573A873E2
:085A1700EFF6E57324F9F573C5
:105A1F00E5732408F8E664026003025F5FE5732410
:105A2F000CF8CBE6CB08E6FA08E6F9120983A8735F
:105A3F00120A6EE4FFFE7D207C41A873120A151234
:105A4F000344600B4009A873120A8641200000E44A
:105A5F00FFFE7D207CC1A873120A15120344500962
:105A6F00A873120A86C1200000E4FFFE7D207C414E
:105A7F00A873120A151200ADE4FBFA79A07841124F
:105A8F0002A77B007AFF797F784712019EE4FBFA29
:105A9F00F9783F1200AD1203FBE5732404F8EEF61C
:105AAF0008EFF612C945C2B3000000000000000065
:105ABF00000000000000000000000000D2B0000055
:105ACF0000000000000000000000000000000000C7
:105ADF000000C2B0C2B300000000000000000000D0
:105AEF0000000000000000000000D2B00000000025
:105AFF000000000000000000000000000000000097
:105B0F00C2B0E573240BF8E6FFC394045049E57364
:105B1F002406F8E4F6E5732406F8E6C3941640036A
:105B2F00025D0900000000000000000000000000FE
:105B3F0000000000000000D2B000000000000000D4
:105B4F0000000000000000000000000000C2B0E5EF
:105B5F00732406F80680BEC2B300000000000000E8
:105B6F0000000000000000000000000000D2B000A4
:105B7F000000000000000000000000000000000016
:105B8F00000000C2B0D2B30000000000000000000F
:105B9F000000000000000000000000D2B000000074
:105BAF0000000000000000000000000000000000E6
:105BBF0000C2B0C2B30000000000000000000000EF
:105BCF00000000000000000000D2B0000000000044
:105BDF00000000000000000000000000000000C2F4
:105BEF00B0C2B30000000000000000000000000081
:105BFF0000000000000000D2B00000000000000014
:105C0F0000000000000000000000000000C2B0EF24
:105C1F005402D394004003D38001C392B300000019
:105C2F000000000000000000000000000000000065
:105C3F0000D2B000000000000000000000000000D3
:105C4F0000000000000000C2B0E573240BF8E6541A
:105C5F0001D394004003D38001C392B3000000002E
:105C6F000000000000000000000000000000000025
:105C7F00D2B0000000000000000000000000000093
:105C8F00000000000000C2B0E5732406F8E4F6E55A
:105C9F00732406F8E6C394105060E5732404F8E605
:105CAF00FE08E6FFEE5480FCD3E49400EC94004031
:105CBF0003D38001C392B300000000000000000076
:105CCF000000000000000000000000D2B000000043
:105CDF0000000000000000000000000000000000B5
:105CEF0000C2B0E5732404F8EF25E0FFEE33F608A9
:105CFF00EFF6E5732406F8068095C2B300000000A6
:105D0F000000000000000000000000000000000084
:105D1F00D2B00000000000000000000000000000F2
:105D2F00000000000000C2B0C2B30000000000007D
:105D3F000000000000000000000000000000D2B0D2
:105D4F000000000000000000000000000000000044
:105D5F0000000000C2B0E573240BF8E6FFD39403F4
:105D6F004049E5732406F8E4F6E5732406F8E6C324
:105D7F0094164003025F5D00000000000000000069
:105D8F000000000000000000000000D2B000000082
:105D9F0000000000000000000000000000000000F4
:105DAF0000C2B0E5732406F80680BEC2B30000003F
:105DBF0000000000000000000000000000000000D4
:105DCF0000D2B00000000000000000000000000042
:105DDF0000000000000000C2B0D2B30000000000BD
:105DEF00000000000000000000000000000000D2D2
:105DFF00B0000000000000000000000000000000E4
:105E0F000000000000C2B0C2B3000000000000009C
:105E1F0000000000000000000000000000D2B000F1
:105E2F000000000000000000000000000000000063
:105E3F00000000C2B0C2B30000000000000000006C
:105E4F000000000000000000000000D2B0000000C1
:105E5F000000000000000000000000000000000033
:105E6F0000C2B0EF5402D394004003D38001C39219
:105E7F00B300000000000000000000000000000060
:105E8F000000000000D2B000000000000000000081
:105E9F000000000000000000000000C2B0E5732405
:105EAF000BF8E65401D394004003D38001C392B39F
:105EBF0000000000000000000000000000000000D3
:105ECF0000000000D2B00000000000000000000041
:105EDF0000000000000000000000C2B0E5732406BF
:105EEF00F8E4F6E5732406F8E6C394105060E57302
:105EFF002404F8E6FE08E6FFEE5480FCD3E4940099
:105F0F00EC94004003D38001C392B3000000000063
:105F1F00000000000000000000000000000000D2A0
:105F2F00B0000000000000000000000000000000B2
:105F3F000000000000C2B0E5732404F8EF25E0FF75
:105F4F00EE33F608EFF6E5732406F8068095D2B126
:025F5F007F00C1
:075F6100E573240FF5732224
:0B987B007D527F031298867D037F0161
:109886001573A873EDF61573A873EFF615731573B4
:10989600C2B3C2B1000000000000000000000000DA
:1098A6000000000000000000A873E4F6A873E6C3F9
:1098B60094045031C2B0C2B30000000000000000A2
:1098C600000000000000000000000000D2B0000010
:1098D6000000000000000000000000000000000082
:1098E60000000680C7A873E4F6A873087608A87374
:1098F600E6C39404504AC2B008E6FFA873080856A7
:1099060094004003D38001C392B30000000000001E
:109916000000000000000000000000000000D2B0BF
:109926000000000000000000000000000000000031
:1099360000000000A87308EFC313F6A8730680AEF4
:10994600D2B200000000000000000000000000008D
:10995600000000000000C2B2A873E4F6A8730876FF
:1099660080A873E6C39408504DC2B008E6FFE573BD
:109976002403F8E65FD394004003D38001C392B377
:1099860000000000000000000000000000000000D1
:1099960000000000D2B0000000000000000000003F
:1099A60000000000000000000000A87308EFC313C9
:1099B600F6A8730680ABD2B1C2B300000000000067
:0E99C600000000000000000000000000000093
:0799D400E5732404F5732282
:0AB4B4001573A873EFF615731573F6
:10B4BE00C2B3C2B100000000000000000000000096
:10B4CE000000000000000000A873E4F6A8730876E0
:10B4DE0080A873E6C39408504AC2B008E6FFA8736A
:10B4EE0008085694004003D38001C392B3000000B5
:10B4FE00000000000000000000000000000000003E
:10B50E0000D2B000000000000000000000000000AB
:10B51E0000000000000000A87308EFC313F6A87324
:10B52E000680AED2B1C2B3000000000000000000E1
:0BB53E00000000000000000000000002
:07B549000573057305732271
:0B8F4A007B00E5732409F97A007F0426
:108F5500157315731573A873C6EBC608C6EAC6085C
:0D8F6500C6E9C61573A873EFF615731573F2
:108F7200C2B100000000000000000000000000007C
:108F8200000000000000A873E4F6A873E6FFC39493
:108F920004503BC2B0EFB40103D38001C392B300CB
:108FA20000000000000000000000000000000000BF
:108FB200000000D2B000000000000000000000002D
:108FC200000000000000000000A8730680BCA87327
:108FD200E4F6A873087608A873E6C39404504AC25C
:108FE200B008E6FFA87308085694004003D3800136
:108FF200C392B30000000000000000000000000067
:1090020000000000000000D2B000000000000000DC
:1090120000000000000000000000000000A873082B
:10902200EFC313F6A8730680AED2B20000000000B0
:10903200000000000000000000000000000000C26C
:10904200B2A873E4F6E5732403F8CBE6CB08E6FA9C
:1090520008E6F9120AD000000000A873E6C39418CB
:109062005070C2B0000000000000000000000000CC
:109072000000000000000000E5732403F8CBE6CBFB
:1090820008E6FA08E6F91209837801120970C8ECB9
:10909200C8C9EDC9CAEECACBEFCBA2B4E4334BFFC9
:1090A200EAFEE9FDE8FCE5732403F8CBE6CB08E62B
:1090B200FA08E6F91209D3D2B0000000000000005D
:1090C20000000000000000000000000000A873067D
:1090D2008088D2B100000000000000000000000003
:0890E200000000000000000086
:0790EA00E5732406F5732273
:10B17500E573240BF8E6FFE573240CF8E6FD7B0781
:10B185008F448D45CAEBCA7B8012B9FEE4FBAD4501
:10B19500AF4412B2ED7B80AD45AF4412B2ED7551AF
:0DB1A500017B06AD45AF4412943712987B34
:0DB1B20075466475470300D547FCD546F689
:10B1BF00EA5407FF75F008E544A42545F582E43508
:10B1CF00F0F583E5822439F582E583340DF583EFBD
:10B1DF00F0CFEACFCDEFCD7F0212988675F008E55C
:10B1EF0044A42545F582E435F0F583E5822449F53D
:10B1FF0082E583340EF583E4F012C9C2E54475F09D
:10B20F0008A4254525E025E02461F582E4340DF5F9
:04B21F0083020A7A22
:106DF2001573A873EBF61573A873EDF61573A873E4
:086E0200EFF6E57324F7F573C8
:106E0A00240AF8E6B4010312B175E573240AF8E618
:106E1A00FF64027042E573240DF8E6B40839E5739D
:106E2A00240EF8CBE6CB08E6FA08E6F912078CFE40
:106E3A00E573240CF8E6FDE573240BF8E675F00813
:106E4A00A42DF582E435F0F583E5822439F582E54F
:106E5A0083340DF583EEF0EF64036003027194E569
:106E6A0073240DF8E6D3940740057F00027196E576
:106E7A0073240BF8E6FFE573240C12B418E57324A7
:106E8A0008F8E65401D39400405F12C9C2ECC0E08E
:106E9A00EDC0E0EEC0E0EFC0E0E573240BF8E67564
:106EAA00F008A4FFE573240CF8EF2625E025E0247A
:106EBA0061F582E4340DF583E0FCA3E0FDA3E0FE76
:106ECA00A3E0242CFBEE3401FAE43DF9E43CF8D0CB
:106EDA00E0FFD0E0FED0E0FDD0E0FCC312095F5035
:106EEA000312B1757F00027196E573240CF8E6FF70
:106EFA00E573240BF8E675F008A42FF582E435F063
:106F0A00F583E5822449F582E583340EF583E0FFB3
:106F1A00E573240DF8E66F60057F0002719612C9C9
:106F2A00C2EFC0E0E573240BF8E6F975F008A4FF98
:106F3A00E573240CF8E6FB2F25E025E02461F582B1
:106F4A00E4340DF583D0E0FF120A7ACFE9CFCDEB16
:106F5A00CD1294327B00E5732404128F50E573241A
:106F6A0009F8E66468702CE573240CF8E6FFE5730B
:106F7A00240BF8E6FE75F008A42FF582E435F0F547
:106F8A0083E5822449F582E583340EF583E00454CF
:106F9A0003802AE573240CF8E6FFE573240BF8E670
:106FAA00FE75F008A42FF582E435F0F583E5822416
:106FBA0049F582E583340EF583E0045407FD75F044
:106FCA0008EEA42FF582E435F0F583E5822449F52D
:106FDA0082E583340EF583EDF0E573240CF8E6FFC1
:106FEA00E573240BF8E6FE75F008A42FF582E43564
:106FFA00F0F583E5822449F582E583340EF583E0D2
:10700A00C454F04408FD75F008EEA42FF582E43567
:10701A00F0F583E5822439F582E583340DF583E0C2
:10702A004DFD7F02129886E5732404F81209EDE4F7
:10703A001203BDE4FBFA7980784B1202A7E57324A8
:10704A000CF8E6FBE573240BF8E675F008A42BF5BB
:10705A0082E435F0F583E5822439F582E583340D3F
:10706A00F583E025E025E02444F582E4344DF583F8
:10707A00120A2E12019EA873120A6EE5732409F8E9
:10708A00E6B460028014E5732409F8E6B46102806C
:10709A0043E5732409F8E6B46211A873E8C0E01264
:1070AA0009EDE4FBFA7980783F8018E5732409F842
:1070BA00E6B46317A873E8C0E01209EDE4FBFA79B5
:1070CA0020784112019ED0E0F88034E5732409F853
:1070DA00E6B4682EE4FBFA79207840E8C0E0A873A9
:1070EA001209EDD0E0F81202A7E4FBFA79A0784180
:1070FA0012019EE4FBFA792078C11200ADA873123E
:10710A000A6EE5732409F8E6FF64616009EF6463B7
:10711A006004EFB4682A7F007E507DC37C47A87361
:10712A00120A1512019EE4FBFAF9783F1200AD1219
:10713A0003FBEC1203BD7B007A5079C378478028A1
:10714A007F007E247D747C49A873120A1512019E61
:10715A00E4FBFAF9783F1200AD1203FBEC1203BD0F
:10716A007B007A24797478491202A7A873120A6EEE
:10717A00A8731209EDE573240EF8CBE6CB08E6FAFC
:0C718A0008E6F91209D37F0480027F00A0
:07719600E5732411F57322DB
:1064C6001573A873EBF61573A873EDF61573A87319
:0864D600EFF6E57324F3F57302
:1064DE00240EF8E6B4012DE573240FF8E6FFE573FC
:1064EE002410F8E6FD7B0F12B185E5732410F8E653
:1064FE0025E025E02441F582E4340DF583120A9F50
:10650E003F800000E573240EF8E664026003026526
:10651E00D5E5732411F8E6640860030265D5E573CA
:10652E002412F8CBE6CB08E6FA08E6F9120983E561
:10653E00732410F8E6FB25E025E02441F582E434CF
:10654E000DF583120A7AEB25E025E02441F582E46D
:10655E00340DF583E0FCA3E0FDA3E0FEA3E0FF7B9A
:10656E000A7AD77923783C1203446002502AE573E5
:10657E002410F8E625E025E02441F582E4340DF5FB
:10658E0083E0FCA3E0FDA3E0FEA3E0FFE4FBFA79C9
:10659E00207841120344502FE5732410F8E625E0CD
:1065AE0025E02441F582E4340DF583120A9F3F80E5
:1065BE000000E5732412F8CBE6CB08E6FA08E6F9FC
:1065CE00120AD03F800000E573240EF8E6640360E3
:1065DE000302697AE5732411F8E6D3940740057F28
:1065EE000002697CE573240FF8E6FFE573241012B0
:1065FE00B418E5732408F8E65401D39400406F12E2
:10660E00C9C2ECC0E0EDC0E0EEC0E0EFC0E0E57363
:10661E00240FF8E675F008A4FFE5732410F8EF26B2
:10662E0025E025E02461F582E4340DF583E0FCA33A
:10663E00E0FDA3E0FEA3E0242CFBEE3401FAE43DE2
:10664E00F9E43CF8D0E0FFD0E0FED0E0FDD0E0FC75
:10665E00C312095F5013E573240FF8E6FFE57324A8
:10666E0010F8E6FD7B0F12B1857F0002697CE573A1
:10667E002410F8E6FDE573240FF8E6FE75F008A485
:10668E002DF582E435F0F583E5822449F582E58324
:10669E00340EF583E0FFE5732411F8E66F60057F95
:1066AE000002697CCFEECF129432128F4AE573242A
:1066BE0010F8E6FFE573240FF8E6FE75F008A42F38
:1066CE00F582E435F0F583E5822449F582E58334DD
:1066DE000EF583E0045407FD75F008EEA42FF58245
:1066EE00E435F0F583E5822449F582E583340EF531
:1066FE0083EDF0E5732410F8E6FFE573240FF8E65A
:10670E0075F008A42FF582E435F0F583E58224496F
:10671E00F582E583340EF583E0C454F0440FFD7F1B
:10672E0002129886E5732409F81209EDE41203BDEE
:10673E00E4FBFA7980784B1202A77B0A7AD7792389
:10674E00784012019EA873120A6EA8731209EDE525
:10675E00732404F8120A6EE5732411F8E6D394003C
:10676E00403BA873E8C0E01209EDE573240FF8E68C
:10677E0075F008A4FBE5732410F8EB2625E025E060
:10678E002481F582E4340DF583E0F8A3E0F9A3E06B
:10679E00FAA3E0FB1200A9D0E0F8120A6EE573240A
:1067AE0004F81209EDE573240FF8E675F008A4FB62
:1067BE00E5732410F8EB2625E025E02481F582E42C
:1067CE00340DF583120A7AA873E8C0E01209EDECD5
:1067DE00C0E0EDC0E0EEC0E0EFC0E0E5732410F8DD
:1067EE00E625E025E02441F582E4340DF583E0FC56
:1067FE00A3E0FDA3E0FEA3E0FF7B6F7A127983781E
:10680E003A12019EC8ECC8C9EDC9CAEECACBEFCB8D
:10681E00D0E0FFD0E0FED0E0FDD0E0FC1202A7D029
:10682E00E0F8120A6EE573240DF8E6B47318A87337
:10683E00E8C0E01209EDE4FBFA792078411202A7D4
:10684E00D0E0F8120A6E7F757E787D0C7C35A873C9
:10685E00120A1512019EA873120A1512019EA87330
:10686E00120A1512019EECC0E0EDC0E0EEC0E0EFA2
:10687E00C0E07FFA7EED7D6B7C3AA873120A15128A
:10688E00019EA873120A1512019ED0E0FBD0E0FA09
:10689E00D0E0F9D0E0F81200ADECC0E0EDC0E0EED3
:1068AE00C0E0EFC0E07F177ED97D167C40A8731242
:1068BE000A1512019ED0E0FBD0E0FAD0E0F9D0E04C
:1068CE00F81200AD7BD37A4D79E278411200ADA873
:1068DE0073120A6EA873E8C0E01209ED7B337A9347
:1068EE00798878431200A9D0E0F8120A6EE4FFFE10
:1068FE007D207C41A873120A1512019EE4FBFAF961
:10690E00783F1200AD1203FBEC1203BDE4FBFA79E3
:10691E002078411202A7A873120A6E7F007EC07DF6
:10692E00797C44A873120A15120344600B4009A81F
:10693E0073120A864479F99AE4FFFE7D487CC3A857
:10694E0073120A151203445009A873120A86C479E9
:10695E00F99AA8731209EDE5732412F8CBE6CB0869
:0E696E00E6FA08E6F91209D37F0480027F01E1
:07697C00E5732415F57322F9
:105496001573A873EBF61573A873EDF61573A87359
:0854A600EFF6E57324F6F5733F
:1054AE00240BF8E664017055E573240AF8E6B47728
:1054BE0012E573240CF8E6FFE573240DF8E6FD7B88
:1054CE00888010E573240CF8E6FFE573240DF8E6EA
:1054DE00FD7B8C12B185E573240DF8E6FFE5732490
:1054EE000CF8E675F008A42FF582E435F0F583E5A7
:1054FE00822449F582E583340EF583E4F0E57324C6
:10550E000BF8E6640360030259FEE573240EF8E619
:10551E00D3940240057F00025A00E573240CF8E68E
:10552E00FFE573240DF8E6FD7B00E5732404F97A9C
:10553E000012B424E5732404F8E65401D394005009
:10554E00030255DC12C9C2ECC0E0EDC0E0EEC0E0D3
:10555E00EFC0E0E573240CF8E675F008A4FFE573E0
:10556E00240DF8EF2625E025E02461F582E4340DC4
:10557E00F583E0FCA3E0FDA3E0FEA3E0242CFBEE0C
:10558E003401FAE43DF9E43CF8D0E0FFD0E0FED07F
:10559E00E0FDD0E0FCC312095F502EE573240AF83B
:1055AE00E6B47712E573240CF8E6FFE573240DF8E4
:1055BE00E6FD7B888010E573240CF8E6FFE5732486
:1055CE000DF8E6FD7B8C12B1857F00025A00E57363
:1055DE00240DF8E6FDE573240CF8E6FE75F008A43C
:1055EE002DF582E435F0F583E5822449F582E583D5
:1055FE00340EF583E0FFE5732405F8EFF65401FF52
:10560E00E573240EF8EF6660057F00025A00CFEEB8
:10561E00CF1294327B00E5732406128F50E573246B
:10562E000AF8E6647760030256CDE573240DF8E6BA
:10563E00FFE573240CF8E6FE75F008A42FF582E45E
:10564E0035F0F583E5822449F582E583340EF58342
:10565E00E0045401FD75F008EEA42FF582E435F058
:10566E00F583E5822449F582E583340EF583EDF06A
:10567E00E573240DF8E6FF75F008EEA42FF582E42D
:10568E0035F0F583E5822449F582E583340EF58302
:10569E00E070047D8880027D987F02129886E57303
:1056AE002406F81209EDE41203BDE4FBFA798078C2
:1056BE004B1202A77B0A7AD779A3783C02575DE595
:1056CE0073240DF8E6FFE573240CF8E6FE75F0087A
:1056DE00A42FF582E435F0F583E5822449F582E5C1
:1056EE0083340EF583E0045401FD75F008EEA42F0B
:1056FE00F582E435F0F583E5822449F582E58334BD
:10570E000EF583EDF0E573240DF8E6FF75F008EE67
:10571E00A42FF582E435F0F583E5822449F582E580
:10572E0083340EF583E0C454F0448CFD7F0212984E
:10573E0086E5732406F81209EDE41203BDE4FBFAC4
:10574E007980784B1202A77B0A7AD779A3783E121A
:10575E00019EA873120A6EE573240AF8E6FF6475BB
:10576E006008EF64766003025859A873E8C0E0122F
:10577E0009ED7B6F7A127983783A1202A7D0E0F89E
:10578E00120A6EE573240AF8E6B47618A873E8C018
:10579E00E01209EDE4FBFA792078411202A7D0E07D
:1057AE00F8120A6E7F757E787D0C7C35A873120A0E
:1057BE001512019EA873120A1512019EA873120AE1
:1057CE001512019EECC0E0EDC0E0EEC0E0EFC0E0CF
:1057DE007FFA7EED7D6B7C3AA873120A1512019E3C
:1057EE00A873120A1512019ED0E0FBD0E0FAD0E0A9
:1057FE00F9D0E0F81200ADECC0E0EDC0E0EEC0E094
:10580E00EFC0E07F177ED97D167C40A873120A1573
:10581E0012019ED0E0FBD0E0FAD0E0F9D0E0F81211
:10582E0000AD7BD37A4D79E278411200ADA87312A8
:10583E000A6EA873E8C0E01209ED7B337A9379887B
:10584E0078431200A9D0E0F802597CE573240AF8D7
:10585E00E66477600302597FA873E8C0E01209ED91
:10586E007B007A247974784912019ED0E0F8120AEE
:10587E006E7F5D7E0B7D237C2CA873120A151201A0
:10588E009EA873120A1512019EA873120A15120110
:10589E009EA873120A1512019EECC0E0EDC0E0EE58
:1058AE00C0E0EFC0E07F177EEE7D8B7C32A87312D6
:1058BE000A1512019EA873120A1512019EA87312E0
:1058CE000A1512019EC8ECC8C9EDC9CAEECACBEFC3
:1058DE00CBD0E0FFD0E0FED0E0FDD0E0FC1200A97E
:1058EE00ECC0E0EDC0E0EEC0E0EFC0E07F4B7E5FCD
:1058FE007D047C38A873120A1512019EA873120A31
:10590E001512019ED0E0FBD0E0FAD0E0F9D0E0F81D
:10591E001200ADECC0E0EDC0E0EEC0E0EFC0E07F05
:10592E004B7E767D6C7C3DA873120A1512019ED0BB
:10593E00E0FBD0E0FAD0E0F9D0E0F81200AD7B1F2A
:10594E007A85796B78BE1200ADA873120A6EE4FFE9
:10595E00FEFDFCA873120A151203446014A87312FC
:10596E000A15E4FFFE7D7A7C441202A7A873120A80
:10597E006EE4FFFE7DC87C42A873120A1512019ECA
:10598E00E4FBFAF9783F1200AD1203FBEC1203BDF3
:10599E00E4FBFA79C878421202A7A873120A6E7F46
:1059AE005C7EFF7D797C44A873120A151203446055
:1059BE000B4009A873120A864479FF5CE4FFFE7D52
:1059CE00487CC3A873120A151203445009A8731217
:1059DE000A86C479FF5CA8731209EDE573240FF8EB
:1059EE00CBE6CB08E6FA08E6F91209D37F0480026B
:0259FE007F0127
:075A0000E5732412F5732287
:107850001573A873EBF61573A873EDF61573A8737B
:08786000EFF6E57324F7F57360
:10786800E573240AF8E66401704FE573240BF8E623
:10787800FFE573240CF8E6FD7B0512B185E573245A
:107888000CF8E6FFE573240BF8E675F008A42FF56D
:1078980082E435F0F583E5822449F582E583340EE8
:1078A800F583E4F0EF25E025E02441F582E4340D8A
:1078B800F583120A9F3F800000E573240AF8E66406
:1078C800036003027B35E573240DF8E6D394074083
:1078D800057F00027B37E573240BF8E6FFE5732488
:1078E8000CF8E6FD7B00E5732404F97A0012B42451
:1078F800E5732404F8E65401D39400406F12C9C21A
:10790800ECC0E0EDC0E0EEC0E0EFC0E0E573240BB2
:10791800F8E675F008A4FFE573240CF8EF2625E0D7
:1079280025E02461F582E4340DF583E0FCA3E0FD55
:10793800A3E0FEA3E0242CFBEE3401FAE43DF9E4D5
:107948003CF8D0E0FFD0E0FED0E0FDD0E0FCC31270
:10795800095F5013E573240BF8E6FFE573240CF870
:10796800E6FD7B0512B1857F00027B37E573240CA9
:10797800F8E6FDE573240BF8E6FE75F008A42DF58E
:1079880082E435F0F583E5822449F582E583340EF7
:10799800F583E0FFE573240DF8E66F60057F0002CC
:1079A8007B37CFEECF1294327B00E5732405128F1C
:1079B80050E573240CF8E6FFE573240BF8E6FE7532
:1079C800F008A42FF582E435F0F583E5822449F523
:1079D80082E583340EF583E0045407FD75F008EE64
:1079E800A42FF582E435F0F583E5822449F582E594
:1079F80083340EF583EDF0E573240CF8E6FFE573A8
:107A0800240BF8E675F008A42FF582E435F0F58329
:107A1800E5822449F582E583340EF583E0C454F009
:107A28004405FD7F02129886E5732405F81209EDD6
:107A3800E41203BDE4FBFA7980784B1202A77B0AB3
:107A48007AD779A3783F12019EC8ECC8C9EDC9CA94
:107A5800EECACBEFCB7F0A7ED77D237C3F1200A9ED
:107A6800A873120A6EA873E8C0E01209EDE4FBFAE5
:107A7800797A78441202A7D0E0F8120A6EA873E85F
:107A8800C0E01209ED7B007A247974784912019ECE
:107A9800D0E0F8120A6EA873E8C0E01209ED7B9AEC
:107AA8007A99798878431200A9D0E0F8120A6EE42E
:107AB800FFFE7DC87C42A873120A1512019EE4FBE2
:107AC800FAF9783F1200AD1203FBEC1203BDE4FB98
:107AD800FA79C878421202A7A873120A6EE4FFFE68
:107AE8007D167C43A873120A15120344600B4009E3
:107AF800A873120A864479FF5CE4FFFE7D5C7CC2B1
:107B0800A873120A151203445009A873120A86C4EE
:107B180079FF5CA8731209EDE573240EF8CBE6CB68
:0F7B280008E6FA08E6F91209D37F0480027F010C
:077B3700E5732411F5732230
:0CB550007F011299DB7FFC12B55C7F00CC
:08B55C001573A873EFF61573D7
:10B56400C2B3C2B1000000000000000000000000EF
:10B574000000000000000000A873E4F6A873E6C30E
:10B5840094085047D2B008E6FF548094004003D397
:10B594008001C392B300000000000000000000001E
:10B5A400000000000000000000C2B0000000000025
:10B5B400000000000000000000000000000000A8DF
:10B5C4007308EF25E0F6A8730680B1D2B1C2B300C8
:10B5D4000000000000000000000000000000000067
:03B5E40000000064
:05B5E70005730573224D
:1099DB001573A873EDF61573A873EFF6157315735E
:1099EB00C2B3C2B100000000000000000000000084
:1099FB000000000000000000A8730808E62450A82F
:109A0B007308F6A873E4F6A873E6C394085047D21C
:109A1B00B008E6FF548094004003D38001C392B397
:109A2B00000000000000000000000000000000002B
:109A3B0000000000C2B000000000000000000000A9
:109A4B0000000000000000000000A87308EF25E0F4
:109A5B00F6A8730680B1A8730808E62450A873080B
:109A6B00F6A873E4F6A873E6C394085040D2B0C2CC
:109A7B00B300000000000000000000000000000028
:109A8B000000000000C2B000000000000000000059
:109A9B00000000000000000000000008E8C0E0E645
:109AAB0025E0FFD0E0F8EFF6A8730680B8A873E4C2
:109ABB00F6A873E6C39408504ED2B0E5732403F8AE
:109ACB00E6FF5480D394004003D38001C392B300CC
:109ADB00000000000000000000000000000000007B
:109AEB00000000C2B00000000000000000000000F9
:109AFB00000000000000000000E5732403F8EF25D0
:109B0B00E0F6A8730680AAD2B1C2B3000000000031
:0F9B1B000000000000000000000000000000003B
:079B2A00E5732404F573222A
:10971500157315731573A873C6EBC608C6EAC60894
:09972500C6E9C6E57324FCF573E6
:10972E00C2B10000000000000000000000000000B8
:10973E00000000000000F8087601A873E4F6A87394
:10974E00E6C394085047D2B008E6FF548094004018
:10975E0003D38001C392B30000000000000000009C
:10976E000000000000000000000000C2B000000079
:10977E0000000000000000000000000000000000DB
:0D978E0000A87308EF25E0F6A8730680B16F
:10979B00A87308087605A8730808E6D3940040223E
:1097AB00E5732403F87613E5732403F8E6D39400EA
:1097BB00400900E5732403F81680ECA8730808161B
:0297CB0080D448
:1097CD00A873E4F6E5732404F8CBE6CB08E6FA08B3
:1097DD00E6F9120AD000000000A873E6C3941850F1
:1097ED0070D2B0000000000000000000000000007A
:1097FD0000000000000000E5732404F8CBE6CB0860
:10980D00E6FA08E6F91209837801120970C8ECC866
:10981D00C9EDC9CAEECACBEFCBA2B4E4334BFFEA14
:10982D00FEE9FDE8FCE5732404F8CBE6CB08E6FA87
:10983D0008E6F91209D3C2B00000000000000000D4
:10984D00000000000000000000000000A87306806A
:10985D0088D2B100000000000000000000000000F0
:07986D0000000000000000F4
:07987400E5732407F57322E0
:10719D001573A873EBF61573A873EDF61573A87335
:0871AD00EFF6E57324F6F5731B
:1071B500240BF8E66401600302728CE573240CF875
:1071C500E6FFE573240D12C9507D027F001299DB9D
:1071D5001D7F021299DB7DD07F031299DB7FF012B0
:1071E500B55CE5732404F8120A86000000007FA050
:1071F5007E867D017C00E5732404F8120A15C3120E
:07720500095F505730B5543A
:10720C00E5732408F87601E5732408F8E6D39400B6
:10721C004023E5732409F87603E5732409F8E6D3D3
:10722C009400400900E5732409F81680ECE57324FA
:05723C0008F81680D2E5
:10724100E5732404F81209EDEF2401FFE43EFEE4A6
:107251003DFDE43CFCE5732404F8120A6E80937D45
:107261000F12B550E573240DF8E6FFE573240CF811
:10727100E675F008A42FF582E435F0F583E5822464
:10728100F1F582E583340DF583E4F0E573240BF821
:10729100E664036003027519E573240EF8E6D394DE
:1072A1000740057F0002751BE573240CF8E6FFE536
:1072B10073240D12C950E5732404F8120A860000E4
:1072C1000000E47F107E27FDFCE5732404F8120A18
:0A72D10015C312095F505730B55481
:1072DB00E5732408F87601E5732408F8E6D39400E7
:1072EB004023E5732409F87603E5732409F8E6D304
:1072FB009400400900E5732409F81680ECE573242B
:05730B0008F81680D215
:10731000E5732404F81209EDEF2401FFE43EFEE4D6
:107320003DFDE43CFCE5732404F8120A6E8094E40D
:107330007F107E27FDFCE5732404F8120A15C312A2
:10734000095F7004FF02751BE573240DF8E6FEE586
:1073500073240CF8E675F008A42EF582E435F0F5F8
:1073600083E58224F1F582E583340DF583E0FDE5C4
:1073700073240EF8E66D60057F0002751BE573242B
:107380000DF8E6FFE573240CF8E6FCED045407FD68
:1073900075F008ECA42FF582E435F0F583E582243E
:1073A000F1F582E583340DF583EDF075F008ECA47A
:1073B0002EF582E435F0F583E58224F1F582E5834C
:1073C000340DF583E0C454F0440FFD12B5507B003A
:1073D000E5732404F97A00129715E5732404F81272
:1073E00009ED7808120970EC1203BDA873120A6E39
:1073F000E4FBFA7980784FE8C0E0A8731209EDD079
:10740000E0F81202A7E4FBFA79A0784012019EA8E6
:1074100073120A6EE573240AF8E6B46402803FE54D
:1074200073240AF8E6B4652DE4FBFA79207840E885
:10743000C0E0A8731209EDD0E0F81202A7E4FBFA4D
:1074400079A0784112019EE4FBFA792078C11200FC
:10745000ADA873803EE573240AF8E6B46617A873F6
:10746000E8C0E01209EDE4FBFA7980783F12019E52
:10747000D0E0F8801EE573240AF8E6B46718A87314
:10748000E8C0E01209EDE4FBFA7920784112019E90
:10749000D0E0F8120A6EE573240AF8E6FF6465602E
:1074A00004EFB4672A7F007E407D1C7C46A87312DF
:1074B0000A1512019EE4FBFAF9783F1200AD12039F
:1074C000FBEC1203BD7B007A40791C784680287F54
:1074D000007E507DC37C47A873120A1512019EE4FA
:1074E000FBFAF9783F1200AD1203FBEC1203BD7BEF
:1074F000007A5079C378471202A7A873120A6EA8BF
:10750000731209EDE573240FF8CBE6CB08E6FA0811
:0B751000E6F91209D37F0480027F011E
:07751B00E5732412F5732251
:10838B001573A873EBF61573A873EDF61573A87335
:08839B00EFF6E57324F5F5731C
:1083A300240CF8E66403600302862EE573240FF8B9
:1083B300E6FED3940340057F000286307401C8EEC5
:1083C300C8088002C333D8FCA8730808F675840173
:1083D300E5732403F8120A8600000000A873E4F68C
:1083E300A873E6C3940A400302849BE4F5CCF5CD5D
:1083F300F5C975C804E573240DF8E6FFE573240E8B
:1084030012C950E573240DF8E6FFE573240EF8E670
:10841300FDE4FB12C9557F0012C722E573240DF852
:10842300E6FFE573240EF8E6FD7B00A973097A00E5
:1084330012B424A8730808C9E8C9A87308E65760EA
:1084430005E5C830E7D0E4F5C8E5732403F8E8C0D0
:10845300E01209EDECC0E0EDC0E0EEC0E0EFC0E0FB
:10846300AFCDEFFEADCC7C00E42DFFEC3ECBEFCBEC
:10847300FAE4F9F8D0E0FFD0E0FED0E0FDD0E0FC74
:10848300EF2BFFEE3AFEE93DFDE83CFCD0E0F812AD
:108493000A6EA873060283E3E5C85480FFBF012771
:1084A300E573240BF8E6B4700FE5732407F8120A9A
:1084B30086411FFFFF028611E5732407F8120A861F
:1084C3004479FFFE028611E5732403F81209EDE4F3
:1084D3001203BDECC0E0EDC0E0EEC0E0EFC0E0A8E9
:1084E30073E6FCE41203C7C8ECC8C9EDC9CAEECAF7
:1084F300CBEFCBD0E0FFD0E0FED0E0FDD0E0FC122C
:1085030002A7E4FBFA79C478421202A7E4FBFA79E2
:1085130040784112019EE5732407F8120A6EE57351
:108523002407F8E8C0E01209ED7B007A2479747817
:10853300491202A7D0E0F8120A6EE573240BF8E69D
:1085430064707BCD7ACC798C783F7044E8C0E0E5E9
:10855300732407F81209EDD0E0F81202A77B007A22
:10856300B8790878491202A77B287A6B796E784E1E
:1085730012019EE5732407F8120A6EE5732407F8C7
:10858300E8C0E01209ED7B777ABE799F783D8041A0
:10859300E8C0E0E5732407F81209EDD0E0F8120211
:1085A300A7E4FBFA79AF78451202A77B287A6B79A7
:1085B3006E784E12019EE5732407F8120A6EE57376
:1085C3002407F8E8C0E01209ED7B9A7A9979F978E3
:1085D300401200A9D0E0F8120A6EE4FFFE7D7A7C17
:1085E30044E5732407F8120A1512019EE4FBFAF915
:1085F300783F1200AD1203FBEC1203BDE4FBFA79E2
:108603007A78441202A7E5732407F8120A6EE57319
:108613002407F81209EDE5732410F8CBE6CB08E63E
:0D862300FA08E6F91209D37F0480027F01F6
:07863000E5732413F573222A
:1022C6001573A873EBF61573A873EDF61573A8735B
:0822D600EFF6E57324F0F57347
:1022DE00E5732412F8E675F008A4FFE5732413F8ED
:1022EE00EF26FFE573240DF8EFF6E5732411F8E6FB
:1022FE006404600302241EE5732414F8E67032E5CC
:10230E0073240DF8E625E025E024A1F582E4340DD2
:10231E00F583120A9F42960000E5732415F8CBE66A
:10232E00CB08E6FA08E6F9120AD04296000002241B
:10233E0019E5732414F8E6B40132E573240DF8E6BA
:10234E0025E025E02429F582E4340EF583120A9F58
:10235E0000000000E5732415F8CBE6CB08E6FA087A
:10236E00E6F9120AD000000000022419E5732414C5
:10237E00F8E6B40231E573240DF8E625E025E024F5
:10238E00C1F582E4340DF583120A9F3F800000E50B
:10239E00732415F8CBE6CB08E6FA08E6F9120AD054
:1023AE003F8000008065E5732414F8E6FFB4032B2C
:1023BE00E573240DF8E625E024E1F582E4340DF50D
:1023CE0083E4F0A3743CF0E5732415F8CBE6CB0858
:1023DE00E6FA08E6F9E475F03C802DEFB4042CE53E
:1023EE0073240DF8E625E02471F582E4340FF583AD
:1023FE00E4F0A37405F0E5732415F8CBE6CB08E6FC
:10240E00FA08E6F9E475F00512091C7F00022C2F7C
:10241E00E573240DF8E62481F582E4340FF583E0AC
:10242E0060030224F512C9C2E573240DF8E625E017
:10243E0025E024F9F582E4340DF583E0F8A3E0F904
:10244E00A3E0FAA3E0FBC3EF9BFFEE9AFEED99FD2E
:10245E00EC98FCECC0E0EDC0E0EEC0E0EFC0E0E5D3
:10246E0073240DF8E625E024E1F582E4340DF583BE
:10247E00E0FEA3E0FF7C007D64120806CBEFCBCA22
:10248E00EECAE4F9F8D0E0FFD0E0FED0E0FDD0E0F7
:10249E00FCC312095F40030225D1E573240DF8E653
:1024AE002481F582E4340FF5837401F012C9C2E57C
:1024BE0073240DF8E6FB25E025E024F9F582E434DB
:1024CE000DF583120A7AEB25E025E024A1F582E4CE
:1024DE00340DF583E0FCA3E0FDA3E0FEA3E0FFA82E
:1024EE0073120A6E02259A12C9C2E573240DF8E61C
:1024FE0025E025E024F9F582E4340DF583E0F8A318
:10250E00E0F9A3E0FAA3E0FBC3EF9BFFEE9AFEED2A
:10251E0099FDEC98FCECC0E0EDC0E0EEC0E0EFC041
:10252E00E0E573240DF8E625E02471F582E4340F1E
:10253E00F583E0FEA3E0FF7C007D64120806CBEF7E
:10254E00CBCAEECAE4F9F8D0E0FFD0E0FED0E0FD51
:10255E00D0E0FCC312095F506AE573240DF8E6243F
:10256E0081F582E4340FF583E4F012C9C2E57324D9
:10257E000DF8E625E025E024F9F582E4340DF58327
:10258E00120A7AA873120A8600000000A973157346
:10259E0015731573A873760008760008C6E9C6157C
:1025AE0073A873E4F6E5732417F8E61573A873F6AB
:1025BE00E5732417F8E6FB7D02E5732415F8E6FFB4
:1025CE001222C6E5732411F8E66401600302267137
:1025DE00E5732412F8E6FFE5732413F8E6FD7B0E8F
:1025EE0012B9FEE5732412F8E6FFE5732413F8E63C
:0C25FE00FD7B0E12B2ED12942412987BAB
:10260A00E573240EF87664E573240EF8E6D3940095
:10261A004023E573240FF87603E573240FF8E6D315
:10262A009400400900E573240FF81680ECE5732442
:05263A000EF81680D22D
:10263F007D077F02129886E573240DF8E62481F555
:10264F0082E4340FF5837401F012C9C2E573240DCF
:10265F00F8E625E025E024F9F582E4340DF5831240
:10266F000A7AE5732411F8E664026003022947E54C
:10267F00732414F8E6703FE5732415F8CBE6CB0806
:10268F00E6FA08E6F9120983E4FBFAF9F8120344B3
:10269F005024E5732415F8CBE6CB08E6FA08E6F9E3
:1026AF00120983E573240DF8E625E025E024A1F552
:1026BF0082E4340D8058E5732414F8E6B40124E560
:1026CF00732415F8CBE6CB08E6FA08E6F91209836E
:1026DF00E573240DF8E625E025E02429F582E4349E
:1026EF000E802BE5732414F8E6B40229E573241544
:1026FF00F8CBE6CB08E6FA08E6F9120983E573246E
:10270F000DF8E625E025E024C1F582E4340DF583CC
:10271F00120A7A8062E5732414F8E6FFB4032BE5FE
:10272F00732415F8CBE6CB08E6FA08E6F91208B9D8
:10273F00FDE573240DF8E625E024E1F582E4340D80
:10274F00F583E5F0F0A3EDF0802DEFB40429E573E8
:10275F002415F8CBE6CB08E6FA08E6F91208B9FF1C
:10276F00E573240DF8E625E02471F582E4340FF5C6
:10277F0083E5F0F0A3EFF0E5732414F8E6D39400AB
:10278F0040057F00022C2FE5732415F8CBE6CB080C
:10279F00E6FA08E6F9120983A873120A6EE4FFFE3F
:1027AF00FDFCA873120A151203445009A873120AEC
:1027BF008600000000E4FFFE7DC87C42A873120A69
:1027CF0015120344600B4009A873120A8642C80011
:1027DF0000E4FBFA79C87842E8C0E0A8731209ED6B
:1027EF00D0E0F81202A77B007AFF797F78471201B9
:1027FF009E1203FBE573240AF8EEF608EFF6E57375
:10280F002412F8E6FFE5732413F8E6FDE4FB12B299
:10281F00EDE573240CF8E4F6E573240CF8E6FFC33A
:10282F0094045033EF940140047F0480027F001220
:10283F00B2D1E5732412F8E6FFE5732413F8E6FD31
:10284F00E5732405F8E64408FB12B2ED12B2D8E5A1
:10285F0073240CF80680C1E573240CF8E4F6E573D5
:10286F00240CF8E6C39404504DE5732414F8E65491
:10287F0008D3940040047F0480027F0012B2D1E598
:10288F00732412F8E6FFE5732413F8E6FDE57324CD
:10289F0005F8E64408FB12B2ED12B2D8E573241422
:1028AF00F8E8C0E0E625E0FFD0E0F8EFF6E57324A6
:1028BF000CF80602286DE573240CF8E4F6E5732492
:1028CF000CF8E6C39410505DE573240AF8E65480C3
:1028DF00FED3E49400EE940040047F0480027F0056
:1028EF0012B2D1E5732412F8E6FFE5732413F8E66C
:1028FF00FDE5732405F8E64408FB12B2ED12B2D8D9
:10290F00E573240AF8E8C0E0C9E8C909E725E0FF44
:10291F0019E733FED0E0F8EEF608EFF6E573240C76
:10292F00F8060228CCE5732412F8E6FFE5732413AA
:10293F00F8E6FD7B0E12B2EDE5732411F8E66403A1
:10294F006003022C2DE5732414F8E67013E573244D
:10295F000DF8E625E025E024A1F582E4340D80365C
:10296F00E5732414F8E6B40113E573240DF8E62596
:10297F00E025E02429F582E4340E801AE57324144F
:10298F00F8E6B40221E573240DF8E625E025E024EE
:10299F00C1F582E4340DF583E0FCA3E0FDA3E0FE76
:1029AF00A3E0FF022C14E5732414F8E6FEB4032809
:1029BF00E573240DF8E625E024E1F582E4340DF506
:1029CF0083E0F9A3E0FDE5732415F8CBE6CB08E629
:1029DF00FA08E6C98DF0802AEEB4042EE573240DB3
:1029EF00F8E625E02471F582E4340FF583E0F9A3CE
:1029FF00E0FFE5732415F8CBE6CB08E6FA08E6C945
:102A0F008FF012091C7F02022C2FE5732414F8E6B5
:102A1F00640560057F00022C2FE5732412F8E6FF92
:102A2F00E5732413F8E6FD7B00E5732404F97A00BF
:102A3F0012B424E5732404F8E65401D3940040053E
:102A4F007F00022C2F1294247B00E5732406128F33
:102A5F00507D077F02129886E5732406F81209ED60
:102A6F00E41203BDE4FBFA7980784B1202A77B0ACC
:102A7F007AD779A3784012019E7B0A7AD779237887
:102A8F00C01200ADA873120A6EA873E8C0E0120955
:102A9F00ED7B387A1F7943784112019ED0E0F8120E
:102AAF000A6EA873E8C0E01209EDECC0E0EDC0E0DB
:102ABF00EEC0E0EFC0E0E573240DF8E625E025E079
:102ACF0024A1F582E4340DF583E0FCA3E0FDA3E03F
:102ADF00FEA3E0FFE4FBFA797A78441202A7C8EC70
:102AEF00C8C9EDC9CAEECACBEFCBD0E0FFD0E0FE2C
:102AFF00D0E0FDD0E0FC1202A7D0E0F8120A6E7B06
:102B0F00CD7ACC792C7840E8C0E0A8731209EDD0CB
:102B1F00E0F81202A7C8ECC8C9EDC9CAEECACBEFDC
:102B2F00CBE4FFFE7DC87C421200A9A873120A6E87
:102B3F00E573240DF8E625E025E02429F582E43439
:102B4F000EF583E0F8A3E0F9A3E0FAA3E0FBE8C0F9
:102B5F00E0A8731209EDD0E0F81200A9E573240D77
:102B6F00F8E625E025E024C1F582E4340DF583E095
:102B7F00F8A3E0F9A3E0FAA3E0FB12019EA87312F9
:102B8F000A6E7F007E507DC37C47A873120A151210
:102B9F00019EE4FBFAF9783F1200AD1203FBEC1231
:102BAF0003BD7B007A5079C378471202A7A873122E
:102BBF000A6EE573240DF8E62481F582E4340FF5EF
:102BCF0083E06401705412C9C2E573240DF8E62541
:102BDF00E025E024F9F582E4340DF583E0F8A3E075
:102BEF00F9A3E0FAA3E0FBC3EF9BFFEE9AFEED998A
:102BFF00FDEC98FCE47B64FAF9F8C312095F501AF4
:102C0F00A8731209EDE5732415F8CBE6CB08E6FAA5
:102C1F0008E6F91209D37F0480067F0080027F0146
:072C2F00E5732418F5732280
:108637001573A873EBF61573A873EDF61573A87386
:08864700EFF6E57324F5F5736D
:10864F00E573240CF8E664017021E573240DF8E658
:10865F00FFE573240EF8E6FD7BFF12B2EDE5732400
:10866F000DF8E6FFE573240E12B9F9E573240CF843
:10867F00E6640360030288D0E573240FF8E67012F6
:10868F00E573240DF8E6FFE573240EF8E6FD7BFE97
:10869F008010E573240DF8E6FFE573240EF8E6FD70
:1086AF007BFD12B2EDE573240DF8E6FFE573240EA2
:0386BF0012C9508D
:1086C200E5732409F8760AE5732409F8E6D39400E1
:1086D2004023E573240AF87603E573240AF8E6D307
:1086E2009400400900E573240AF81680ECE573242F
:0586F20009F81680D21A
:1086F70030B418E573240DF8E6FFE573240EF8E6A9
:10870700FD7BFF12B2ED7F000288D2E5732404F8E7
:10871700120A8600000000E5732408F8E4F6E57302
:108727002408F8E6C3941B50750000000000000001
:1087370000000000000000000000000000D2B000B0
:108747000000000000000000000000000000000022
:10875700000000C2B00000000000000000000000A0
:10876700000000000000000000E5732404F812096F
:10877700ED7801120970C8ECC8C9EDC9CAEECACBB9
:10878700EFCBA2B4E4334BFFEAFEE9FDE8FCE57367
:108797002404F8120A6EE5732408F8068080E5734E
:1087A700240DF8E6FFE573240EF8E6FD7BFF12B211
:1087B700EDE5732404F81209EDE4FFFEFDEC540225
:1087C700FC601EE5732404F81209EDE4FFFEFDECDE
:1087D7005401FC600CA873120A864020000002882E
:1087E7006DE5732404F81209EDE4FFFEFDEC540275
:1087F700FCE4FBFAF9F8C312095F701DE573240462
:10880700F81209EDE4FFFEFDEC5401FC600BA873C0
:10881700120A8600000000804DE5732404F812094F
:10882700EDE4FFFEFDEC5402FCE4FBFAF9F8C31299
:10883700095F700CE5732404F81209ED74FF8009D1
:10884700E5732404F81209EDE4FC1203BDE4FBFA16
:108857007980784B1202A7E4FBFA7920784012015D
:108867009EA873120A6EE4FFFEFD7C41A873120AEC
:108877001512019EE4FBFA792078C11200ADA873A6
:10888700120A6E7F007E247D747C49A873120A1534
:1088970012019EE4FBFAF9783F1200AD12B0C57BD6
:1088A700007A24797478491202A7A873120A6EA86D
:1088B700731209EDE5732410F8CBE6CB08E6FA0846
:0B88C700E6F91209D37F0480027F0055
:0788D200E5732413F5732286
:108B1E00E5732412F8E675F003A42421F582E434FB
:108B2E000DF583E0FBA3E0FAA3E0F9E573240DF85D
:108B3E00E675F004A4F58285F0831209A38F4B8E9F
:108B4E004A8D498C48E573240FF8E6FFE57324112E
:108B5E00F8E6FDE5732412F8E6FBE573240DF8E65E
:028B6E00F547C9
:068B70008F448D458B4689
:108B7600E4FFFEFDFCAB4BAA4AA949A848120344F0
:108B86005009E4F54BF54AF549F548E544B4852026
:108B9600E4FFFE7D347C43AB4BAA4AA949A84812A0
:108BA600034460324030E4F54BF54A75493480237E
:108BB600E544B48621E4FFFE7D8C7C43AB4BAA4A98
:108BC600A949A848120344600D400BE4F54BF54A49
:108BD60075498C754843AF4BAE4AAD49AC48E5463E
:108BE60075F008A4254725E025E02471F582E434D4
:108BF6000EF583120A7AE544B48519E4FBFA7993F3
:108C06007842AF4BAE4AAD49AC481202A7E4FBFA34
:108C160079208018E4FBFA79937842AF4BAE4AADDF
:108C260049AC481202A77B6F7A1279837840120208
:108C3600A77B007AFF797F784712019E1203FB8E8D
:108C46004C8F4D7B48AD46AF4512B2ED7B06AD4627
:108C5600AF4512C955E4FDEDD394014003D380011D
:108C6600C392B300000000000000000000000000F6
:108C760000000000000000D2B0000000000000006C
:108C860000000000000000000000000000C2B00D5F
:108C9600BD04C4E4FDE5475408D394004003D380E3
:108CA60001C392B3000000000000000000000000B5
:108CB6000000000000000000D2B00000000000002C
:108CC6000000000000000000000000000000C2B02C
:108CD600E54725E0F5470DBD04BBE4FDE54C5480B2
:108CE600FED3E49400EE94004003D38001C392B314
:108CF600000000000000000000000000000000006E
:108D060000000000D2B000000000000000000000DB
:108D160000000000000000000000C2B0E54D25E0A4
:108D2600F54DE54C33F54C0DBD10B17B40AD46AF6E
:048D36004502B2ED53
:0EABDC00E5732411F8E6FFE5732412F8E6FD98
:10ABEA008F448D457B7812B9FEE4FBAD45AF441224
:02ABFA00B2EDBA
:0DABFC0075466475470300D547FCD546F645
:10AC09007B40AD45AF4412B2ED7B70AD45AF441208
:10AC1900B2ED7B06AD45AF4412C95512987B7D1143
:05AC29007F0712988670
:0DAC2E0075466475470300D547FCD546F612
:10AC3B007D577F0212988675F008E544A42545F5EB
:10AC4B0082E435F0F583E5822419F582E583340E31
:10AC5B00F583E4F075F008E544A42545F582E43569
:10AC6B00F0F583E5822421F582E583340EF583E448
:10AC7B00F07B40AD45AF4412B2ED12C9C2E544754D
:10AC8B00F008A4254525E025E02461F582E4340D88
:10AC9B00F583120A7A12C9C2E54475F008A425455A
:10ACAB0025E025E02451F582E4340EF583020A7A7F
:10353C001573A873EBF61573A873EDF61573A873D2
:08354C00EFF6E57324F1F573BD
:10355400E5732411F8E6FF75F008A4FEE573241260
:10356400F8E6FD2EFEE573240EF8EEF6E57324105E
:10357400F8E6B4011212ABEA7E017F007D007B0104
:103584007A0C7921120C66E5732410F8E664026063
:1035940003023639E5732413F8E6FED39407400595
:1035A4007F00023E19EE7029E5732414F8CBE6CBB4
:1035B40008E6FA08E6F9E5732412F8E675F003A4C0
:1035C4002421F582E4340DF583EBF0A3EAF0A3E9BA
:1035D400F0E5732414F8CBE6CB08E6FA08E6F91212
:1035E4000983E4FBFA798078BF1200ADA873120A4C
:1035F4006EE573240FF8E6FFEFC0E0E5732411F8DD
:10360400E6FDEDC0E0E5732412F8E6FBE573241350
:10361400F8E6F547A8731209ED8F4B8E4A8D498C55
:1036240048D0E0FDD0E0FF128B7012C9C28F178E14
:10363400168D158C14E5732410F8E66403600302F8
:103644003E17E5732413F8E6FFC394084006EFD34E
:10365400941740057F00023E19E5732411F8E6FF34
:10366400E573241212B418E5732408F8E65401D360
:103674009400407C12C9C2ECC0E0EDC0E0EEC0E0B2
:10368400EFC0E0E5732411F8E675F008A4FFE573D4
:103694002412F8EF2625E025E02461F582E4340DB8
:1036A400F583E0FCA3E0FDA3E0FEA3E0242CFBEE05
:1036B4003401FAE43DF9E43CF8D0E0FFD0E0FED078
:1036C400E0FDD0E0FCC312095F502512ABDCE573CA
:1036D400240DF8E4F6E573240DF8E6C39408500BC2
:1036E400128B1EE573240DF80680EA7F00023E1952
:1036F400E5732408F8E65402D39400407C12C9C24E
:10370400ECC0E0EDC0E0EEC0E0EFC0E0E5732411F2
:10371400F8E675F008A4FFE5732412F8EF2625E017
:1037240025E02451F582E4340EF583E0FCA3E0FDAA
:10373400A3E0FEA3E0242CFBEE3401FAE43DF9E41B
:103744003CF8D0E0FFD0E0FED0E0FDD0E0FCC312B6
:10375400095F502512ABDCE573240DF8E4F6E5733C
:10376400240DF8E6C39408500B128B1EE573240D48
:10377400F80680EA7F00023E19E5732408F8E63073
:10378400E003023B6CE5732412F8E6FFE5732411B1
:10379400F8E675F008A42FF582E435F0F583E582A8
:1037A4002419F582E583340EF583E02408FFE4331D
:1037B400FEE5732413F8E66F7001EE60057F0002E6
:1037C4003E1912C9C2EFC0E0E5732411F8E6F97599
:1037D400F008A4FFE5732412F8E6FB2F25E025E0AA
:1037E4002461F582E4340DF583D0E0FF120A7ACF28
:1037F400E9CFCDEBCD7B5012B2EDE5732411F8E6A1
:10380400FFE573241212942F128F4AE5732412F8E1
:10381400E6FFE5732411F8E6FE75F008A42FF5829F
:10382400E435F0F583E5822419F582E583340EF559
:1038340083E0045407FD75F008EEA42FF582E43507
:10384400F0F583E5822419F582E583340EF583EDE2
:10385400F0E5732412F8E6FFE5732411F8E675F039
:1038640008A42FF582E435F0F583E5822419F58266
:10387400E583340EF583E0904D6493C454F044071B
:10388400FD7F02129886E5732411F8E6FFE57324A0
:1038940012F8E6FD7B4012B2EDE573240FF8E6B4AE
:1038A4008529E5732409F81209EDE41203BDE4FB4C
:1038B400FA7980784B1202A77B0A7AD779A37840E9
:1038C40012019E7B0A7AD779238030E573240FF89E
:1038D400E6B48633E5732409F81209EDE41203BD56
:1038E400E4FBFA7980784B1202A77B587A3979067F
:1038F400784112019E7B3F7A35798678C01200ADFB
:10390400A873120A6E8009A873120A8600000000C8
:10391400A873E8C0E01209EDE4FBFA79CA78421210
:10392400019ED0E0F8120A6EE5732412F8E675F0F1
:1039340008A4FFE5732413F8E67C002FFFEC35F0B0
:10394400FEEF7802C333CE33CED8F92401F5827466
:103954000C3EF583E0FCA3E0FDA3E0FEA3E0FFE55D
:10396400732404F8120A6EE4FFFE7D807CBFE573C5
:103974002404F8120A151203446048A873E8C0E04E
:103984001209EDECC0E0EDC0E0EEC0E0EFC0E07F76
:103994000A7ED77D237C3CE5732404F8120A1512B1
:1039A400019EC8ECC8C9EDC9CAEECACBEFCBD0E0C2
:1039B400FFD0E0FED0E0FDD0E0FC1200A9D0E0F89A
:1039C400120A6EE4FFFE7D7A7C44A873120A151273
:1039D400019EE4FBFAF9783F1200AD1203FBEC12EE
:1039E40003BDE4FBFA797A78441202A7A873120A99
:1039F4006EA8731209EDE5732414F8CBE6CB08E640
:103A0400FA08E6F91209D312C9C2C8ECC8C9EDC94B
:103A1400CAEECACBEFCBE5172432FFE43516FEE439
:103A24003515FDE43514FCD312095F5003023B67DE
:103A3400E5732413F8E624F8FFE434FFFEEF78027C
:103A4400C333CE33CED8F9FFE5732412F8E675F00C
:103A540003A42421F582E4340DF583E0FBA3E0FA0A
:103A6400A3E0F98F828E83120A3EE8C0E0A87312A5
:103A740009EDD0E0F81200A9E5732404F8120A6EE7
:103A8400E5732404F81209ED12CA5F7B6F7A127988
:103A940083783A1203444003023B67E5732404F835
:103AA4001209ED12CA5FE4FBFA792078411203444B
:103AB40060025003023B67E4FFFEFD7C40E5732493
:103AC40004F8120A15120344600E400CE573240432
:103AD400F8120A8640000000E4FFFEFD7CC0E57396
:103AE4002404F8120A15120344500CE5732404F854
:103AF400120A86C0000000E5732412F8E675F00887
:103B0400A4FFE5732413F8E67C002FFFEC35F0FEE8
:103B1400EF7802C333CE33CED8F92451F582740E34
:103B24003EF583E0FCA3E0FDA3E0FEA3E0FFE57324
:103B34002404F8120A151200A98F4B8E4A8D498C61
:103B440048E573240FF8E6FFE5732411F8E6FDE574
:103B5400732412F8E6FBE5732413F8E624F8F5471A
:103B6400128B707F04023E19E5732408F8E630E1F5
:103B740003023E13E5732412F8E6FFE5732411F8FB
:103B8400E675F008A42FF582E435F0F583E5822488
:103B940021F582E583340EF583E02410FFE433FE3F
:103BA400E5732413F8E66F7001EE60057F00023EB2
:103BB4001912C9C2EFC0E0E5732411F8E6F975F0F3
:103BC40008A4FFE5732412F8E6FB2F25E025E02482
:103BD40051F582E4340EF583D0E0FF120A7ACFE97E
:103BE400CFCDEBCD7B6012B2EDE5732411F8E6FF87
:103BF400E573241212942F128F4AE5732412F8E607
:103C0400FFE5732411F8E6FE75F008A42FF582E4AD
:103C140035F0F583E5822421F582E583340EF583BE
:103C2400E0045407FD75F008EEA42FF582E435F0A6
:103C3400F583E5822421F582E583340EF583EDF0E6
:103C4400E5732412F8E6FFE5732411F8E675F0082D
:103C5400A42FF582E435F0F583E5822421F582E58D
:103C640083340EF583E0904D6C93C454F04406FD08
:103C74007F02129886E5732411F8E6FFE573241297
:103C8400F8E6FD7B4012B2EDE5732413F8E624F068
:103C9400FFE434FFFEEF7802C333CE33CED8F9FF0E
:103CA400E5732412F8E675F003A42421F582E434C4
:103CB4000DF583E0FBA3E0FAA3E0F98F828E831273
:103CC40009A3E4FBFA79707841120344600E400CB6
:103CD400A873120A86BF800000023DADE573240F6D
:103CE400F8E6B4852BE5732409F81209EDE4120310
:103CF400BDE4FBFA7980784B1202A77B0A7AD77964
:103D040023784012019E7B0A7AD779A378BF803248
:103D1400E573240FF8E6B48633E5732409F8120931
:103D2400EDE41203BDE4FBFA7980784B1202A77B21
:103D3400DD7A247986784012019E7BDD7A24790627
:103D440078C01200ADA873120A6E8009A873120A13
:103D540086000000007B007A40791C7846E8C0E0C9
:103D6400A8731209EDD0E0F81202A77B007A247937
:103D740074784912019EA873120A6EE4FFFE7D7ADC
:103D84007C44A873120A1512019EE4FBFAF9783FE9
:103D94001200AD1203FBEC1203BDE4FBFA797A784E
:103DA400441202A7A873120A6EA8731209EDECC09C
:103DB400E0EDC0E0EEC0E0EFC0E0E5732412F8E609
:103DC40075F008A4FFE5732413F8E67C002FFFECDC
:103DD40035F0FEEF7802C333CE33CED8F924E1F5C3
:103DE40082740B3EF583D0E0FFD0E0FED0E0FDD03E
:103DF400E0FC120A7AA8731209EDE5732414F8CBD7
:103E0400E6CB08E6FA08E6F91209D37F0480067FB8
:053E14000080027F01A7
:073E1900E5732417F5732285
:104D7400506C6561736520696E73657274206D6F24
:104D840064756C6500202755696E202B2D313056D3
:104D9400272028307836312920002020202020693F
:104DA4006E746F20706F72742030202020200020D9
:104DB40027446F75742032345627202830783430D5
:104DC400292020002020202020696E746F20706F1D
:104DD40072742034202020200020202744696E2073
:104DE40035562720283078343029202020002020F0
:104DF400202020696E746F20706F7274203520201B
:104E040020200020002A2A2000202A2A00202041D5
:104E14006464726573733A2020202530345800206E
:104E2400205265766973696F6E3A202025730020DD
:104E3400202020202020202020202020202020206E
:104E44002020200057726F6E672043504C44206628
:104E540069726D7761726500536C61766520616477
:104E640064723A20256264005265713A202530321A
:104E7400626420213D204163743A2025303262640B
:104E8400004F76657263757272656E74203E312EC2
:104E94003541206F6E00202020323456206F757407
:104EA4007075742021212120202000202020536CA3
:104EB40061766520616464723A202562640052451B
:104EC400534554004F76657263757272656E742033
:104ED4003E302E3541206F6E002020202035562094
:104EE4006F757470757420212121002020202053B7
:104EF4006C61766520616464723A202562640020E6
:104F040020202055203D2025312E326620560025B4
:104F14003033426430302530336430323D3F002535
:104F2400303342640D002530334264313025303350
:104F34006430362530366C640025303342643130B9
:104F44002530336430332530336C640050312A3AD1
:104F54002025392E3245206D6261720050313A208D
:104F64002531302E3245206D6261720050322A3A6A
:104F74002025392E3245206D6261720050323A206C
:104F84002531302E3245206D626172004552524FF8
:104F9400523A20747572626F20636F6D6D2E2020FB
:104FA400004552524F523A20666F72652076616313
:104FB4006375756D20004552524F523A206D6169F8
:104FC4006E207661636375756D2000544D502045E5
:104FD40052524F523A2025732020202000544D5025
:104FE4003A2025346420487A2C2025342E32662039
:104FF4004100526D7020646F776E20544D503A25F5
:10500400346420487A0050756D702073746174693B
:105014006F6E206F666620202020005374617274C6
:10502400696E6720666F72652070756D7020200050
:1050340050756D70696E672062756666657220745E
:10504400616E6B200050756D70696E6720726563C8
:10505400697069656E7420202000565030005650E7
:105064003100565630200056563120004856300044
:105074004856310042563000425631004F464600F1
:105084004F4E2000554E4C4F434B00204C4F434B4A
:1050940020002020202020202020002532626400CF
:1050A40050554D502D53544154494F4E002449649A
:1050B400240001340000004572726F720000000188
:1050C40011220000000000000000000000000000A9
:1050D4000000013200000053746174696F6E0001B6
:1050E400112300000000003F8000003F800000000A
:1050F400000001320000004C6F636B656400000126
:10510400112400000000003F8000003F80000000E8
:1051140000000132000000566163204F4B00000183
:10512400112500000000003F8000003F80000000C7
:10513400000001320000004D616E4D6F6465000196
:10514400112600000000003F8000003F80000000A6
:1051540000000132000000466F726570756D7001C9
:10516400112700000000003F8000003F8000000085
:1051740000000132000000466F7265766C76000113
:10518400112800000000003F8000003F8000000064
:10519400000001320000004D61696E766C760001FA
:1051A400112900000000003F8000003F8000000043
:1051B40000000132000000427970766C7600000134
:1051C400112A00000000003F8000003F8000000022
:1051D40000000132000000547572626F206F6E018E
:1051E400112B00000000003F8000003F8000000001
:1051F40000000214000000526F7453706400000138
:10520400112C00000000000000000000000000005D
:1052140000000406000001544D5063757200000143
:10522400112E00000000000000000000000000003B
:10523400000001320000005650206F6E0000000193
:105244001132000000000000000000000000000017
:10525400000001320000005656206F70656E000198
:1052640011330000000000000000000000000000F6
:1052740000000132000000565620636C6F73650114
:1052840011340000000000000000000000000000D5
:10529400000001320000004856206F70656E000166
:1052A40011350000000000000000000000000000B4
:1052B40000000132000000485620636C6F736501E2
:1052C4001136000000000000000000000000000093
:1052D400000001320000004256206F70656E00012C
:1052E4001137000000000000000000000000000072
:1052F40000000132000000425620636C6F736501A8
:105304001138000000000000000000000000000050
:1053140000000416FD0001485600000000000001D2
:10532400113900000000000000000000000000002F
:1053340000000416FD0001565600000000000001A4
:10534400113D00000000000000000000000000000B
:105354000000021400000846696E537064000001E6
:1053640011420000000000000000000000000000E6
:105374000000013400000850425200000000000107
:1053840011410000000000000000000000000000C7
:105394000000020400000854696D656F7574000113
:1053A400114400000000004396000041200000006A
:1053B400000002030000084650206379636C650115
:1053C4001146004120000044160000412000000066
:1053D40000000416FD00095656206D617800000196
:1053E4001148013F800000412000003F8000000080
:1053F40000000416FD00095656206D696E00000178
:10540400114C013DCCCCCD3F8000003DCCCCCD0037
:1054140000000416FD000948562074687273680180
:105424001150033A83126F3F8000003A83126F00D9
:105434000000013400000853746174650000000129
:1054440011540000000000000000000000000000F3
:1054540000000A38000008544D50457272000001E3
:1054640011550000000000000000000000000000D2
:105474000000000000000000000000000000000028
:105484000000000000000000000000000000000018
:02549400000016
:10C24900017A010318FF50B6C113C112C114C115F7
:10C25900C108C109C10AC10BC10CC10D4110DDFFE3
:07C269004410DE000000009C
:109DBC0075840F75A4F575A5FF75A6FF75A70FE43F
:109DCC00F584F5BA75BC9875E880F5D1F58475D134
:109DDC0003F58475D48075840175D480FDFF12C998
:109DEC009B7B61E4FDFF12C5BFEF70297BFF7A4DB1
:109DFC0079741269E57BFF7A4D79891269E57BFFED
:109E0C007A4D799E1269E5E4FF12BF92EF7006FF5E
:109E1C0012C72280F27B407D04E4FF12C5BFEF70B5
:109E2C00297BFF7A4D79741269E57BFF7A4D79B302
:109E3C001269E57BFF7A4D79C81269E5E4FF12BF20
:109E4C0092EF7006FF12C72280F27B207D05E4FFA3
:109E5C0012C5BFEF70297BFF7A4D79741269E57BCF
:109E6C00FF7A4D79DD1269E57BFF7A4D79F2126943
:109E7C00E5E4FF12BF92EF7006FF12C72280F212C8
:109E8C00BDEC157315731573A8737600087600086E
:109E9C0076001573A873E4F61573A873F6FB7D01B1
:109EAC007F61126DF2157315731573A87376000824
:109EBC0076000876001573A873E4F61573A873760C
:109ECC0004FB7D017F401295A1157315731573A8C2
:109EDC007376000876000876001573A873E4F615FF
:0D9EEC0073A8737605FB7D017F2002A7039C
:0290F1008F44AA
:1090F3007D017F0012C6F57D007F0112C6F5E49065
:109103001164F0901164E0FFC39403500B12AF4F4E
:10911300901164E004F080EB120003E5446042E444
:10912300901123F0A3F0A3F0A3F0A3F0A3F0A3F016
:10913300A3F0901141F0901144F0A3743CF0A3E428
:10914300F0A37414F0A3120A9F4080000090114C06
:10915300120A9F3ECCCCCD901150120A9F3A831233
:109163006F9011547401F0E4FF12CA78E4FF12CA3D
:1091730082E4FF120019E4FF12CA28E4901164F09C
:10918300901164E0FFC39414500B12C9159011643D
:10919300E004F080EB7D037F0112C2947B017A111E
:1091A30079657F3B7E0112A2AA7B017A1179651250
:1091B300B223901142EEF0A3EFF0754B07754AB25C
:1091C3007549017548007D067F177E0012ACC2E425
:1091D300FDFF12C99BE4901164F07B007A00799241
:1091E30012C9867C007D0212086DC374079FFFE4D9
:1091F3009EFE901164E0C39FEE6480F874809850E3
:10920300117BFF7A4E790712C779901164E004F05D
:1092130080C87BFF7A4E790912C7797B007A00797F
:109223009212C7797BFF7A4E790D12C7797D01E4DB
:10923300FF12C99B7BFF7A4E7911788CE6F54F08B4
:10924300E6F5501269E57D02E4FF12C99B78657C5F
:10925300117D017BFF7A5079C6120C497B017A118B
:1092630079657D2012C8ACE41207D2754F017550A1
:10927300117551657BFF7A4E79231269E57D03E40D
:10928300FF12C99B7BFF7A4E79331269E5E4901193
:0292930022F0C7
:0192950022B6
:07BF8B00EF24FF92107F0379
:10BF9200E4F58420130FD213F58475D103F5BA7535
:0DBFA200BC9875E880C374079F5407F5BB79
:0DBFAF0075440275451300D545FCD544F6D8
:10BFBC00C2AFC2EDD2EC30EDFDD2AFAFBFEFFFADF3
:10BFCC00BEED90119ECFF0A3EFF0C3E094E890117A
:0CBFDC009EE0940350047F0180027F006F
:01BFE8002236
:1080D800E4901197F012C9C2C8ECC8C9EDC9CAEE3C
:1080E800CACBEFCB9010D9E0FCA3E0FDA3E0FEA340
:1080F800E0240AFFE43EFEE43DFDE43CFCD3120923
:108108005F501A12C9C29010D9E0F8A3E0F9A3E0B1
:10811800FAA3E0FBD312095F500302837612C9C2A7
:108128009010D9120A7AE4901198F0901198E0FF13
:10813800C3940140030283857B017A11799612B7B3
:10814800B6901196E0C4540F640260617A007B64B3
:108158007D017F0112B84820154B12CA52E4FDFF79
:1081680012C99B7BFF7A4E794812C7797D01E4FFDB
:1081780012C99B901198E0FFD39400400B7BFF7AC3
:108188004E795C8F4F1269E57D02E4FF12C99B7B33
:10819800FF7A4E796C754F02901196E0FFC4540F28
:1081A800F5501269E5D2159011977401F090119865
:1081B800E0FF754201754311754499754503E4FB69
:1081C8007D01129EF9901199E020E3030282587A0A
:1081D800007B647D017F0112B84820144E12CA52F8
:1081E800E4FDFF12C99B7BFF7A4E79851269E57D14
:1081F80001E4FF12C99B7BFF7A4E799A1269E57DEB
:1082080002E4FF12C99B901198E0FFD39400400B41
:108218007BFF7A4E79AF8F4F1269E57D037F0F128E
:10822800C99B7BFF7A4E79C21269E5D2147F03128B
:10823800BF92EF6015901198E0FF12C871C2147FC9
:108248000312BF92EF70F812CA529011977401F09E
:1082580012C9C2E47B64FAF9F8C312095F40030249
:10826800836D901198E0FF75420175431175449C28
:108278007545027B037D02129EF990119CE0C4F8BB
:1082880054F0C868FCA3E0C4540F48FDE41203C2CC
:10829800E4FBFA79C8784012019EE4FBFA79807809
:1082A800451202A7E4FBFA79907840120344600271
:1082B800500302835920124912CA527A007B647D06
:1082C800017F0112B848E4FDFF12C99B7BFF7A4E7B
:1082D80079C81269E57D01E4FF12C99B7BFF7A4EDC
:1082E80079DD1269E57D02E4FF12C99B901198E0DF
:1082F800FFD39400400B7BFF7A4E79EF8F4F1269C2
:10830800E57D03E4FF12C99B90119CE0C4F854F08A
:10831800C868FCA3E0C4540F48FDE41203C2E4FBA0
:10832800FA79C8784012019EE4FBFA798078451200
:1083380002A78F528E518D508C4F7BFF7A4F790355
:108348001269E5D2129011637401F0901197F080D0
:1083580014301211901198E0FF901163E06F7005CE
:10836800C21212CA52901198E004F002813320140C
:10837800062012033015069011977401F09011979A
:02838800E0FF14
:01838A0022D0
:08A2A2007B017A1179647E0151
:0AA2AA008E458F468B478A4889498C
:10A2B40012C466754FFF75504F7551137552018561
:10A2C40045538546547B017A1179891269DFE490FC
:10A2D40011ABF09011A9F09011A9E0FFC3940C50B8
:10A2E4001A74892FF582E43411F583E0FF9011ABE1
:10A2F400E02FF09011A9E004F080DC754FFF755059
:10A304004F7551239011ABE0F5527B017A11799589
:10A314001269DFE49011A9F07B017A11798912C9DD
:10A32400869011A9E0FDC39FEE6480F87480985074
:10A334001774892DF582E43411F583E0FF12C53ECC
:10A344009011A9E004F080D012C8147B017A11792D
:10A35400897550147D2012B9699011A9EFF0D39436
:10A36400024057901191E024D075F00AA4FFA3E0B5
:10A3740024D02F9011ACF0E49011AAF09011ACE02D
:10A38400FF9011AAE0FEC39F502174932EF582E43E
:10A394003411F583E0AB47AA48A9498E827583003E
:10A3A4001207E49011AAE004F080D1AB47AA48A9AF
:0CA3B400498E82758300E40207E47F00FC
:01A3C000227A
:07ACBB00F5487D067F0CFE49
:06ACC2008E458F468D4710
:10ACC80012C466E547B4060B754FFF75504F7551B2
:10ACD8002A800EE547B40327754FFF75504F75510D
:10ACE8003D755201854553854654854B58854A57CD
:10ACF8008549568548557B017A1179961269DFE4B2
:10AD08009011B7F09011B6F09011B6E0FFC394100F
:10AD1800501A74962FF582E43411F583E0FF9011F0
:10AD2800B7E02FF09011B6E004F080DC754FFF75A6
:10AD3800504F7551239011B7E0F5527B017A117984
:10AD4800A61269DFE49011B6F07B017A11799612A8
:10AD5800C9869011B6E0FDC39FEE6480F8748098B0
:10AD6800501774962DF582E43411F583E0FF12C56F
:10AD78003E9011B6E004F080D012C8147B017A111D
:0FAD880079967550327D2012B9699011B6EFF0AF
:01AD97002299
:10C915001573A873EFF6A873E624E2F582E43410E4
:08C92500F5837401F005732293
:05CA8C008F397F00223C
:10C6C8008B398A3A893B12078CAB3CAA3DA93E12AA
:10C6D80007D2AB39AA3AA93B9000011207A5AB3C97
:0DC6E800AA3DA93E9000011207E47F022246
:07CA2100E4FF12CA78E4FFF4
:0ACA2800901127EFF07F0502C915F9
:0ACA7800901128EFF07F0602C915A7
:0ACA8200901129EFF07F0702C9159B
:0B000E00FF12CA78E4FF12CA82E4FF70
:0A00190090112AEFF07F0802C915CC
:100D0D0030160312CA52E4FDFF12C99B901127E061
:100D1D00600CA3E060087BFF7A4F795080067BFF63
:100D2D007A4F796090113DE0FCA3E0FDA3E0FEA3B6
:100D3D00E0F5528E518D508C4F1269E57D01E4FF27
:100D4D0012C99B90112BE0600A901129E07010A33D
:100D5D00E0700C901127E0600E90112AE060087B86
:100D6D00FF7A4F797080067BFF7A4F798090113929
:100D7D00E0FCA3E0FDA3E0FEA3E0F5528E518D5003
:100D8D008C4F1269E5901122E0600B7A007B647D37
:100D9D00017F0112B8487D02E4FF12C99B90112218
:100DAD00E030E0097BFF7A4F7990020E9790112287
:100DBD00E030E1097BFF7A4F79A5020E9790112261
:100DCD00E030E2097BFF7A4F79BA020E979011223B
:100DDD00E030E312754F017550117551557BFF7A57
:100DED004F79CF020E97901126E060257BFF7A4F49
:100DFD0079E190112CE0F54FA3E0F550A3E0FCA3B1
:100E0D00E0FDA3E0FEA3E0F5548E538D528C51808E
:100E1D0079901154E0B40124D390112DE0940A90EF
:100E2D00112CE094007BFF400D7A4F79F6E0F54FE1
:100E3D00A3E0F55080547A50790A804E901154E019
:100E4D00B402087BFF7A50791F803F901154E0B4B3
:100E5D0003087BFF7A5079348030901154E07BFF8A
:100E6D00B405067A50794980217A4F79E190112C99
:100E7D00E0F54FA3E0F550A3E0FCA3E0FDA3E0FEF9
:100E8D00A3E0F5548E538D528C511269E5901126C5
:100E9D00E07003020FA27D03E4FF12C99B9011279E
:100EAD00E07BFF60067A50795E80047A5079621299
:100EBD0069E57D037F0512C99B901128E07BFF60DA
:100ECD00067A50796680047A50796B1269E57D0354
:100EDD007F0B12C99B901129E07BFF60067A507938
:100EED007080047A5079741269E57D037F1012C900
:100EFD009B90112AE07BFF60067A50797880047A06
:100F0D0050797C1269E5300E14200811901127E0FC
:100F1D0070047F0180027F00901127EFF0300F14D5
:100F2D00200911901128E070047F0180027F00904C
:100F3D001128EFF0301014200A11901129E07004DF
:100F4D007F0180027F00901129EFF0301114200BEA
:100F5D001190112AE070047F0180027F0090112A08
:100F6D00EFF07F0512C9150F12C9150F12C9150F14
:100F7D0012C91520100302102C20110302102C7F12
:100F8D000212BF9212BF8BEF24FF92112010F0209E
:100F9D0011ED7F01227D03E4FF12C99B901123E027
:100FAD007BFF60067A50798080047A5079841269CB
:100FBD00E57D037F0412C99B901124E07BFF600641
:100FCD007A50798880047A50798F1269E57BFF7A9F
:100FDD005079961269E57BFF7A50799F901154E014
:100FED00F54F1269E5300E14200811901123E070B1
:100FFD00047F0180027F00901123EFF0300F142049
:10100D000911901124E070047F0180027F0090117E
:10101D0024EFF0201609201106300B037F0122A2C8
:10102D000E9208A20F9209A210920AA211920B9091
:10103D001123E06024200C21E4F54BF54AF549120B
:10104D00ACBB1200127F0112CA289011547402F029
:10105D0012C9C290115F120A7A901154E0B4024382
:10106D0012C9C2C8ECC8C9EDC9CAEECACBEFCB9044
:10107D00115FE0FCA3E0FDA3E0FEA3E024DCFFEEA6
:10108D003405FEE43DFDE43CFCD312095F40147FC2
:10109D000112CA7812C9C290115F120A7A901154C6
:1010AD007403F0901154E0B4034312C9C2C8ECC8E4
:1010BD00C9EDC9CAEECACBEFCB90115FE0FCA3E03E
:1010CD00FDA3E0FEA3E02490FFEE345FFEE43DFDC2
:1010DD00E43CFCD312095F4014901154740CF09051
:1010ED0011227402F012CA21E4FF1200199011545A
:1010FD00E06403600302118690114CE0FCA3E0FD57
:10110D00A3E0FEA3E0FF90113DE0F8A3E0F9A3E01A
:10111D00FAA3E0FB1203445060E4FFFE7D807C3FA8
:10112D00901139E0F8A3E0F9A3E0FAA3E0FB120374
:10113D0044501112C9C290115F120A7A9011547461
:10114D0005F08035901124E0601B90112B7401F097
:10115D00FF12CA7812C9C290115F120A7A90115407
:10116D007407F08014E4FF12CA789011547404F0DF
:10117D0012C9C290115F120A7A901154E0B404435F
:10118D0012C9C2C8ECC8C9EDC9CAEECACBEFCB9023
:10119D00115FE0FCA3E0FDA3E0FEA3E024F4FFEE6D
:1011AD003401FEE43DFDE43CFCD312095F40147FA5
:1011BD000112001912C9C290115F120A7A901154CE
:1011CD007405F0901154E06405706BD3901145E0F7
:1011DD009400901144E09400405C12C9C2ECC0E050
:1011ED00EDC0E0EEC0E0EFC0E0901144E0FEA3E002
:1011FD00FF7C177D70120B5090115FE0F8A3E0F9A2
:10120D00A3E0FAA3E02FFBEA3EFAE93DF9E83CF84A
:10121D00D0E0FFD0E0FED0E0FDD0E0FCC312095FCE
:10122D005014901154740CF09011227404F0E4FFDA
:10123D0012001912CA21901154E0B4052EE4FFFEDC
:10124D007D807C3F901139E0F8A3E0F9A3E0FAA38B
:10125D00E0FB1203445014E4FF12001912C9C290AE
:10126D00115F120A7A9011547406F0901154E0B483
:10127D00063312C9C2C8ECC8C9EDC9CAEECACBEF54
:10128D00CB90115FE0FCA3E0FDA3E0FEA3E024C83A
:10129D00FFE43EFEE43DFDE43CFCD312095F400556
:1012AD007F0112CA78901154E0B4066512C9C2C804
:1012BD00ECC8C9EDC9CAEECACBEFCB90115FE0FC0B
:1012CD00A3E0FDA3E0FEA3E02490FFEE3401FEE4D5
:1012DD003DFDE43CFCD312095F403690114CE0FC1F
:1012ED00A3E0FDA3E0FEA3E0FF90113DE0F8A3E035
:1012FD00F9A3E0FAA3E0FB120344501590112B74EF
:10130D0001F012C9C290115F120A7A90115474073C
:10131D00F0901154E064076014E06408600FE0641D
:10132D0009600AE0640A6005E0640B7041E4FFFEA9
:10133D007D807C40901139E0F8A3E0F9A3E0FAA399
:10134D00E0FB12034460274025901124E0701FFF3D
:10135D0012CA82E4FF12CA78E490112BF090112387
:10136D00E0600BC20C9011547401F07F00229011BB
:10137D0024E07037901154E0B40730E4FFFE7D8017
:10138D007C3F901139E0F8A3E0F9A3E0FAA3E0FB6C
:10139D0012034460164014E4FF12CA7812C9C290B9
:1013AD00115F120A7A9011547404F0901124E060C8
:1013BD0003021469901154E06407600302146990EC
:1013CD001142E0FCA3E0FDE41203C27BCD7ACC799F
:1013DD004C783F12019EECC0E0EDC0E0EEC0E0EFB6
:1013ED00C0E090112CE0FCA3E0FDE41203C2C8ECB8
:1013FD00C8C9EDC9CAEECACBEFCBD0E0FFD0E0FE35
:10140D00D0E0FDD0E0FC1203446051404FE4FFFEFC
:10141D007D807C3F901139E0F8A3E0F9A3E0FAA3B9
:10142D00E0FB120344503590114CE0FCA3E0FDA30A
:10143D00E0FEA3E0FF90113DE0F8A3E0F9A3E0FA90
:10144D00A3E0FB12034450147F0112CA8212C9C2D9
:10145D0090115F120A7A9011547408F0901124E0E3
:10146D00640160030214FD901154E06407600302EF
:10147D0014FD901142E0FCA3E0FDE41203C27BCD0C
:10148D007ACC794C783F12019EECC0E0EDC0E0EED5
:10149D00C0E0EFC0E090112CE0FCA3E0FDE41203EE
:1014AD00C2C8ECC8C9EDC9CAEECACBEFCBD0E0FFBC
:1014BD00D0E0FED0E0FDD0E0FC12034460324030BD
:1014CD0090114CE0FCA3E0FDA3E0FEA3E0FF901122
:1014DD003DE0F8A3E0F9A3E0FAA3E0FB12034450CA
:1014ED000F12C9C290115F120A7A9011547408F04C
:1014FD00901154E0640860030215E7901142E0FC7E
:10150D00A3E0FDE41203C27BCD7ACC794C783F1277
:10151D00019EECC0E0EDC0E0EEC0E0EFC0E0901148
:10152D002CE0FCA3E0FDE41203C2C8ECC8C9EDC970
:10153D00CAEECACBEFCBD0E0FFD0E0FED0E0FDD0BD
:10154D00E0FC1203445014E4FF12CA8212C9C29087
:10155D00115F120A7A9011547407F012C9C2ECC0CF
:10156D00E0EDC0E0EEC0E0EFC0E0901146E0FEA37C
:10157D00E0FF7C007D64120806E4FD90115FE0F849
:10158D00A3E0F9A3E0FAA3E02FFBEA3EFAED39F967
:10159D00EC38F8D0E0FFD0E0FED0E0FDD0E0FCC3A9
:1015AD0012095F503590114CE0FCA3E0FDA3E0FE65
:1015BD00A3E0FF90113DE0F8A3E0F9A3E0FAA3E06A
:1015CD00FB1203445014E4FF12CA78901154740BAB
:1015DD00F012C9C290115F120A7A901154E0B40B47
:1015ED003A12C9C2C8ECC8C9EDC9CAEECACBEFCB15
:1015FD0090115FE0FCA3E0FDA3E0FEA3E0242CFF2F
:10160D00EE3401FEE43DFDE43CFCD312095F400BDA
:10161D00E4FF12CA289011547409F0901154E0B4EB
:10162D000937901148E0FCA3E0FDA3E0FEA3E0FF25
:10163D0090113DE0F8A3E0F9A3E0FAA3E0FB12035B
:10164D0044601640147F0112CA28901154740AF098
:10165D0012C9C290115F120A7A901154E0B40A3A7D
:10166D0012C9C2C8ECC8C9EDC9CAEECACBEFCB903E
:10167D00115FE0FCA3E0FDA3E0FEA3E024E8FFEE94
:10168D003403FEE43DFDE43CFCD312095F400B7FC7
:10169D000112CA789011547408F0901150E0FCA317
:1016AD00E0FDA3E0FEA3E0FF901139E0F8A3E0F91F
:1016BD00A3E0FAA3E0FB120344600250047F018013
:1016CD00027F00901125EFF07F0312C915901123B1
:1016DD00E07038300C3512000EE4FF12CA28E49089
:1016ED00112BF0754B07754AB275490112ACBBE46D
:1016FD00F54BF54AF549F5487D037F1EFE12ACC248
:10170D009011547401F0E4901122F0901124E060D6
:10171D0006200D03120012901124E060030217C57C
:10172D00200D030217C5901123E070030217C51297
:10173D00C9C290115F120A7A901142E0FCA3E0FD3C
:10174D00E41203C27BCD7ACC794C783F12019EEC2A
:10175D00C0E0EDC0E0EEC0E0EFC0E090112CE0FC89
:10176D00A3E0FDE41203C2C8ECC8C9EDC9CAEECAB4
:10177D00CBEFCBD0E0FFD0E0FED0E0FDD0E0FC120F
:10178D00034460294027E4FFFE7D807C3F901139A2
:10179D00E0F8A3E0F9A3E0FAA3E0FB120344500D37
:1017AD009011547408F07F0112CA82800B9011546D
:1017BD007402F07F0112CA28901123E024FF920CCD
:1017CD00A3E024FF920D901122E0B4010F9011546B
:0E17DD00740CF0E412000EE4FF12CA287F0024
:0117EB0022DB
:105F68009010E7E06026E4F0157315731573A873B5
:105F780076010876110876271573A87376021573CB
:105F8800A8737604FB7D027F401295A19010E8E08B
:105F98006026E4F0157315731573A87376010876F7
:105FA800110876281573A87376031573A8737604F9
:105FB800FB7D027F401295A19010E9E06026E4F095
:105FC800157315731573A873760108761108762969
:105FD8001573A87376041573A8737604FB7D027F86
:105FE800401295A19010EAE06026E4F0157315734D
:105FF8001573A873760108761108762A1573A873A5
:1060080076051573A8737604FB7D027F401295A16F
:10601800157315731573A87376010876110876251C
:106028001573A87376061573A87376047B007D0232
:106038007F401295A1157315731573A8737601081F
:1060480076110876251573A87376071573A87376E5
:10605800047B007D027F401295A11573157315739B
:10606800A87376010876110876851573A873E4F687
:106078001573A873F6FB7D037F61126DF215731516
:10608800731573A87376010876110876851573A8B9
:106098007376011573A873E4F6FB7D037F61126DB7
:1060A800F2157315731573A87376010876110876BF
:1060B800851573A87376021573A873E4F6FB7D0340
:1060C8007F61126DF2157315731573A87376010845
:1060D80076110876851573A87376031573A873E48B
:1060E800F6FB7D037F61126DF2901184EFF0D3947B
:1060F80000500302617D901141E070267F427E606E
:106108007DD57C3F901185E0F8A3E0F9A3E0FAA3E0
:10611800E0FB12019E7BAE7A47793578C11200AD5B
:106128008022E4FFFE7DF87CC0901185E0F8A3E0B2
:10613800F9A3E0FAA3E0FB1200ADE4FBFA7940789A
:106148003F1202A78F468E458D448C437F007E0008
:106158007D207C4112A3C1901185120A7AC2AF90AA
:106168001185E0FCA3E0FDA3E0FEA3E0FF90113958
:10617800120A7AD2AF157315731573A873760108CE
:1061880076110876851573A87376041573A873E4D9
:10619800F6FB7D037F61126DF2157315731573A8F5
:1061A8007376010876110876851573A87376051538
:1061B80073A873E4F6FB7D037F61126DF29011847E
:1061C800EFF0D394004047E4FFFE7DB07CC0A3E02D
:1061D800F8A3E0F9A3E0FAA3E0FB1200AD8F468E26
:1061E800458D448C437F007E007D207C4112A3C1F5
:1061F800901185120A7AC2AF901185E0FCA3E0FDE8
:10620800A3E0FEA3E0FF90113D120A7AD2AF157306
:1062180015731573A87376010876110876851573BA
:10622800A87376061573A873E4F6FB7D037F6112E5
:106238006DF2157315731573A87376010876110836
:1062480076851573A87376071573A873E4F6FB7D36
:10625800037F61126DF2157315731573A8737601B8
:106268000876110876321573A87376021573A87329
:1062780076057B007D037F2012A703157315731520
:1062880073A87376010876110876331573A87376A8
:10629800031573A87376057B007D037F2012A7037F
:1062A800157315731573A87376010876110876347B
:1062B8001573A87376041573A87376057B007D03A0
:1062C8007F2012A703157315731573A87376010839
:1062D80076110876351573A87376051573A8737645
:1062E800057B007D037F2012A703157315731573B3
:1062F800A87376010876110876361573A8737606A2
:106308001573A87376057B007D037F2012A70315FC
:106318007315731573A87376010876110876371507
:1063280073A873E4F61573A8737605FB7D037F20C5
:1063380012A703157315731573A8737601087611E0
:106348000876381573A87376011573A87376057BDC
:10635800007D037F2012A703E4FF12BF92EF24FF02
:10636800920E7F0112BF92EF24FF920F7F0212BF9D
:106378009212BF8BEF24FF921112C9C2C8ECC8C990
:10638800EDC9CAEECACBEFCB9010DEE0FCA3E0FD6E
:10639800A3E0FEA3E024C8FFE43EFEE43DFDE43CA8
:1063A800FCD312095F50030264C39010DDE0FF9034
:1063B800112BE06F602BE0600A7F077EB27D017CC5
:1063C800008005E4FFFEFDFC8F4B8E4A8D498C480A
:1063D8007D067F0A7E0012ACC290112BE09010DD82
:1063E800F07F3512A2A2EF7003026484901122E0BC
:1063F80054FEF07B017A11796412B22390112CEECD
:10640800F0A3EFF07B017A1179647F367E0112A246
:10641800AAEF601F7B017A11796412B223CCEECC0B
:10642800CDEFCDEC1203C2E4FBFA79C87842120230
:10643800A7800312C9AF90112E120A7A7B017A1134
:1064480079647F2F7E0112A2AAEF60417B017A1145
:10645800796412B223EF4E9011226015E04408F0DF
:1064680078557C117D017B017A117964120C498081
:106478001CE054F7F0E4901155F0801190112C7441
:1064880027F0A3740FF0901122E04401F0C390119B
:1064980043E09464901142E0940050167F3B12A2AE
:1064A800A27B017A11796412B223901142EEF0A313
:0E64B800EFF012C9C29010DE120A7A0217EC41
:10C6630020202020557067726164696E6700202066
:10C6730020204669726D776172652E2E2E0032304E
:10C6830031362D30392D3237202D20386365336410
:03C6930038660006
:109B31007BFF7AC679817D2D12C149EA494B6019B3
:109B41007BFF7AC679817D2D12C149E92402F9E4AE
:109B51003A8B44F54589468004E4FEFF22AB44AAD2
:109B610045A9469000011207A5FFC3648094B04047
:109B71000ED3EF648094B95006EF24D0FF801E907D
:109B810000011207A5FFC3648094E1400ED3EF6486
:109B91008094E65006EF24A9FF80027F00EF7D004C
:109BA100FC12078CFFC3648094B0400ED3EF648035
:109BB10094B95006EF24D0FF8021AB44AA45A946B1
:109BC10012078CFFC3648094E1400ED3EF6480944C
:109BD100E65006EF24A9FF80027F00EFC454F04C49
:109BE100FCAB44AA45A9469000021207A5FFC36435
:109BF1008094B0400ED3EF648094B95006EF24D026
:109C0100FF801E9000021207A5FFC3648094E1400B
:109C11000ED3EF648094E65006EF24A9FF80027F03
:109C210000EF75F010A4FFEC45F0FEED4FFF900042
:109C3100031207A5FDC3648094B0400ED3ED648088
:109C410094B95006ED24D0FD8024AB44AA45A94621
:109C51009000031207A5FDC3648094E1400ED3ED8B
:109C6100648094E65006ED24A9FD80027D00EF4D4D
:099C7100FF901164EEF0A3EFF086
:019C7A0022C7
:107E0F00E47880F612C9E8C28575840F75E104E441
:107E1F00F5E275E344F58475B7B075840F758A8301
:107E2F00F597438901758D01758F01758E04F542A4
:107E3F00F5430543E54370020542640F454270F276
:107E4F00438902E4F542F543AE42AF43E4FCFD7BC8
:107E5F00507AC3F9F8D3120949400FE58920E40A93
:107E6F000543E54370E2054280DE75970212BD803F
:107E7F0012BE578F41E4F584E541D39400400EE5DF
:107E8F00EF5402D394004005AF4112929612C833BB
:107E9F00E4FF12C85243EF04E4F542F5437D01AF0E
:107EAF004312C6F50543E54370020542C39402E54C
:107EBF0042940040E8E4F520C22CC22AC230C22FFF
:107ECF00C22E7880F6C23108F67885F618F6788AD1
:107EDF00F6F542F54374992543F582740F3542F553
:107EEF0083E4F00543E54370020542B400E7E54241
:107EFF00B401E2E4F542F54374992543F582741019
:107F0F003542F583E4F00543E543700205426440D2
:107F1F00454270E4E4F584E5EF20E10CE5EF540809
:107F2F00D394004003D38001C392037D08E4FF1272
:107F3F00C294129DBCE47889F67882F6AB18AA1920
:107F4F00A91A7882E6FF75F020A4F58285F08312D6
:107F5F0007A5FE788926F6EE600578820680DDEFAC
:107F6F00D394004032AB18AA19A91A90000D120A27
:107F7F00FA12078CF54174551207D212078C64550B
:107F8F006002D22E74AA1207D212078C64AA600262
:107F9F00D22EE5411207D2E4F584E5EF5402D394D3
:107FAF000040047F018002E4FF12AA0D8F40E540DC
:107FBF0020E036C22B74FF788CF608F608F608F628
:107FCF007E007F107D007B007A007992120C66751F
:107FDF0048FF754950754AA4754B00754C107B00CE
:107FEF007A00799212C1F18002D22B129B317890D4
:107FFF00A60608A607E54030E1030280AFE4F5428C
:10800F00F543E543AE427805C333CE33CED8F9FFFF
:10801F00AB18AA19A91AF5828E831207A56078E901
:10802F002FF9EA3EFA9000041207A520E25EE4F56C
:10803F003FE53FC3787A965053E543AE427805C388
:10804F0033CE33CED8F9AB18AA19A91AF5828E837D
:10805F001207A5FF7E00C006C0077D00E543AE42B4
:10806F007805C333CE33CED8F929F9EA3EFA90001A
:10807F000D120AFA7889E6853FF0A429F9EA35F05E
:10808F00FAD007D006120C66053F80A50543E543DD
:10809F00700205420280117F011290F1C22D8007FC
:1080AF00E4FF1290F1D22DE4F542F5437A007B966E
:1080BF007D03AF4312B8480543E54370020542C341
:0880CF009402E542940040E434
:0180D7002286
:05CA9100788AE6FF2297
:0300230002A4D85C
:10A4D800C0E0C0F0C083C082C0D075D000C000C04A
:10A4E80001C002C003C004C005C006C00730993EC1
:10A4F800C2997885067985E77881667015F678853A
:01A50800F65C
:0DA5090075270A75281300D528FCD527F604
:04A51600C285801C5E
:0DA51A0075271475281300D528FCD527F6E9
:10A527007885E62499F582E43410F583E0F59920DF
:10A53700980302A5D3209A08202C05C29802A5CF1C
:10A54700C29A7884E6062499F582E4340FF583E508
:10A5570099F0C298E6FFB40112900F99E0FE7003DC
:10A56700F68069EE54072402788BF6EFB4020D7873
:10A577008BE6B40907900F9AE02403F67884E6FF88
:10A58700B40007E4B40103F68042EFC3788B96402A
:10A597003B7884E624FFFDE434FFFC7B017A0F79E6
:10A5A7009912BA867884E62498F582E4340FF58305
:08A5B700E06F600476008014DF
:0DA5BF0075271475281300D528FCD527F644
:10A5CC00122C3678847600D007D006D005D004D073
:10A5DC0003D002D001D000D0D0D082D083D0F0D024
:02A5EC00E0325B
:10002600900F9AE075F020A4AB18251AF9E519355A
:10003600F0FA90000D120AFA788AE6FF18E68FF0B9
:10004600A4252BF582E435F0F5831207A5FF7B0086
:040056007A0079298A
:10005A008F398B3A8A3B893CE4F584EA494B601C28
:10006A00AB3AAA3BA93C12078CFFE539FD7C00128A
:0C007A00CA6CAB3AAA3BA93CEF1207D2BB
:0D008600753D14753E1300D53EFCD53DF6CA
:0E0093008539997F0112C7223099FDC299224A
:10C62D009010997478F07884E62498F582E4340FAC
:09C63D00F583E090109AF07F02F1
:09C64600E4F5847881EFF6D28559
:0DC64F00753914753A1300D53AFCD539F64B
:07C65C00901099E0F599220E
:10C4AF00C9EFC9E964017028EDC39B4034787AE67F
:10C4BF00FFEB2FFFE433FEEDC39FEE6480F8748033
:10C4CF0098501ED22CC3ED9B788AF678867601227F
:10C4DF00B90214ED6B700AD22C788AF67886760240
:08C4EF0022C22CE47886F6223B
:10BF2A00C9EFC9BAFF15BBFF12ED6B7002EC6A705C
:10BF3A0049D22C788AF67886E9F622E964017025D6
:10BF4A00C3ED9BEC9A401C787AE62BFFE43AFEC3D9
:10BF5A00ED9FEC9E500DD22CC3ED9B788AF6788625
:10BF6A007601228015B90218ED6B7002EC6A700A2C
:10BF7A00D22C788AF67886760222C22CE47886F663
:01BF8A002294
:102C3600900F99E0FF54F8F52AE4F584EF120B2A79
:102C46002C86092C930A2CA6102CAF112CC0122C02
:102C5600D7192CED1A2D12202D1B282DB7292EB988
:102C6600332EF4372F24392F3E412F49492F544E06
:102C76002F87502FCF612E83702FC79800002FFF0C
:102C8600900F9AE0FD788DE6FB7F018027900F9AE2
:102C9600E0FCA3E0FD788CE6FA08E6FB7F01802BDA
:102CA600D22C78867603022FFF900F9AE0FD788F5C
:102CB600E6FB7F0212C4AF022FFF900F9AE0FCA33F
:102CC600E0FD788EE6FA08E6FB7F0212BF2A022FA5
:102CD600FF900F9AE0FD788DE6FB7F0112C4AF20CE
:102CE6002C03022FFF801A900F9AE0FCA3E0FD78D8
:102CF6008CE6FA08E6FB7F0112BF2A202C03022F7E
:102D0600FF9010997478F07F01022FFCE4F584752A
:102D1600EF10022FFFC2ACE4F529D285FB7A0079C9
:102D2600297F7F12005A7B007A0079297F1E1200C4
:102D36005A7B007A0079297F0512005A7882E612BA
:102D46000053788CE6120053788DE6120053788E85
:102D5600E6120053788FE61200537890E61200537D
:102D66007891E6120053E4F52B7492252BF8E612BF
:102D76000053052BE52BC3941040EEE4F52B748924
:102D8600252BF582E4340FF583E0120053052BE57D
:102D96002BC3940640E87B007A007900AF29120025
:012DA6005AD2
:0D2DA70075370A75381300D538FCD537F69E
:102DB400022E6E900F9AE0FFC37882964003022E93
:102DC40075EF75F020A4251AF9E51935F085183446
:102DD400F5358936C2ACE4F529D285FB7A00792928
:102DE4007F7F12005A7B007A0079297F0D12005AE6
:102DF400AB34AA35A93612078C120053AB34AA356A
:102E0400A936900001120050AB34AA35A9369000BF
:102E140002120050AB34AA35A936900003120050B8
:102E2400AB34AA35A936900004120050E4F52BAB5C
:102E340034E5362405F9E43535FA7E00E9252BF925
:102E4400EE3AFA12078C120053052BE52BC39408B3
:0D2E540040DD7B007A007900AF2912005AA2
:0D2E610075370A75381300D538FCD537F6E3
:102E6E00C285D2AC022FFF9010997478F0E4A3F0D3
:102E7E007F02022FFC12C9D578A2120A6E90109909
:102E8E00747CF078A2E6A3F008E6A3F008E6A3F0BF
:102E9E0008E6A3F07C007D057B017A10799912BAC1
:102EAE008690109EEFF07F06022FFC900F9AE0FFA7
:102EBE00B4010FA3E0FDA3E0788CCDF608EDF60289
:102ECE002FC7EFB4020A900F9BE0788CF6022FC743
:102EDE00900F9AE0B4030CA3E0FFA3E0788ECFF638
:102EEE0008EFF6022FC7E4F52B900F9AE0FFE52BC3
:102EFE00C39F501B749B252BF582E4340FF583E0A2
:102F0E00FF7492252BF8EFF6052BE52BB410DAE4BF
:102F1E0078A1F6022FC77A007B327D01788AE6FF10
:102F2E0012B848900F9AE0FDE4FF12C294022FFFF0
:102F3E00900F9AE024FF9202022FFF900F9AE02446
:102F4E00FF9201022FFF7A007B327D017F0012B8C3
:102F5E0048E4F52B749A252BF582E4340FF583E0C3
:102F6E00FF748F252BF582E4340FF583EFF0052BDC
:102F7E00E52BB406DFD2318078788AE66005752DB0
:102F8E0002800B202F05752D038003752D019010E7
:102F9E00997479F0A3E52DF07C007D027B017A1007
:102FAE00799912BA8690109BEFF07F0312C646E510
:102FBE002D6401703CD2308002D22A788076F18066
:102FCE00307A007B327D017F0012B84890109974E0
:102FDE0079F0900F9AE090109AF07C007D027B01C0
:102FEE007A10799912BA8690109BEFF07F0312C671
:102FFE0046E52A64A0600302320E900F99E064A1A8
:10300E0060030230FEA3E0C378829640030230F3E1
:10301E00AB18AA19A91AE0FF75F020A4F58285F065
:10302E00831207A5F52DEF75F020A429F9EA35F0E6
:10303E00FA9000041207A530E237900F9AE012CAF8
:10304E008C8F2D901099747FF0A3E52DF02402FD46
:10305E00E433FC7B017A10799912BA86749B252D84
:10306E00F582E43410F583EFF0E52D2403FF0232F0
:10307E000B900F9AE0FF12CA8CC2ACE4F529D285F0
:10308E00E52DD39406402B7B007A0079297F7F12A1
:10309E00005A7B007A007929AF2D12005AE4F52BE5
:1030AE00E52BC3952D5007120026052B80F2052D1A
:1030BE008018E52D2478120053E4F52BE52BC395EB
:1030CE002D5007120026052B80F27B007A00790026
:0530DE00AF2912005AA9
:0D30E30075370A75381300D538FCD537F65F
:1030F0000231FD9010997478F07F0102320B900F2D
:1031000099E064A2600302320E7882E6FFA3E0FE3B
:10311000C39F4003023203A3E0FDC39F400302327A
:1031200003EE9D4003023203900F9AE0F52BE4F585
:1031300032F533900F9BE0FFE52BD39F5026AF2B4A
:1031400012CA8CAB18AA19A91A75F020E52BA4F5A0
:103150008285F0831207A52533F533E43532F53245
:10316000052B80CFC2ACE4F529D285FB7A00792902
:103170007F7F12005AC3E5339480E53294005002F9
:103180008007E5324480120053AF33120054900F91
:103190009AE0F52B900F9BE0FFE52BD39F5046E480
:1031A000F52CAB18AA19A91A75F020E52BA4F58205
:1031B00085F0831207A5FFE52CC39F5024E52B75EE
:1031C000F020A429F9EA35F0FA90000D120AFA78F5
:1031D0008AE6FF18E68FF0A4252C120049052C8002
:1031E000C1052B80AF7B007A007900AF2912005A0D
:0D31F00075370A75381300D538FCD537F651
:1031FD00C285D2AC800B9010997478F07F0112C605
:10320D0046E52A6458704DFA7B327D01788AE6FFD7
:10321D0012B848753C01753D10753E9A7B017A0FC9
:10322D00799A12C6C88F2DE52D2478901099F0EF5C
:10323D002401FDE433FC7B017A10799912BA86746E
:10324D009A252DF582E43410F583EFF0E52D240257
:10325D00FF12C646E52A64806009E52A648860038A
:10326D000234037886E6B4010F7A007B327D017853
:10327D008AE6FF12B848801AE4F52BE52BC3787A5D
:10328D0096500F7A007B327D01AF2B12B848052B7B
:10329D0080E9900F99E05407F52DB4070A752C01BC
:1032AD00A3E0F52DA38006E4F52C900F9AE0F52E02
:1032BD00152DE52EC37882964003023403AB18AA70
:1032CD0019A91A75F020E52EA4F58285F083120751
:1032DD00A5FFE52DD39F40028F2D7886E6B4010919
:1032ED00788AE6F531F5308009E4F530787AE61420
:1032FD00F531788AA630788AE6D3953140030233CA
:10330D00F7E4F52BE52BC3952D40030233ECE52EA9
:10331D0075F020A4AB18251AF9E51935F0FA9000CF
:10332D00041207A530E2030233E79000011207A54E
:10333D0064387041E52DD394044011E52C252B24E0
:10334D009BF582E4340FF583E0FD80707884E6C34D
:10335D00952BFFE49400FE74972FF582740F3EF5C4
:10336D0083E0FDE52E75F020A4AB18251AF9E519BB
:10337D0035F0FA8047AB18AA19A91A75F020E52E79
:10338D00A4F58285F0831207A5FF7884E6C39FFF1D
:10339D00E49400FE7C00EF252BFFEC3EFEEF252C88
:1033AD00FFEC3EFE74982FF582740F3EF583E0FD21
:1033BD00E52E75F020A429F9EA35F0FA90000D12EA
:1033CD000AFA788AE6FF18E68FF0A4FFE52B2FF5B1
:1033DD0082E435F0F583ED1207E4052B023311AFCE
:1033ED002E12C915788A06023303788AA630E52A8B
:1033FD00B4880312C62DE52A64A8600302353B7814
:10340D0086E6B4010F7A007B327D01788AE6FF12E1
:10341D00B848801AE4F52BE52BC3787A96500F7ACD
:10342D00007B327D01AF2B12B848052B80E9900F40
:10343D009AE030E711547FFEA3E0FDEEF532EDF595
:10344D0033752C03800C900F9AE0753200F53375AF
:10345D002C027499252CF582E4340FF583E0FF746A
:10346D009A252CF582E4340FF583E0F52F8F2EE5A8
:10347D002ED3952F4003023538E52EC37882964022
:10348D0003023533AB18AA19A91A75F020E52EA43D
:10349D00F58285F0831207A5F52D7886E6B401092E
:1034AD00788AE6F531F5308009E4F530787AE6145E
:1034BD00F531788AA630788AE6D39531505EE4F5F9
:1034CD002BE52BC3952D504AE52E75F020A4AB1896
:1034DD00251AF9E51935F0FA9000041207A520E236
:1034ED002DE52C252B249BF582E4340FF583E0FD8F
:1034FD0090000D120AFA788AE6FF18E68FF0A4FF05
:10350D00E52B2FF582E435F0F583ED1207E4052B5D
:10351D0080AFAF2E12C915788A06809A788AA630A8
:0E352D00E52D252CF52C052E02347C12C62D22
:01353B00226D
:10F000007880E664F1600302F668E478B1F608F609
:05F010007881E6601E9E
:0DF0150075510A75521300D552FCD551F605
:10F0220078B206E61870010678B1B627E108B61084
:10F03200DDC2AF7584015398FC75FFDE75FFADE448
:10F0420078ADF618F6E4F584209830E478B1F60845
:10F05200F6209823C378B2E6948818E694135017E2
:0DF0620075510A75521300D552FCD551F6B8
:10F06F0078B206E61870DD0680DAB28680CD78AC0D
:10F07F00A699C298E6FF641A6008EF640A6003025B
:10F08F00F168E478B1F608F6209823C378B2E694D5
:07F09F008818E694135017D6
:0DF0A60075510A75521300D552FCD551F674
:10F0B30078B206E61870DD0680DA30988778ADA658
:10F0C30099C298E478B1F608F6209823C378B2E69B
:08F0D300948818E6941350170D
:0DF0DB0075510A75521300D552FCD551F63F
:10F0E80078B206E61870DD0680DA20980302F04749
:10F0F80078ADA699C298E478B1F608F6209823C3AB
:0BF1080078B2E6948818E694135017C4
:0DF1130075510A75521300D552FCD551F606
:10F1200078B206E61870DD0680DA20980302F04710
:10F1300078ADA699C29818E6641A600302F659D20F
:03F1400085C299EC
:0DF1430075511475521300D552FCD551F6CC
:06F150007599783099FD6D
:0DF1560075510A75521300D552FCD551F6C3
:10F16300C28502F65978ACE6FF6450600302F1FDF4
:10F1730078B1F608F6209823C378B2E6948818E6A7
:04F18300941350177A
:0DF1870075510A75521300D552FCD551F692
:10F1940078B206E61870DD0680DA20980302F0479C
:0AF1A40078ADA699C298D285C299F1
:0DF1AE0075511475521300D552FCD551F661
:08F1BB007599793099FDC299A4
:0DF1C30075511475521300D552FCD551F64C
:08F1D0007599013099FDC29907
:0DF1D80075511475521300D552FCD551F637
:06F1E500E4F5993099FDEC
:0DF1EB0075510A75521300D552FCD551F62E
:0EF1F800C28502F659EF6401703ED285C299BD
:0DF2060075511475521300D552FCD551F608
:08F213007599783099FDC2994C
:0DF21B0075511475521300D552FCD551F6F3
:06F22800E4F5993099FDA8
:0DF22E0075510A75521300D552FCD551F6EA
:10F23B00C28502F65978ACE66402600302F30C78DF
:10F24B00B1F608F6209823C378B2E6948818E694B2
:03F25B0013501736
:0DF25E0075510A75521300D552FCD551F6BA
:10F26B0078B206E61870DD0680DA20980302F047C4
:10F27B0078ADA699C298E408F618E6FF13B3928608
:10F28B00EF25E0FEC3E49400EE94F0502DE6FD7FF5
:10F29B000025E0FEC394E05021ED20E024E4F5844A
:10F2AB0043B701758F0378B3EEF608EFF6F5828E50
:10F2BB0083E4F053B7F0F58F800478AE76FFE4F576
:05F2CB0084D285C29908
:0DF2D00075511475521300D552FCD551F63E
:08F2DD007599783099FDC29982
:0DF2E50075511475521300D552FCD551F629
:08F2F20078AEE6F5993099FDB4
:0DF2FA0075510A75521300D552FCD551F61E
:10F30700C28502F65978ACE66403600302F46778B5
:10F31700B1F608F6209823C378B2E6948818E694E5
:03F3270013501769
:0DF32A0075510A75521300D552FCD551F6ED
:10F3370078B206E61870DD0680DA20980302F047F7
:10F3470078ADA699C298E478B1F608F6209823C359
:0BF3570078B2E6948818E69413501773
:0DF3620075510A75521300D552FCD551F6B5
:10F36F0078B206E61870DD0680DA20980302F047BF
:10F37F0078AFA699C29878ADE6FF139286EF25E095
:10F38F00FEC3E49400EE94F0400302F047E67D00E4
:10F39F0025E0FCC394E0400302F047E4F58443B753
:10F3AF0001758F0178AFE675F020A42DFFE5F03CD5
:10F3BF0078B3F608EFF6E4F58478B0F678B0E6C3E4
:10F3CF009420504CE408F608F6209823C378B2E650
:08F3DF00948818E694135017FE
:0DF3E70075510A75521300D552FCD551F630
:10F3F40078B206E61870DD0680DA20980302F0473A
:10F4040078B30806E618CEE6CE70010614F5828EAF
:10F4140083E599F0C29878B00680ACE4F58453B7DC
:09F42400F0F58FF584D285C29940
:0DF42D0075511475521300D552FCD551F6DF
:08F43A007599783099FDC29923
:0DF4420075511475521300D552FCD551F6CA
:06F44F00E4F5993099FD7F
:0DF4550075510A75521300D552FCD551F6C1
:10F46200C28502F65978ACE6FD6404600302F52415
:10F4720078B1F608F6209823C378B2E6948818E6A5
:04F482009413501778
:0DF4860075510A75521300D552FCD551F690
:10F4930078B206E61870DD0680DA20980302F0479A
:10F4A30078ADA699C298E625E078B5F608E4F67833
:10F4B300AEF678B1F608F678B50806E618CEE6CECD
:10F4C30070010614F5828E83E49378AE26F678B243
:10F4D30006E61870010678B2E6700418E664027056
:05F4E300D6D285C2999C
:0DF4E80075511475521300D552FCD551F624
:08F4F5007599783099FDC29968
:0DF4FD0075511475521300D552FCD551F60F
:08F50A0078AEE6F5993099FD99
:0DF5120075510A75521300D552FCD551F603
:10F51F00C28502F659ED6405600302F64D78B1F627
:10F52F0008F6209823C378B2E6948818E69413500F
:01F53F0017B4
:0DF5400075510A75521300D552FCD551F6D5
:10F54D0078B206E61870DD0680DA20980302F047DF
:10F55D0078ADA699C298E478B1F608F6209823C341
:0BF56D0078B2E6948818E6941350175B
:0DF5780075510A75521300D552FCD551F69D
:10F5850078B206E61870DD0680DA20980302F047A7
:0AF5950078AFA699C298D285C299FA
:0DF59F0075511475521300D552FCD551F66C
:08F5AC0075997F3099FDC299A9
:0DF5B40075511475521300D552FCD551F657
:10F5C1007599203099FD78ADE625E0FC78AFE675B8
:10F5D100F020A42400FFE5F03C78B5F608EFF6E44E
:08F5E10078AEF678B0F6C2998D
:0DF5E90075511475521300D552FCD551F622
:10F5F60078B5E6FE08E6F5828E83E493F5993099B0
:10F60600FD78B50806E618CEE6CE70010614F5823A
:10F616008E83E49378AE26F678B006E6B420C2C2AE
:01F62600994A
:0DF6270075511475521300D552FCD551F6E3
:08F6340078AEE6F5993099FD6E
:0DF63C0075510A75521300D552FCD551F6D8
:10F64900C285800C78ACE6B40606E4F58475EF1043
:0FF6590078ACE66407600302F0477880F6D2AF22
:01F66800227F
:10AAF5007F0012C72212C41D202B0B7A007B327DEA
:10AB0500017F0012B848302E0B7A007B1E7D017F35
:10AB15000012B848302A17302F147A007B327D0195
:10AB2500788AE6FF12B848C22A12B375D22B202DB7
:10AB35000C302F09788076F112B375D22D30302A7A
:10AB4500302F27C23012CA52E4FDFF12C99B7BFF8A
:10AB55007AC6796312C7797D01E4FF12C99B7BFF31
:10AB65007AC6797112C77912F00030310B7B017A00
:10AB75000F798F12BC28C23112C9C2C8ECC8C9ED01
:10AB8500C9CAEECACBEFCB900F951209F9EF245A3B
:10AB9500FFE43EFEE43DFDE43CFCD312095F500FAB
:10ABA50012C9C2900F95120A22D312095F401212E0
:10ABB500C9C2900F95120A7A7B017A0F798912AE74
:10ABC50074202F1212C9C2E47B2C7A01F9F8C31242
:07ABD500095F5002D22F229C
:10C97100E4F58475EF027F64DFFE127E0F12AAF5E3
:05C98100125F6880F860
:10A034004D656D6F727920746573742E2E2E004DEC
:10A04400656D6F7279206572726F722062616E6BDA
:10A054002025626400005EBCE2613FDD83C29C7E19
:10A0640020A3FD1F419DC3217FFCA2401E5F01E38D
:10A07400BD3E6082DC237D9FC1421CFEA0E1BF5D2A
:10A084000380DE3C62BEE0025CDF81633D7C22C073
:10A094009E1D43A1FF4618FAA427799BC584DA388C
:10A0A40066E5BB5907DB856739BAE406581947A545
:10A0B400FB7826C49A653BD987045AB8E6A7F91BEE
:10A0C40045C6987A24F8A6441A99C7257B3A64862B
:10A0D400D85B05E7B98CD2306EEDB3510F4E10F258
:10A0E400AC2F7193CD114FADF3702ECC92D38D6FF5
:10A0F40031B2EC0E50AFF1134DCE90722C6D33D1C2
:10A104008F0C52B0EE326C8ED0530DEFB1F0AE4CDA
:10A114001291CF2D73CA947628ABF517490856B41B
:10A12400EA6937D58B5709EBB536688AD495CB29BC
:10A1340077F4AA4816E9B7550B88D6346A2B759775
:10A14400C94A14F6A8742AC896154BA9F7B6E80AA2
:10A1540054D7896B35000000002B6096CBDDEE00F0
:09A164002C96CBDDE5EEF7FAFDC7
:10C27000C1B3420C0D0009420C150009420C0F0815
:09C2800009420C17080901740AB7
:10C9AF0074FFF542F541F540F53FAF42AE41AD4062
:02C9BF00AC3F8B
:01C9C1002253
:10BA860015731573A873ECF608EDF6157315731593
:10BA960073A873C6EBC608C6EAC608C6E9C6E57348
:04BAA60024FCF57314
:10BAAA00F80808E4F6A873F608F6E5732407F9A877
:10BABA0073E6FE08E6FFC3099719E76480F8EE64A7
:10BACA0080985037E5732404F8CBE6CB08E6FA08E9
:10BADA00E6F98F828E831207A5A873080866FFE528
:10BAEA00732403F8EFF6E690A05993A8730808F6B2
:10BAFA00A8730806E61870B20680AFA8730808E6AD
:01BB0A00FF3B
:07BB0B00E5732409F5732224
:0BCA6C00ED6F78A6F6E690A05993FF4E
:01CA7700229C
:0300A30002B72180
:10B72100C0E0C0F0C083C082C0D0E8C0E0EEC0E09D
:10B73100EFC0E0E59830E11B900C0FE0FEA3E0FFC5
:10B74100900C17E06E7003A3E06F7002C2845398EF
:10B75100FDD233E59830E049900C16E02401FF90CA
:10B761000C15E03400FE900C0DE06E7003A3E06F49
:10B771007002802A900C15E475F0011208A385F07F
:10B7810082F583E599F0900C15E064087004A3E05C
:10B791006409700A900C157400F0A37409F05398B1
:10B7A100FED0E0FFD0E0FED0E0F8D0D0D082D08350
:05B7B100D0F0D0E032F1
:10C41D00900C0FE0FEA3E0FF900C17E06E7003A3ED
:10C42D00E06F6034303331C233D284758401900CA7
:10C43D000FE475F0011208A385F082F583E0F599FC
:10C44D00900C0FE0640C7004A3E06409700A900C6A
:09C45D000F7408F0A37409F02229
:10C19F00900C0DE0FEA3E0FF900C15E06E7003A372
:10C1AF00E06F6039900C0DE475F0011208A385F073
:10C1BF0082F583E0787BF6900C0DE064087004A3A1
:10C1CF00E06409700A900C0D7400F0A37409F07804
:10C1DF007BE6FEB40D037F0A22CFEECF2212AAF523
:02C1EF0080AE20
:02C3D1001573E2
:10C3D300900C0DE0FEA3E0FF900C15E06E7003A33C
:10C3E300E06F6031900C0DE475F0011208A385F045
:10C3F30082F583E0A873F6900C0DE064087004A343
:10C40300E06409700A900C0D7400F0A37409F0A89D
:07C4130073E6FF80027FFFCA
:03C41A0005732285
:08B969008B4C8A4D894E8D4F75
:10B9710012C9C278A7120A6EE478ABF612C3D1EFEE
:10B98100F46037EF640A6032BF0D13AB4CAA4DA9C6
:10B991004E78ABE6FFF582758300E40207E4AB4C19
:10B9A100AA4DA94E78ABE606F582758300EF120722
:10B9B100E478ABE6FF654F70012212AAF512C9C205
:10B9C100ECC0E0EDC0E0EEC0E0EFC0E0AF50E4FC61
:10B9D100FDFE78A7120A15EF2BFBEE3AFAED39F9C5
:10B9E100EC38F8D0E0FFD0E0FED0E0FDD0E0FCD3B1
:07B9F10012095F50877F007F
:01B9F800222C
:10C53E00900C18E02401FD900C17E03400FC900CD8
:10C54E000FE06C7003A3E06D700122900C17E47580
:10C55E00F0011208A385F082F583EFF0900C17E03E
:10C56E00640C7004A3E06409700A900C177408F050
:05C57E00A37409F02286
:10C81400900C0FE0FEA3E0FF900C17E06E7003A3F2
:0FC82400E06F600A7F0012C72212C41D80E2225B
:10C466007E007F09900C15EEF0A3EFF0900C0DEE18
:10C47600F0A3EFF07E087F09900C17EEF0A3EFF023
:10C48600900C0FEEF0A3EFF07E087F007D007B019D
:10C496007A007909120C667E047F007D007B017AA2
:09C4A600087909120C66D2332258
:10C29400EF7025F5847598D0F584759115F584753E
:10C2A400C90875CBFFED90A15893F5CA75C804E48D
:10C2B400F584D2ACC2BC8026758401759850E4F52F
:10C2C40084E589540F4420F589758E02ED90A162AE
:10C2D40093F58DD28E43E74043F74012C466D2AF44
:01C2E4002237
:10BDEC00900C09120A9F00000000900C11120A9F7F
:10BDFC00000000009000007464F0E478A7F678A7C7
:10BE0C00E6FFC394025043EF25E025E02401F582C0
:10BE1C00E43400F583E4F0EF25E025E02402F5821C
:10BE2C00E43400F583E4F0EF25E025E02403F5820B
:10BE3C00E43400F583E4F0EF25E025E02404F582FA
:0ABE4C00E43400F583E4F00680B44E
:01BE560022C9
:10C83300D2AFD2A9C2BBE4F584E589540F4401F514
:0FC8430089758E02758CAFE4F58AD28C02BDEC3C
:02A91B001573B2
:10A91D00A873E4F6A873E6FFC39402400302AA0AE3
:10A92D00EF25E025E02404F582E43400F583E0FF13
:10A93D00D39400500302A9DFE625E025E02402F5BB
:10A94D0082E43400F583E0600302A9DFEF30E01903
:10A95D00E6FF25E025E02404F582E43400F583E0EC
:10A96D00D3940140047D0080067D01A873E6FF129B
:10A97D00BD12A873E6FF25E025E02404F582E4343A
:10A98D0000F583E0B401057D0112BD12A873E6FF49
:10A99D0025E025E02404F582E43400F583E014F08D
:10A9AD00EF25E025E02404F582E43400F583E06032
:10A9BD0021E6FF25E025E02403F582E43400F5834C
:10A9CD00E0FEEF25E025E02402F582E43400F58376
:10A9DD00EEF0A873E6FF25E025E02402F582E434CD
:10A9ED0000F583E06011EF25E025E02402F582E417
:0DA9FD003400F583E014F0A8730602A921D0
:03AA0A00057322AF
:03000B0002B5EC4F
:10B5EC00C0E0C0F0C083C082C0D0E8C0E0E9C0E0D9
:10B5FC00EAC0E0EBC0E0ECC0E0EDC0E0EEC0E0EF94
:10B60C00C0E0758CAF900C09E0FCA3E0FDA3E0FE5C
:10B61C00A3E02401FFE43EFEE43DFDE43CFC900C81
:10B62C0009120A7A900000E014F0E07025900C11D9
:10B63C00E0FCA3E0FDA3E0FEA3E02401FFE43EFE5A
:10B64C00E43DFDE43CFC900C11120A7A900000746D
:10B65C0064F012A91B12C7F2D0E0FFD0E0FED0E0DC
:10B66C00FDD0E0FCD0E0FBD0E0FAD0E0F9D0E0F87F
:0BB67C00D0D0D082D083D0F0D0E032DC
:10C6F5001573A873EDF61573A873EFF6A873E6FF27
:10C70500C39402501308E6FEEF25E025E02401F569
:0DC7150082E43400F583EEF0057305732215
:10B8480015731573A873EAF608EBF61573A873ED6C
:10B85800F61573A873EFF6A873E6FFC39402506A4F
:10B86800EF25E025E02404F582E43400F583E07058
:10B8780059E6FB25E025E02402F582E43400F5834F
:10B88800E0704708E625E004FFA873E6FA25E025FE
:10B89800E02404F582E43400F583EFF00808E6FEBE
:10B8A80008E6FF7C007D0A12086DEA25E025E02401
:10B8B80003F582E43400F583EFF0EB25E025E0247E
:10B8C80002F582E43400F583E4F0E5732404F573AB
:01B8D800224D
:0EBD12001573A873EDF61573A873EFF615738D
:10BD2000A87308E6FFC394025024EF25E025E02421
:10BD300001F582E43400F583E06013A8730808E697
:10BD400070047F0180027F00A8730808EFF6A873D3
:10BD5000A68475840FA87308E6FF700BA873080803
:10BD6000E624FF9286800DEFB40109A8730808E667
:09BD700024FF9287A873E6F58414
:07BD79000573057305732239
:10C9C200C2AF900C09E0FCA3E0FDA3E0FEA3E0FFF0
:02C9D200D2AFE2
:01C9D4002240
:10C9D500C2AF900C11E0FCA3E0FDA3E0FEA3E0FFD5
:02C9E500D2AFCF
:01C9E700222D
:10C722001573A873EFF6A873E670057875F608F628
:10C732003032167874E675F064A4FFC37876E69F0B
:0CC7420018E695F0500375FFA505732262
:10C85200D232E47875F608F6EF78746003F6800257
:0FC86200760A75FF0775FFA5E4F58475EF0422CC
:10C9E800C232E47875F608F6787476FF75FFDE755E
:03C9F800FFAD226E
:10C7F200787606E6187001063032167874E675F01F
:10C8020064A4FFC37876E69F18E695F0500375FF9F
:02C81200A5225D
:04C74E008E448F4541
:10C75200E4F546F547C3E5479545E5469544501649
:10C762007FE87E0312C0417F0112C7220547E547D9
:06C7720070E3054680DFC4
:01C77800229E
:04C041008E6B8F6C07
:10C04500D3E56C94FAE56B94005010AF6CEFD39484
:10C055000040407E1600DEFD1F80F2856B6D856C0D
:10C065006ED3E56E94FAE56D940040157FFA7E0077
:10C0750012C0417406256EF56E74FF356DF56D8041
:10C08500E0D3E56C9400E56B94004007AF6EAE6DB0
:03C0950012C04195
:01C098002285
:10BEC20075500075510075524A7B007A0079487DA1
:01BED200026D
:08BED3008B4C8A4D894E8D4F06
:10BEDB007F0112C722AB50AA51A9521208B92400F4
:10BEEB00FFE5F034E0FE854C53854D54854E55E40B
:10BEFB00FDEDC3954F501BEF2DF582E43EF583E42A
:10BF0B0093AB53AA54A9558D827583001207E40D88
:0FBF1B0080DFAB50AA51A952E4854FF00208E431
:10B01000755312755434755B00755C00755D557B16
:07B02000007A0079537D0264
:08B027008B578A5889598D5A94
:10B02F007880E664F1600302B0C412C9E8C2AFE4ED
:10B03F00F58443B701758F01AB5BAA5CA95D12085C
:10B04F00B92400FFE5F034E078ACF608EFF6AA5823
:10B05F00A95978B0A65708C6EAC608C6E9C6E47863
:10B06F00AEF678AEE6C3955A503278B0CBE6CB0841
:10B07F000806E618CAE6CA70010614F912078C789A
:10B08F00AFF6E6FF78AC0806E618CCE6CC70010602
:10B09F0014F5828C83EFF078AE0680C6E4F58F53FB
:10B0AF00B7F0AB5BAA5CA95D855AF01208E4D2AF8A
:05B0BF00E4FF12C8527D
:01B0C4002269
:10C335007880E664F17046C2AF12C9E8E4F584433B
:10C34500B701758F0378AD76E008F678ACF678AD71
:10C35500E6FE08E6F5828E83E4F07F0112C72278B7
:10C36500AEE426F618740236F61806E6C3940840BD
:0DC37500DDE4F58F53B7F0D2AFFF12C852D0
:01C382002298
:10B3750012C335E4F555F556F55B755C00755D55FD
:10B38500FB7A00798C7D1612B02712B010E4F552C5
:10B39500E552C3787A965073E4F551AB18AA19A90A
:10B3A5001A75F020E551A4F58285F0831207A56092
:10B3B50056E55175F020A429F9EA35F0FA90000D0B
:10B3C500120AFA7889E68552F0A429F9EA35F0FAE5
:10B3D500EBC0E0EAC0E0E9C0E0AB18AA19A91A750C
:10B3E500F020E551A4F58285F0831207A5FD755B74
:10B3F50000755C00755D55D0E0F9D0E0FAD0E0FB52
:10B4050012B027055180940552808512B010E4785A
:02B4150080F6BF
:01B417002212
:02AA0D008F4474
:10AA0F00E4F54AF54BF547F55075510075524AFB81
:10AA1F007A00798C7D1612BED312BEC2E54964341A
:10AA2F007004E54864127003434701E4F546E546B8
:10AA3F00C3787A96400302AAE0E4F545AB18AA1949
:10AA4F00A91A75F020E545A4F58285F0831207A5B4
:10AA5F00607AE5446054E54575F020A429F9EA359C
:10AA6F00F0FA90000D120AFA7889E68546F0A429CB
:10AA7F00F9EA35F0FAEBC0E0EAC0E0E9C0E0AB1864
:10AA8F00AA19A91A75F020E545A4F58285F083125D
:10AA9F0007A5FD75500075510075524AD0E0F9D0E9
:10AAAF00E0FAD0E0FB12BED3801DAB18AA19A91A89
:10AABF0075F020E545A4F58285F0831207A5254B97
:10AACF00F54BE4354AF54A054502AA4B054602AA5D
:10AADF003D12BEC2E54964347004E5486412700348
:05AAEF00434702AF47E0
:01AAF400223F
:10C88F00EF540778A9F6EF30E306E64420F680046C
:0CC89F0078A9E6F678A9E644C0F6F5C8D2
:01C8AB00226A
:029296008F4403
:1092980012CA527D017F0212C99B7BFF7AA07934E2
:1092A8001269E5E478A8F612C9E8C2AFE478A7F62F
:1092B80078A7E6FFC3954440030293F912C88F7854
:1092C800A7E6FF7D0312C99B7FDA12C95B902000D5
:1092D800AF82AE83C3EF94FFEE94FF5005E4F0A392
:1092E80080EE902000AF82AE83C3EF94FFEE94FF30
:1092F800500CE0600678A876018003A380E778A880
:10930800E660030293F978A7E6FF7D0312C99B7F05
:10931800D912C95B902000AF82AE83C3EF94FFEEF1
:1093280094FF50067455F0A380ED902000AF82AEF4
:1093380083C3EF94FFEE94FF500EE0645560067807
:10934800A876018003A380E578A8E660030293F974
:1093580078A7E6FF7D0312C99B7FD812C95B9020CE
:1093680000AF82AE83C3EF94FFEE94FF500674AA59
:10937800F0A380ED902000AF82AE83C3EF94FFEEA0
:1093880094FF500EE064AA600678A876018003A3D3
:1093980080E578A8E6705A78A7E6FF7D0312C99B96
:1093A8007FD712C95B902000AF82AE83C3EF94FFD2
:1093B800EE94FF500674FFF0A380ED902000AF827A
:1093C800AE83C3EF94FFEE94FF500DE0F46006788F
:1093D800A876018003A380E678A8E6701478A7E64B
:1093E800FF7D0312C99B7FD612C95B78A70602923C
:1093F800B8D2AFE4FF12C85212C88F78A8E6601B33
:109408007D02E412C99B7BFF7AA0794378A7E6F531
:0B9418004F1269E57F0012C72280F9A7
:019423002226
:10BE5700E4F58475A338F5A275A10475840F759C64
:10BE6700FF759DFF759EFF759FFF75F8FF75E8FFCE
:10BE770075D8FF75C8FFFF12C88F902000E078A71C
:10BE8700F67455F0E064556008E6F0E4F584F5A330
:10BE97002278A7E6F07F0812C88FE078A7F674AA81
:10BEA700F0E0B4AA0AE6F0E4FF12C88F7F10227808
:0ABEB700A7E6F0E4FF12C88F7F0831
:01BEC100225E
:10752200202020202020202020200025622A6264A2
:107532000025622A62750025622A640025622A7586
:107542000025622A2E622A660025622A6C640025C2
:10755200622A6C7500253262753A2573002020205C
:107562002020202020004E6F207661726961626CBB
:10757200657320646566696E6564002020202020A2
:1075820020202020202020202020202020200045F4
:10759200534320454E5445522020202D20202020A8
:1075A2002B20200045534320454E54455220202095
:1075B2002D20202020202B200045534320454E54CF
:1075C2004552202020004553432020202020202007
:1075D2002020002020202020002000506172616DB8
:1075E2006574657273207772697474656E00746F66
:1075F20020666C617368206D656D6F72792E00F480
:1076020070000000F76E000000FA8F000000FD6DB0
:107612000000000000000000036B000000064D00A7
:10762200000009470000000C540000006300000045
:1076320000016D00000002670000000373000000FB
:10764200046D00000005680000000641000000070C
:107652004B000000088043000009804600001448E7
:107662007A00001550610000166261000017570091
:107672000000185600000019B50000001A5400005E
:10768200001B6C2F73001C52504D001D4600000061
:107692001E4A0000005A250000005B52504D005C5B
:1076A200636E74005D780000000000000000023587
:1076B2000000004E6F64652041647200008C01007E
:1076C200000000000000003F8000000000000235C2
:1076D200000000477270204164720000008E0100B9
:1076E200000000000000003F8000000000000A3897
:1076F20000000054696D65000000000111FE0100E8
:10770200000000000000003F8000000000000A3876
:1077120000000044617465000000000111EE0100E8
:10772200000000000000003F80000000000004088C
:1077320000000154656D70000000000111C60200D6
:10774200000000000000003F80000000000004185C
:10775200000001312E3856000000000111DE020047
:1077620000000000000000400000000000000418BB
:10777200000001332E3356000000000111CA02003E
:10778200000000000000004000000000000004189B
:1077920000000135566578740000000111D2020024
:1077A200000000000000004000000000000004187B
:1077B20000000132345600000000000111D6020020
:1077C200000000000000003F8000000000000418DC
:1077D20000000132345665787400000111DA0200AB
:1077E200000000000000003F8000000000000406CE
:1077F20000000149203234560000000111CE02007F
:107802000000000000000040000000000000003204
:10781200000004466C617368000000000000000074
:107822000000000000000000000000000000003224
:107832000000045265626F6F7400000000000000D7
:0E784200000000000000000000000000000038
:0AC28900C1A1C129C128C122C123AF
:067B3E008B3F8A408941E3
:107B44009000011207A56438706085424885434956
:107B540085444AF54B754C0A7B017A1179E212C1CE
:107B6400F17B017A1179E212C986C3EF940AEE64BB
:107B74008094805032E4901196F07B017A1179E27E
:107B840012C986C3740A9FFFE49EFE901196E0C357
:107B94009FEE6480F8748098500D7F2012C95B902A
:107BA4001196E004F080D3027E05E49011E2F0AB7C
:107BB4003FAA40A9419000021207A56068E4901111
:107BC40096F0901196E075F005A42401F582E43452
:107BD40076F583E493FF64636019AB3FAA40A9413F
:107BE4009000021207A5FEEF6E6008901196E00463
:107BF400F080CF901196E0FF75F005A42401F58282
:107C0400E43476F583E493601CEF75F005A4240254
:107C1400F9747635F07548FFF549894A7B017A1184
:107C240079E212C0F1AB3FAA40A9419000011207CA
:107C3400A56066E4901196F0901196E075F005A4A5
:107C44002433F582E43476F583E493FF6019AB3F83
:107C5400AA40A9419000011207A5FEEF6E600890AA
:107C64001196E004F080D1901196E0FF75F005A420
:107C74002433F582E43476F583E493601CEF75F0E5
:107C840005A42434F9747635F07548FFF549894A1A
:107C94007B017A1179E212C0F17B017A1179E21247
:107CA400C986901197EFF0AB3FAA40A94112078C07
:107CB40014601D14606424FE7003027D6E2404604D
:107CC40003027E057BFF7A75792212C779027E054D
:107CD400AB3FAA40A9419000041207A59011973028
:107CE400E11CE0FFC3740A9FF54FAB42AA43A944C9
:107CF40012078CF5507BFF7A75792D027E02E0FF26
:107D0400C3740A9FF54FAB42AA43A94412078CF5EA
:107D1400507BFF7A757933027E02AB3FAA40A941BA
:107D24009000041207A590119730E11FE0FFC3747F
:107D34000A9FF54FAB42AA43A9441208B9F55185ED
:107D4400F0507BFF7A757939027E02E0FFC3740A32
:107D54009FF54FAB42AA43A9441208B9F55185F0E7
:107D6400507BFF7A75793E027E02AB3FAA40A9415F
:107D74009000041207A530E033901197E0FFC3741C
:107D84000A9FF54F9000101207A5FF600280027F42
:107D9400038F50AB42AA43A9441209838F548E53D4
:107DA4008D528C517BFF7A7579438052AB3FAA4048
:107DB400A9419000041207A590119730E121E0FF3A
:107DC400C3740A9FF54FAB42AA43A9441209838F97
:107DD400538E528D518C507BFF7A75794B801FE006
:107DE400FFC3740A9FF54FAB42AA43A94412098307
:107DF4008F538E528D518C507BFF7A757951126955
:0A7E0400E57B017A1179E212C779DB
:017E0E002251
:0D3E2000901189E0FBA3E0FAA3E0F97DFF1B
:103E2D008D428B3F8A4089419000011207A564386D
:103E3D007003024631AB3FAA40A94112078C24FE04
:103E4D00700302409224FE70030242EB24036003D0
:103E5D000246319000041207A520E103023F4CAB4E
:103E6D003FAA40A941900019120A3EC000C001C0EE
:103E7D0002C003AC42EC1203C7D003D002D001D074
:103E8D000012019EC004C005C006C0079011B8E025
:103E9D00FC1203C7D003D002D001D0001200AD1226
:103EAD0003FB9011B8EFF0AB3FAA40A9419000156C
:103EBD001209A3900011120A3E1203447003024628
:103ECD0031AB3FAA40A9419000111209A3C004C013
:103EDD0005C006C0079011B8E0FC1203C7A804A9DD
:103EED0005AA06AB07D007D006D005D004120344AF
:103EFD005014AB3FAA40A9419000111209A312031F
:103F0D00FB9011B8EFF0AB3FAA40A94190001512FC
:103F1D0009A3C004C005C006C0079011B8E0FC128B
:103F2D0003C7A804A905AA06AB07D007D006D0057C
:103F3D00D0041203446002500302463102407DE575
:103F4D0042F4704CAB3FAA40A9419000111209A355
:103F5D00C004C005C006C0079011B8E0FCE4120310
:103F6D00C7A804A905AA06AB07D007D006D005D06F
:103F7D0004120344701AAB3FAA40A94190001512D8
:103F8D0009A3900011120A3E120344600302463148
:103F9D00AB3FAA40A941900019120A3EC000C001D2
:103FAD00C002C003AC42EC1203C7D003D002D00153
:103FBD00D00012019EC004C005C006C0079011B804
:103FCD00E0FCE41203C7D003D002D001D0001200F0
:103FDD00AD1203FB9011B8EFF0AB3FAA40A9419091
:103FED0000151209A3900011120A3E12034470032A
:103FFD00024631AB3FAA40A9419000111209A3C05E
:10400D0004C005C006C0079011B8E0FCE41203C758
:10401D00A804A905AA06AB07D007D006D005D00481
:10402D001203445014AB3FAA40A94190001112094C
:10403D00A31203FB9011B8EFF0AB3FAA40A941903A
:10404D0000151209A3C004C005C006C0079011B821
:10405D00E0FCE41203C7A804A905AA06AB07D00724
:10406D00D006D005D004120344600250030246313D
:10407D00AB3FAA40A9419000151209A31203FB9072
:10408D0011B8EFF022AB3FAA40A9419000041207EE
:10409D00A520E103024190900019120A3EC000C014
:1040AD0001C002C003AC42EC1203C7D003D002D052
:1040BD0001D00012019EC004C005C006C0079011BA
:1040CD00B8E0FCA3E0FDEC1203C2D003D002D00196
:1040DD00D0001200AD1203FB9011B8EEF0A3EFF07B
:1040ED00AB3FAA40A9419000151209A390001112EF
:1040FD000A3E1203447003024631AB3FAA40A94168
:10410D009000111209A3C004C005C006C00790118C
:10411D00B8E0FCA3E0FDEC1203C2A804A905AA06B1
:10412D00AB07D007D006D005D0041203445017AB0F
:10413D003FAA40A9419000111209A31203FB90114F
:10414D00B8EEF0A3EFF0AB3FAA40A94190001512D5
:10415D0009A3C004C005C006C0079011B8E0FCA3B8
:10416D00E0FDEC1203C2A804A905AA06AB07D0070F
:10417D00D006D005D004120344600250030246312C
:10418D000242D3E542F4704FAB3FAA40A9419000E3
:10419D00111209A3C004C005C006C0079011B8E0F4
:1041AD00FCA3E0FDE41203C2A804A905AA06AB070F
:1041BD00D007D006D005D004120344701AAB3FAA25
:1041CD0040A9419000151209A3900011120A3E1248
:1041DD0003446003024631AB3FAA40A94190001948
:1041ED00120A3EC000C001C002C003AC42EC120373
:1041FD00C7D003D002D001D00012019EC004C0056B
:10420D00C006C0079011B8E0FCA3E0FDE41203C2A4
:10421D00D003D002D001D0001200AD1203FB9011DB
:10422D00B8EEF0A3EFF0AB3FAA40A94190001512F4
:10423D0009A3900011120A3E120344700302463185
:10424D00AB3FAA40A9419000111209A3C004C005BB
:10425D00C006C0079011B8E0FCA3E0FDE41203C254
:10426D00A804A905AA06AB07D007D006D005D0042F
:10427D001203445017AB3FAA40A9419000111209F7
:10428D00A31203FB9011B8EEF0A3EFF0AB3FAA40E1
:10429D00A9419000151209A3C004C005C006C007AE
:1042AD009011B8E0FCA3E0FDE41203C2A804A90537
:1042BD00AA06AB07D007D006D005D0041203446080
:1042CD00025003024631AB3FAA40A941900015129E
:1042DD0009A31203FB9011B8EEF0A3EFF022AB3F50
:1042ED00AA40A9419000041207A520E0030243ADA6
:1042FD009011B8E0F8A3E0F9A3E0FAA3E0FBC00049
:10430D00C001C002C003AB3FAA40A94190001912E1
:10431D000A3EC000C001C002C003AC42EC1203C78C
:10432D00D003D002D001D00012019ED003D002D014
:10433D0001D0001200AD9011B8120A7AAB3FAA401D
:10434D00A9419000111209A39011B8E0F8A3E0F96A
:10435D00A3E0FAA3E0FB1203445012AB3FAA40A91D
:10436D00419000111209A39011B8120A7AAB3FAA1D
:10437D0040A9419000151209A39011B8E0F8A3E0EF
:10438D00F9A3E0FAA3E0FB120344600250030246D6
:10439D0031AB3FAA40A9419000151209A302462B4B
:1043AD00AB3FAA40A9419000041207A520E10302EA
:1043BD0044C8900019120A3EC000C001C002C003DB
:1043CD00AC42EC1203C7D003D002D001D0001201D1
:1043DD009EC004C005C006C0079011B8E0FCA3E064
:1043ED00FDA3E0FEA3E0FFEC1203BDD003D002D08D
:1043FD0001D0001200AD1203FB9011B8120A7AAB76
:10440D003FAA40A9419000151209A3900011120A6C
:10441D003E1203447003024631AB3FAA40A94190BE
:10442D0000111209A3C004C005C006C0079011B841
:10443D00E0FCA3E0FDA3E0FEA3E0FFEC1203BDA8AA
:10444D0004A905AA06AB07D007D006D005D00412E3
:10445D0003445015AB3FAA40A9419000111209A386
:10446D001203FB9011B8120A7AAB3FAA40A94190F2
:10447D0000151209A3C004C005C006C0079011B8ED
:10448D00E0FCA3E0FDA3E0FEA3E0FFEC1203BDA85A
:10449D0004A905AA06AB07D007D006D005D0041293
:1044AD00034460025003024631AB3FAA40A941903C
:1044BD0000151209A31203FB02462BE542F47055B9
:1044CD00AB3FAA40A9419000111209A3C004C00539
:1044DD00C006C0079011B8E0FCA3E0FDA3E0FEA369
:1044ED00E0FFE41203BDA804A905AA06AB07D00797
:1044FD00D006D005D004120344701AAB3FAA40A9D0
:10450D00419000151209A3900011120A3E120344A6
:10451D006003024631AB3FAA40A941900019120A2F
:10452D003EC000C001C002C003AC42EC1203C7D0B4
:10453D0003D002D001D00012019EC004C005C006F8
:10454D00C0079011B8E0FCA3E0FDA3E0FEA3E0FFDF
:10455D00E41203BDD003D002D001D0001200AD1281
:10456D0003FB9011B8120A7AAB3FAA40A941900003
:10457D00151209A3900011120A3E12034470030292
:10458D004631AB3FAA40A9419000111209A3C004C6
:10459D00C005C006C0079011B8E0FCA3E0FDA3E084
:1045AD00FEA3E0FFE41203BDA804A905AA06AB070C
:1045BD00D007D006D005D0041203445015AB3FAA46
:1045CD0040A9419000111209A31203FB9011B812DA
:1045DD000A7AAB3FAA40A9419000151209A3C00465
:1045ED00C005C006C0079011B8E0FCA3E0FDA3E034
:1045FD00FEA3E0FFE41203BDA804A905AA06AB07BC
:10460D00D007D006D005D00412034460174015AB77
:10461D003FAA40A9419000151209A31203FB901166
:05462D00B8120A7A2218
:10C4F7008F3FE92405F9E43AFA78E27C117D017E61
:10C50700007F08120766E49011EAF09011E8E0FF57
:10C5170060079011E7F0E4A3F0853F4F7550017570
:10C5270051117552E27BFF7A7579571269E57BFFE6
:07C537007A75795F02C779F4
:1017EC001280D8EF6003D22122302140E49011C541
:1017FC00F09011BD120A9F000000009011C1120A56
:10180C009F00000000C224C225C226C227E490110A
:10181C008FF012C9C2E47B2C7A01F9F8C312095F6C
:10182C0040030222C5C221D216120D0D20291EC260
:10183C0016120D0D90118FEFF070030222B5D22904
:10184C00E0640260030222B5D2280222B5202803EC
:10185C00021C239011EE742DF0E4A3F09011FE7491
:10186C002DF0E4A3F0754201754311754490754554
:10187C0002FB7D02FF129EF9901190E0C4F854F027
:10188C00C868FCA3E0C4540F48FDE41203C2E4FB97
:10189C00FAF978411202A7901192120A7AE4FFFE2B
:1018AC007D207C41901192E0F8A3E0F9A3E0FAA32B
:1018BC00E0FB12019EE4FBFAF9783F1200AD120333
:1018CC00FBEC1203BDE4FBFA792078411202A790DD
:1018DC0011C6120A7A75420175431175449075450B
:1018EC00027B017D02E4FF129EF9901190E0C4F896
:1018FC0054F0C868FCA3E0C4540F48FDE41203C2C2
:10190C00E4FBFA79A0784012019EE4FBFA79807826
:10191C00451202A7901192120A7AE4FFFE7DC87C50
:10192C0042901192E0F8A3E0F9A3E0FAA3E0FB12D5
:10193C00019EE4FBFAF9783F1200AD1203FBEC12A6
:10194C0003BDE4FBFA79C878421202A79011CA12BF
:10195C000A7A7542017543117544907545027B02F4
:10196C007D02E4FF129EF9901190E0C4F854F0C887
:10197C0068FCA3E0C4540F48FDE41203C2E4FBFA74
:10198C007920784012019EE4FBFA798078451202A6
:10199C00A7901192120A7A901192E0FCA3E0FDA399
:1019AC00E0FEA3E0FF7B007AC0792878451202A7FD
:1019BC00901192120A7A901192E0FCA3E0FDA3E040
:1019CC00FEA3E0FF7B007AC0795A784612019E9004
:1019DC001192120A7AE4FFFE7DC87C42901192E0CB
:1019EC00F8A3E0F9A3E0FAA3E0FB12019EE4FBFAF2
:1019FC00F9783F1200AD1203FBEC1203BDE4FBFAC5
:101A0C0079C878421202A79011CE120A7A75420157
:101A1C007543117544907545027B037D02E4FF12FA
:101A2C009EF9901190E0C4F854F0C868FCA3E0C48F
:101A3C00540F48FDE41203C2E4FBFA79C878401253
:101A4C00019EE4FBFA798078451202A7901192125C
:101A5C000A7AE4FFFE7DC87C42901192E0F8A3E084
:101A6C00F9A3E0FAA3E0FB12019EE4FBFAF9783F3C
:101A7C001200AD1203FBEC1203BDE4FBFA79C8783B
:101A8C00421202A79011D2120A7A754201754311C3
:101A9C007544907545027B047D02E4FF129EF9901B
:101AAC001190E0C4F854F0C868FEA3E0C4540F4889
:101ABC00FF7C007D0B120806AC06AD07E41203C2D6
:101ACC00E4FBFA7920784012019EE4FBFA798078E5
:101ADC00451202A7901192120A7AE4FFFE7DC87C8F
:101AEC0042901192E0F8A3E0F9A3E0FAA3E0FB1214
:101AFC00019EE4FBFAF9783F1200AD1203FBEC12E5
:101B0C0003BDE4FBFA79C878421202A79011D612F1
:101B1C000A7A7542017543117544907545027B052F
:101B2C007D02E4FF129EF9901190E0C4F854F0C8C5
:101B3C0068FEA3E0C4540F48FF7C007D0B1208061E
:101B4C00AC06AD07E41203C2E4FBFA79207840122C
:101B5C00019EE4FBFA798078451202A7901192124B
:101B6C000A7AE4FFFE7DC87C42901192E0F8A3E073
:101B7C00F9A3E0FAA3E0FB12019EE4FBFAF9783F2B
:101B8C001200AD1203FBEC1203BDE4FBFA79C8782A
:101B9C00421202A79011DA120A7A754201754311AA
:101BAC007544907545027B067D02E4FF129EF99008
:101BBC001190E0C4F854F0C868FCA3E0C4540F487A
:101BCC00FDE41203C2E4FBFA7920784012019EE492
:101BDC00FBFA798078451202A7901192120A7AE4E6
:101BEC00FFFE7DC87C42901192E0F8A3E0F9A3E0DF
:101BFC00FAA3E0FB12019EE4FBFAF9783F1200AD68
:101C0C001203FBEC1203BDE4FBFA79C87842120212
:101C1C00A79011DE120A7A90118930281374FFF004
:101C2C00A37476F0A374B0F090118D740CF0801343
:101C3C00E518F0A3E519F0A3E51AF07882E6149004
:101C4C00118DF090118DE0FFC394035005E4A3F0C7
:101C5C00801B9011C5E0FE7002800EEE9011C5B590
:101C6C000705E024FE8002E01490118EF07882E6E5
:101C7C007014202811FDFF12C99B7BFF7A757968BF
:101C8C001269E5021DDBE490118CF090118CE0FDE3
:101C9C00C394034003021DDBE4FF12C99B90118C1B
:101CAC00E0FF90118EE02FFFE433FE9011C5E07C35
:101CBC0000B50708ECB506047F1580027F2012C919
:101CCC005B90118CE0FD7F0112C99B90118CE0FFA1
:101CDC0090118EE02FFFE433FE90118DE0FDD3EFD9
:101CEC009D7480F86E98400C7BFF7A75797D126933
:101CFC00E5021DD290118CE0FE90118EE0FD2EFFBE
:101D0C00C007EEFFED2FFFE433FEEF7805C333CEB3
:101D1C0033CED8F9FF901189E0FBA3E0FAA3E02FB2
:101D2C00F9EA3EFAD00712C4F790118CE0FD7F0A55
:101D3C0012C99B30224090118CE0FF90118EE02F45
:101D4C00FFE433FE9011C5E07C00B50729ECB50625
:101D5C0025EF7805C333CE33CED8F9FF901189E047
:101D6C00FBA3E0FAA3E02FF9EA3EFA7542017543B2
:101D7C00117544B8804D90118CE0FF90118EE02FBE
:101D8C00FFE433FEEF7805C333CE33CED8F9FF90A2
:101D9C001189E0FBA3E0FAA3E02FF9EA3EFAC003B5
:101DAC00C002C001901189A3E0FAA3E02FF9EA3E2A
:101DBC00FA90000D120AFA8B428A438944D001D062
:101DCC0002D003127B3E90118CE004F0021C979021
:101DDC0011C5E075F020A430280F24B0F9747635C5
:101DEC00F0FA90118974FF800D251AF9E51935F078
:101DFC00FA901189E518F0A3EAF0A3E9F030235A20
:101E0C007D03E4FF12C99B7BFF7A75799112C77928
:101E1C009011BCE075F003A4240DFF90118EE0FE30
:101E2C009011C5E0C39EFD12C99B200E0A302407F9
:101E3C00C223E4FF12CA32200F030222B53025035D
:101E4C000222B59011BCE004F0E0640360030222AE
:101E5C00B5C223FF12CA320222B520220302202A65
:101E6C007D03E4FF12C99B7BFF7A7579A612C779B3
:101E7C0090118EE0FF9011C5E0C39FFD7F1312C936
:101E8C009B200E0A302407C222E4FF12CA32300F04
:101E9C0053202550C222E4FF12CA32901189E0FB74
:101EAC00A3E0FAA3E0F912078CFF7E00901189A33E
:101EBC00A3E090000D120AFAA801AC02AD037B015D
:101ECC007A1179B81207663028129011C5E0FF60BC
:101EDC0003B40110D22A788076F180089011C5E005
:101EEC00FF12C91530100F20260C123E2012C9C249
:101EFC009011BD120A7A30102D12C9C2A804A9057E
:101F0C00AA06AB079011BDE0FCA3E0FDA3E0FEA385
:101F1C00E02446FFE43EFEE43DFDE43CFCD3120924
:101F2C005F4003123E2030103B12C9C2A804A90521
:101F3C00AA06AB079011BDE0FCA3E0FDA3E0FEA355
:101F4C00E024F4FFEE3401FEE43DFDE43CFCD3124E
:101F5C00095F4010901189E0FBA3E0FAA3E0F97D42
:101F6C00F7123E2D20100A9011BD120A9F0000009E
:101F7C000030111C202719901189E0FBA3E0FAA373
:101F8C00E0F97D01123E2D12C9C29011C1120A7ADC
:101F9C0030113A12C9C2A804A905AA06AB079011C0
:101FAC00C1E0FCA3E0FDA3E0FEA3E02446FFE43E79
:101FBC00FEE43DFDE43CFCD312095F401090118916
:101FCC00E0FBA3E0FAA3E0F97D01123E2D30113BBA
:101FDC0012C9C2A804A905AA06AB079011C1E0FC5E
:101FEC00A3E0FDA3E0FEA3E024F4FFEE3401FEE445
:101FFC003DFDE43CFCD312095F4010901189E0FBDD
:10200C00A3E0FAA3E0F97D09123E2D301103022260
:10201C00B59011C1120A9F000000000222B57D0389
:10202C00E4FF12C99B7882E6D39400500330283722
:10203C00901189E0FBA3E0FAA3E0F99000191209D2
:10204C00A3E4FBFAF9F81203444014901189E0FB65
:10205C00A3E0FAA3E0F99000041207A530E2087B94
:10206C00FF7A7579BB80067BFF7A7579C812C779C0
:10207C007F1212C95B7BFF7A7579D512C7797F13F2
:10208C0012C95B7BFF7A7579DB12C779200E0C3095
:10209C002409C229C228D216120D0D200F030221C9
:1020AC00933025030221937882E6D394004061900B
:1020BC001189E0FBA3E0FAA3E0F912078CFFD3949B
:1020CC0004504DEF940040489000191209A3E4FB12
:1020DC00FAF9F81203445038D222901189E0FBA38C
:1020EC00E0FAA3E0F912078CFF7E0090000D120AB3
:1020FC00FA78B87C117D0112076690118EE0FF9082
:10210C0011C5E0C39FFD7F1312C99B7F0112CA3218
:10211C0030282A9011C5E0FF64026004EFB4031D5F
:10212C00D223E49011BCF090118EE0FF9011C5E029
:10213C00C39FFD7F0D12C99B7F0112CA3230283715
:10214C009011C5E0640B702FD22A788076F112CAF8
:10215C0052E4FDFF12C99B7BFF7A7579DD12C779BA
:10216C007D01E4FF12C99B7BFF7A7579F012C77968
:10217C007FB87E0B12C74E30280D9011C5E0B40C01
:10218C0006E4F58475EF1030102A2026279011C52F
:10219C00E070122028077882E614F0800E9011C5AA
:1021AC00740CF080069011C5E014F012C9C29011A5
:1021BC00BD120A7A30104812C9C2A804A905AA0691
:1021CC00AB079011BDE0FCA3E0FDA3E0FEA3E0246F
:1021DC0046FFE43EFEE43DFDE43CFCD312095F40C7
:1021EC001E9011C5E070122028077882E614F0804A
:1021FC000E9011C5740CF080069011C5E014F020FF
:10220C00100A9011BD120A9F00000000302808909F
:10221C00118C740DF080077882E690118CF03011DF
:10222C00252027229011C5E02401FFE433FE9011F4
:10223C008CE0FD7C001208189011C5EDF012C9C29B
:10224C009011C1120A7A30114312C9C2A804A9050F
:10225C00AA06AB079011C1E0FCA3E0FDA3E0FEA32E
:10226C00E02446FFE43EFEE43DFDE43CFCD31209D1
:10227C005F40199011C5E02401FFE433FE90118CEE
:10228C00E0FD7C001208189011C5EDF020110A90A9
:10229C0011C1120A9F0000000030100D30110A20ED
:1022AC002807E49011C5F0D228A20E9224A20F9216
:0922BC0025A2109226A21192271E
:0122C50022F6
:03CA96002020005D
:0AC5F600AB51AA52A9531207A5FF8A
:02C600008F5455
:10C60200E478B0F6E5541392927F0A7E0012C0419C
:10C61200D2937F0A7E0012C041C293E554C313F540
:0AC622005478B006E6C3940840DA2D
:01C62C0022EB
:02BC9E008F71A4
:10BCA000C293E4F58475D2FF75D30F7F0AFE12C0EC
:10BCB0004175840F43A504AF7112C60075840F53FC
:10BCC000A5FBD2927F0A7E0012C041E47878F61874
:10BCD000F6787976013092077878E6797947F6D266
:10BCE000937F0A7E0012C041C2937F0A7E0012C079
:10BCF000417879E625E0F6787706E6C3940840D5E2
:10BD0000E4F584F5D2F5D37F0AFE12C0417878E6D7
:01BD1000FF33
:01BD1100220F
:06AE74008B518A52895344
:10AE7A00C293E4F58475D2FF75D30F7F0AFE12C020
:10AE8A004175840F43A5047FBF12C60075840F5312
:10AE9A00A5FBD2927F0A7E0012C041E478ADF6E4A7
:10AEAA0078AEF678ACF678AF760130920778AEE6EF
:10AEBA0079AF47F6D2937F0A7E0012C041C2937FD0
:10AECA000A7E0012C04178AFE625E0F678AC06E6C5
:10AEDA00C3940840D578ADE6FFC39403501908E639
:10AEEA00FEEFFDC374059DFDE49400AB51AA52A97F
:10AEFA00538D82F583801E78ADE6FFC39405501802
:10AF0A0008E6FEEF7C0024FDF582EC34FFF583AB06
:10AF1A0051AA52A953EE801178ADE6B4060E08E69E
:10AF2A00AB51AA52A9539000021207E478AD06E683
:10AF3A00C39407500302AEA9E4F584F5D2F5D37F92
:05AF4A000AFE02C041F7
:10C696008F458D46C293E4F58475D2FF75D30F7F1F
:10C6A6000AFE12C04175840F43A504AF4512C600A9
:10C6B600AF4612C600E4F584F5D2F5D37F0AFE0232
:02C6C600C04171
:10BC28008B518A528953C293E4F58475D2FF75D338
:10BC38000F7F0AFE12C04175840F43A5047FBE1210
:10BC4800C60090000512C5F690000412C5F6AB5167
:10BC5800AA52A95390000312C5FCAB51AA52A9538A
:10BC680012078CFF12C600AB51AA52A953900001CB
:10BC780012C5FC7F0112C600AB51AA52A95390000D
:10BC88000212C5FCE4FF12C600E4F584F5D2F5D330
:06BC98007F0AFE02C0411C
:10C583008D72EF14601614601914601C14601F146C
:10C59300602224057025AD727F86801CAD727F8872
:10C5A3008016AD727F8C8010AD727F84800AAD726D
:0CC5B3007F828004AD727F8012C6962249
:10A813008B088A09890A12078CFFF47049AB0BAACB
:10A823000CA90D900007743F1207E4900006743FD3
:10A833001207E4900004743F1207E4900003743F8E
:10A843001207E4900001743F1207E4743F1207D229
:10A85300AB0BAA0CA90D900005742D1207E4900010
:10A8630002742D02A910EFC4540F2430AB0BAA0CB1
:10A87300A90D1207D2AB08AA09A90A12078C540F13
:10A883002430AB0BAA0CA90D9000011207E4900031
:10A8930002742D1207E4AB08AA09A90A9000011259
:10A8A30007A5C4540F2430AB0BAA0CA90D900003C9
:10A8B3001207E4AB08AA09A90A9000011207A554DC
:10A8C3000F2430AB0BAA0CA90D9000041207E490DF
:10A8D3000005742D1207E4AB08AA09A90A90000227
:10A8E3001207A5C4540F2430AB0BAA0CA90D90007A
:10A8F300061207E4AB08AA09A90A9000021207A5E9
:10A90300540F2430AB0BAA0CA90D9000071207E4D7
:08A91300900008E41207E422A1
:10A5EE008B0E8A0F891012078CF47049AB11AA12C8
:10A5FE00A913900007743F1207E4900006743F12EF
:10A60E0007E4900004743F1207E4900003743F12B5
:10A61E0007E4900001743F1207E4743F1207D2ABB7
:10A62E0011AA12A913900005743A1207E4900002C1
:10A63E00743A02A6F8AB0EAA0FA9109000031207E7
:10A64E00A5C4540F2430AB11AA12A9131207D2AB12
:10A65E000EAA0FA9109000031207A5540F2430ABB9
:10A66E0011AA12A9139000011207E4900002743A85
:10A67E001207E4AB0EAA0FA9109000041207A5C48E
:10A68E00540F2430AB11AA12A9139000031207E441
:10A69E00AB0EAA0FA9109000041207A5540F243078
:10A6AE00AB11AA12A9139000041207E490000574CE
:10A6BE003A1207E4AB0EAA0FA9109000051207A5D7
:10A6CE00C4540F2430AB11AA12A91390000612071E
:10A6DE00E4AB0EAA0FA9109000051207A5540F2483
:10A6EE0030AB11AA12A9139000071207E4900008CC
:05A6FE00E41207E42254
:10C2E5007B017A12790812AE74901208E0F4603F6F
:10C2F500750B01750C12750D0E7B017A12790812FA
:10C30500A8137B017A12790E12C7797BFF7ACA7955
:10C315009612C77975110175121275130E7B017A84
:0FC3250012790812A5EE7B017A12790E12C779F0
:01C3340022E6
:10C9FB00E4FF12BC9E787CEFF6F460047F018002AA
:02CA0B007F00AA
:01CA0D002206
:07000300E4FD7F8E02C696AA
:049EF9008D408B41CC
:109EFD007B08E4FD12C955E490119EF0E54054082D
:109F0D00D394004003D38001C392B300000000003E
:109F1D00000000000000000000000000000000D262
:109F2D00B000000000000000000000000000000074
:109F3D000000000000C2B0E54025E0F54090119E04
:109F4D00E004F0E0B404B5E490119EF0E54154084E
:109F5D00D394004003D38001C392B30000000000EE
:109F6D00000000000000000000000000000000D212
:109F7D00B000000000000000000000000000000024
:109F8D000000000000C2B0E54125E0F54190119EB2
:109F9D00E004F0E0B404B5E490119EF0E54575F0F1
:109FAD0008A4FF90119EE0FDC39FE5F06480F87456
:109FBD008098505CED9400400FE05407700A042522
:109FCD0044F544E43543F543C2B000000000000001
:109FDD000000000000000000000000000000AB4287
:109FED00AA43A94412078C25E0FFA2B4E4334F1213
:109FFD0007D2D2B0000000000000000000000000F9
:10A00D00000000000000000090119EE004F0808C24
:10A01D00D2B20000000000000000000000000000AF
:06A02D000000000000002D
:01A03300220A
:04AD98007D0AAF453C
:04AD9C008D468B470E
:10ADA000D2B200000000000000000000000000001F
:10ADB000000000000000C2B200000000000000001F
:10ADC0000000000000000000000000007B08E4FD1F
:10ADD00012C955E490119EF0E5465408D394004002
:10ADE00003D38001C392B300000000000000000004
:10ADF0000000000000000000000000D2B0000000D1
:10AE00000000000000000000000000000000000042
:10AE100000C2B0E54625E0F54690119EE004F0E062
:10AE2000B404B5E490119EF0E5475408D394004073
:10AE300003D38001C392B3000000000000000000B3
:10AE40000000000000000000000000D2B000000080
:10AE500000000000000000000000000000000000F2
:10AE600000C2B0E54725E0F54790119EE004F0E010
:03AE7000B404B572
:01AE730022BC
:10C38300E490116EF0EF5480D394004003D3800106
:10C39300C392B30000000000000000000000000092
:10C3A30000000000000000D2B00000000000000008
:10C3B30000000000000000000000000000C2B0EF19
:0DC3C30025E0FF90116EE004F0E0B408B832
:01C3D000224A
:02AF4F008F452C
:10AF5100E4FB7D0712AD9CE4FB12AD98E4FF12C344
:10AF610083E4FF12C3837B0212AD98E4FF12C38313
:10AF7100E4FF12C383E490116BF090116BE0FBC30B
:10AF8100940750697D0CAF4512AD9C90116BE0FFA9
:10AF9100700AA37403F0A37420F08017EF90116C72
:10AFA100B402097401F0A374D9F08007740FF0A3FF
:10AFB10074FFF090116CE0C4F854F0C8A3E0C454DD
:10AFC1000F48FF12C38390116DE0540FC4F8540F62
:10AFD100C868FF12C383E4FF12C383E4FF12C38373
:10AFE1007F3A12C38390116BE004F0808DE4FB7D06
:10AFF1000DAF4512AD9C7FFF12C3837FFF12C38348
:0FB00100E4FF12C383E4FF12C3837F1402C383EF
:10C87100E4FB7D0912AD9CD2B20000000000000073
:0EC88100000000000000000000000000002287
:04C7A3008F6F8D7097
:10C7A7007B017A12791C12B7B6E57090121C6006ED
:10C7B700E04401F08004E054FEF090121CE0FDAF6D
:04C7C7006F02BB9EA4
:10C92D007B017A12791DE4FF12B7B690121DE0302B
:07C93D00E7037F00227F01E8
:01C9440022D0
:10C8FC007B017A12791EE4FF12B7B690121EE0305B
:08C90C00E704540FFF227F0035
:01C914002200
:10C8C8007B017A12791F12B7B690121FE0FFF4604D
:0AC8D80007EF60047F0180027F007B
:01C8E2002233
:02C099008F69AD
:10C09B0075840FE4F5A6C290C294D295D2967F0117
:10C0AB00FE12C041C296E4F56A7F0A7E0012C041BF
:10C0BB0030A709056AE56AC394C840ED75840F750E
:10C0CB00A6FFD290C295A22092948569A07F017E93
:10C0DB000012C041D2967F017E0012C041C2967FF2
:06C0EB00017E0002C041CD
:10BD8000D23475840F43A580C2977F017E0012C70D
:10BD90004ED2977F327E0012C74EC296C295C29491
:10BDA00075840F75A6FF43A503D290D291C2207F60
:10BDB0003412C099C2207F0B12C099C2207F30126A
:10BDC000C099C2207F0212C099C2207F0C12C09974
:10BDD000C2207F0112C099C2207F3412C099C220B4
:0CBDE0007F0612C099C2207F3002C0997B
:0DCA5200C2207F0112C099E4FDFF02C99BC4
:10CA3200EF6006C2207F0F8004C2207F0C12C099D3
:01CA420022D1
:10C99B00ED5403C43354E0FEEF541F44804EFFC2EA
:04C9AB002002C0990D
:10C95B008F68E568640D600BE568640A6005D2209A
:06C96B0012C099AF682222
:10C7CB008B1B8A1C891DAB1BAA1CA91D12078C6015
:10C7DB0015051DE51D7002051C14F912078CFFD2FF
:07C7EB002012C09980E0223A
:1000A600020467E86480F8E933E83360110460F01D
:1000B600ED33EC337009E8FCE9FDEAFEEBFF2204C0
:1000C60060DED3EB9FEA9EE99DE8C2E78CF0C2F7BB
:1000D60095F0400CE8CCF8E9CDF9EACEFAEBCFFB87
:1000E60012043285D0F05804700320D5B3E80470AA
:1000F600075002B2D502047192D5EC0460F7E4CC45
:10010600C0E0C398F8603B94186008400DD0E0FB4F
:10011600020449E4FBFAC9FC8028E830E406E4C995
:10012600FBE4CAFCE830E305E4C9CACBFCE85407A3
:100136006010F8C3E913F9EA13FAEB13FBEC13FCAE
:10014600D8F130F52FC3E49CFCEF9BFFEE9AFEED51
:1001560099FDD0E0FBEF4E4D4C701222DB030204FA
:100166006EEC2CFCEF33FFEE33FEED33FDED30E7A6
:10017600EB020449EF2BFFEE3AFEED39FDD0E0FB32
:1001860050130BBB0003020471ED13FDEE13FEEFDB
:0801960013FFEC13FC02044905
:10019E00EC4D6011E8497017ED33EC3304600DE45B
:1001AE00FCFFFEFD22E933E8330470F80204671207
:1001BE00043258046009E4CC248150062850090208
:1001CE00047128400302046EC0E0EB4A7044B9800B
:1001DE0006D0E0FB02045DEF4E701CBD8008EBFF05
:1001EE00EAFEE9FD80EBE98DF0A4FEE5F002028760
:1001FE00E9CDF9EAFEEBFFEF89F0A4FCE5F0CE893C
:10020E00F0A42EFFE435F0CD89F0A42DFEE435F0F8
:10021E008067EF4E7005BD80D780C3EF8BF0A4AC26
:10022E00F0EE8BF0A42CFCE435F0F8EF8AF0A42C61
:10023E00E5F038FCE433CB8DF0A42CFCE5F03BF874
:10024E00EE8AF0A42CFCE5F038F8E433CF89F0A464
:10025E002CFCE5F038CF3400CE89F0A42FFFE5F06A
:10026E003EFEE433C98DF0A42EFEE5F039CD8AF0C2
:10027E00A42FFFE5F03EFEE43DFD33D0E0FB50073A
:10028E000BBB000F020471EC2CFCEF33FFEE33FEC0
:06029E00ED33FD020449EE
:1002A400020471EC5D046005E859047003020467FC
:1002B400120432580460F6EC4860F2EC7004FDFE5F
:1002C400FF22C860DB2481C85009C398600250062D
:1002D40002046E9850CAF582E9294B4A7005AB8234
:1002E40002045D75F0007C1A7880C3EF9BEE9AEDF2
:1002F40099400DC3EF9BFFEE9AFEED99FDE842F0A5
:10030400DC23ACF0D0E0FFD0E0FED0E0FDAB8220F7
:10031400E7101BEB60BAEC2CFCEF33FFEE33FEED81
:1003240033FD020449E803F830E705C0F075F00036
:10033400EF2FFFEE33FEED33FD40B830E7C280AA65
:1003440074F8CC6480CCC86480C8F58204604FC360
:10035400EB9FF5F0EA9E42F0E99D42F0E89C45F0FF
:10036400603C501DE5825FFFE582D313CB5BCBF489
:100374002B5582FB50280ABA002409B900200880B2
:100384001DE5825BFBE582D313CF5FCFF4C3132F4C
:100394005582FF50090EBE00050DBD00010CC3EBD4
:1003A4009FF5F0EA9E42F0E99D42F0E89C45F0603A
:0903B40007CC4820E701B3EC225C
:1003BD0075F020800E75F010800575F0087D007EBB
:1003CD00007F003392D530D50312093BEC3340103A
:1003DD00EF33FFEE33FEED33FDEC33FCD5F0ED22C4
:0E03ED00E5F0247EA2D513CC92E7CDCEFF2200
:1003FB00EDD2E7CD33EC3392D524814006E4FFFEFA
:10040B00FDFC22FCE4CFCECDCC24E0501174FF8058
:10041B00EDC3CC13CCCD13CDCE13CECF13CF0470F5
:07042B00F030D5DE02093BB1
:10698300E563244FF8E6056322784C301E02784F06
:10699300E475F001120AEA02078C2017EB7F2ED26E
:1069A300178018EF540F2490D43440D4FF301B0BBE
:1069B300EF24BFB41A0050032461FFE5646002159D
:1069C300640567E56770020566301E0D784CE47553
:1069D300F001120AEAEF0207D202C95B7403D21E66
:1069E3008003E4C21EF5638B4C8A4D894EE4F56443
:1069F300F566F567E56460077F201269BE80F5756B
:106A030065FFC218C217C219C21AC21CC21DC21F17
:106A130012698CFF700D301E057F001269CFAF67BE
:106A2300AE6622B4255FC2D5C21B12698CFF24D087
:106A3300B40A00501A75F00A786430D50508B6FF19
:106A43000106C6A426F620D5047002D21A80D924E2
:106A5300CFB41A00EF5004C2E5D21B026CBCD218AB
:106A630080C6D21780C0D21980BCD2D580BAD21CBE
:106A730080B47F201269BE2019077401B5640040F9
:106A8300F1126983FF1269BE0269F7D21FD21D801A
:106A930095126983FB126983FA126983F94A4B7071
:106AA3000679B37A6D7BFF20192EE564602A7E0098
:106AB3008E827583001207A560060EEE656570F081
:106AC300C2D5EBC0E0EAC0E0E9C0E0EE126D1CD035
:106AD300E0F9D0E0FAD0E0FB12078CFF60AAEBC02C
:106AE300E0EAC0E0E9C0E01269BED0E02401F9D0D9
:106AF300E03400FAD0E0FBE5650460DCD565D980BD
:106B030087D21980A2126CFF60F7E5657001041249
:106B130004A7A965600DE565600914F565126DA606
:106B2300EF60F3EA30E702F404C3995077EAF425FF
:106B3300650430E701E404F565800D126CFF60C164
:106B4300EA056525651204A7EA7862F630E701E4F1
:106B5300256504D56504201C0114126D1CE4C0E0F6
:106B6300126DA67862E6601320E70714F61269A691
:106B7300802204F6D0E014C0E07F001269A6E56528
:106B8300600712699D1565800B301C0312699DD047
:106B9300E00269F7D0E00480C5126CFF60A0E565F0
:106BA300041204A77862EAF6E565201C026001047A
:056BB3002404126D1C1A
:106BB80074FF04C0E0126DA61269A6E565201C02E8
:106BC800600312699DD0E0B565E87F451269B07829
:106BD80062E67F2B30E7047F2DF404C0E01269BE23
:106BE800D0E075F00A84C0F01269A7D0E01269A756
:106BF8000269F7791080027908C21DC21F8008D285
:106C0800D5790A8004790AC2D5E565047002F5656C
:106C1800E4FAFDFEFF126983FC7B08201813126951
:106C280083FD7B1030170A126983FE126983FF7B8C
:106C380020EC3382D592D55013C3E43017069FFF5A
:106C4800E49EFEE42018039DFDE49CFCE4CBF8C21E
:106C580018EC700CCFCECDCCE824F8F870F3801780
:106C6800C3EF33FFEE33FEED33FDEC33FCEB33FBC8
:106C7800994002FB0FD8E9EB301805F8D0E0C4487A
:106C8800B218C0E00AEC4D4E4F78207B0070C2EA83
:106C9800B5650040BCC0E0126D1ED0F0D0E02018F1
:106CA80004C4C0E0C4B218C0F01269A7D0F0D5F08F
:106CB800EB0269F7120B2A6A94536BFB586A654C0E
:106CC8006A61426BFF4F6C07446C07496A7A436CF0
:106CD8000D556B3E466B9C456B08476DD3506A69F2
:106CE8002D6A6D2E6A902B6A71236A8E206DBC2ADC
:106CF8006A294800006A88E565B4FF0375650612CD
:106D08006983FC126983FD126983FE126983FF7827
:106D18005B0204D6790AA2D5201A14301C09B910CE
:106D2800020404B9080104A2D5201D025001042060
:106D380019689219B564005034C0E07F20301A19E0
:106D48007F30A219721D721C500F126D75C219C2C4
:106D58001DC21CC21F7F30800F301C03E9C0E01227
:106D680069BE301C03D0E0F9D0E0B564CC301C1704
:106D78007F30B9100C1269BE7F58301B077F7880AE
:106D880003B908031269BE3019057F2D0269BE7F59
:106D980020201FF87F2B201DF322921980CF7F001F
:106DA800B407005005245BF8E6FF22286E756C6C6A
:106DB8002900D2181269833018F8C218786430D5BF
:106DC8000108F6026A292D504349581269832403A1
:106DD800B405004001E4906DCE931269AF743A1285
:0A6DE80069AFD21A756404026BFB58
:0DCA5F00ED33EC3360065004EC6480FC22E3
:10B0C5008F478E468D458C4474FFFFFEFDFCAB47D4
:10B0D500AA46A945A844C312095F602C7F807E96C5
:10B0E5007D187C4BAB47AA46A945A844120344608A
:10B0F5000250157F807E967D187CCBAB47AA46A96A
:10B1050045A8441203445009AF47AE46AD45AC448B
:10B1150022AF47AE46AD45AC441203FB8F4B8E4A7A
:10B125008D498C48EC1203BDC8ECC8C9EDC9CAEEFF
:10B13500CACBEFCBAF47AE46AD45AC441200A9E450
:10B14500FBFAF9F8120344601A401874FF254BF511
:10B155004BE54A34FFF54AE54934FFF549E54834FE
:10B16500FFF548AF4BAE4AAD49AC48EC1203BD22E2
:10A3C1008F428E418D408C3FE4FFFE7D807C3FAB10
:10A3D10042AA41A940A83F1203447009AF42AE41CD
:10A3E100AD40AC3F22AF42AE41AD40AC3F12047C28
:10A3F100FBAF46AE45AD44AC4312047CFFBF010840
:10A40100E4FFFE7D807C3F22EF64046022EB640464
:10A41100601DBB0127E4FFFEFDFCAB46AA45A94434
:10A42100A84312034460084006E4FFFEFDFC2274C9
:10A43100FFF546F545F544F54302A4CFE4F547F5AC
:10A4410048FFFEFDFCAB42AA41A940A83F120344CC
:10A45100504BAF46AE45AD44AC431203FB8E478F24
:10A4610048AC47AD48EC1203C2C8ECC8C9EDC9CA33
:10A47100EECACBEFCBAF46AE45AD44AC431200A91B
:10A48100E4FBFAF9F812034470A5AF42AE41AD40C6
:10A49100AC3F1204968F428E418D408C3FAF42AE4D
:10A4A10041AD40AC3F12A1A1AB46AA45A944A84386
:10A4B10012019E12B6BF8F468E458D448C43E548EE
:10A4C10030E00B1204968F468E458D448C43AF4687
:07A4D100AE45AD44AC43228F
:10043200E9D2E7C933E833F892D5EDD2E7CD33EC10
:0704420033FC5002B2D52289
:10044900EC30E7100FBF000C0EBE00080DBD000414
:100459000BEB6014A2D5EB13FCED92E7FD2274FFC0
:10046900FCFDFEFF22E480F8A2D574FF13FC7D8019
:03047900E480EF2D
:10047C00ED33EC33601004700FED547F7005740293
:0A048C0092E0227404220422E4220C
:10049600ED33EC33600A047003BD8004ECB2E7FC74
:0104A6002233
:1004A700F920E72824F950037907E4F42402FB181C
:1004B700DBFDE624FB5014E9600DE4F618E604F6CC
:0F04C700B40A08E4F6D9F57401F60A22C2D52268
:1004D600ED33EC3392D5FA602AB4FF33EDC2E77BF5
:1004E600FF60067A0479FBE4227A05790420D504B4
:1004F6007A0479FF224E614E002B494E46002D4963
:100506004E4600E47A08F608DAFC7B00740722E817
:10051600C0E0ECC0E0EDC0E0EEC0E0EFC0E0EA75A0
:10052600F010A4CAABF075F04DA42BFBE435F0FC3B
:10053600EA2410FAEB34C5FBEC34D9FCEDC2E7FF34
:1005460075F056A4F42411C5F0F434C58FF0A42A2E
:10055600E5F03BE43CF620E714120609D0E0FFD0B4
:10056600E0FED0E0FDD0E0FC1202A78014F40412F5
:100576000609D0E0FFD0E0FED0E0FDD0E0FC12019D
:100586009ED0E0F8E6FAEDD2E7CD33EC332482FBD9
:10059600E4C3CF33CFCE33CECD33CD33DBF37B07BE
:1005A60075F00A846004F6081B0AE5F0F6088FF079
:1005B600740AA4FFACF08EF0740AA42CFEACF050C2
:1005C600010C8DF0740AA42CFDE435F0F608DBDE90
:0305D60074072285
:10B6870033DA929E35B16011377FE5FE392184891F
:10B697003AAEC3FF3C1D955B3D6358473E75FDF0D1
:10B6A7003F3172183F800000C2D50204710204675F
:10B6B700BD80FA50F302046EED33EC330460F17B86
:10B6C7003B7AAA79B8783F12019EED33EC3392D5D5
:10B6D700247B5011A2D570DB500BED44802404501D
:10B6E70004A2D580CEEFFBEEFAEDF9ECF81203FBDE
:10B6F700EFF582F404FC1203C71200ADC08290B6C6
:10B70700877409120658ED33CC33D0F092D525F063
:0AB71700A2D57001C313CC13FD226C
:10A16D003E9248DA3ECCCCCD3F2AAAAB400000004F
:10A17D003F8000003F9837F03FB504F33FD744FCD4
:10A18D003E3172173EB172173F0515913EDE5BD918
:10A19D00D2168002C216EDD2E7F8CD33EC3304703F
:10A1AD000BBD800592D502047102046740FBD314E8
:10A1BD0060F2F5F07C3FEE7A00C39496C8948B4024
:10A1CD00230AC89469C8941A401A0AC89468C89496
:10A1DD001F40110AC8945AC89425400805F07A000A
:10A1ED00CDC2E7CDC0F08C498D4A8E4B8F4CEA2302
:10A1FD0023C0E0247DF582E434A1F583120A2E12EA
:10A20D0000ADECC0E0EDC0E0EEC0E0EFC0E0120A42
:10A21D0005A849A94AAA4BAB4C1200A9D0E0FBD026
:10A22D00E0FAD0E0F9D0E0B2E7F81202A78C498D40
:10A23D004A8E4B8F4C90A16D7403120649A849A903
:10A24D004AAA4BAB4C12019ED0E0600F2489F582D7
:10A25D00E434A1F583120A2E1200AD8C498D4A8E7D
:10A26D004B8F4CD0E0C3947FFDE49400FC1203C2ED
:10A27D007B187A727931783F12019EA849A94AAAB2
:10A28D004BAB4C1200AD30160B7BD97A5B79DE7877
:05A29D003E12019E22AB
:1005D9003F8000004120000042C80000447A00002A
:1005E900461C400047C35000497424004B189680AC
:1005F9004CBEBC205A0E1BCA6753C21C749DC5AEA3
:10060900FB60065407601C2323120637EB5438603D
:100619000912062312063212019EECF8EDF9EEFAE0
:10062900EFCB22EB12063280F1543803241C9005DB
:10063900D9FE93FC0EEE93FD0EEE930ECE93FF22A0
:10064900C0E0EFFBEEFAEDF9ECF812019ED0E0F50F
:10065900F0EFFBEEFAEDF9ECF8120A05A3A3A3A358
:10066900E8C0E0E9C0E0EAC0E0EBC0E0C0F0120198
:100679009E120A2EA3A3A3A31200ADD0F0D0E0FBD3
:0D068900D0E0FAD0E0F9D0E0F8D5F0D422AE
:0300000002BB122E
:0CBB1200787FE4F6D8FD7581B602BB59BF
:10069600E709F608DFFA8046E709F208DFFA803E46
:1006A60088828C83E709F0A3DFFA8032E309F60833
:1006B600DFFA8078E309F208DFFA807088828C839B
:1006C600E309F0A3DFFA806489828A83E0A3F6084F
:1006D600DFFA805889828A83E0A3F208DFFA804C29
:1006E60080D280FA80C680D4806980F28033801000
:1006F60080A680EA809A80A880DA80E280CA803369
:1007060089828A83ECFAE493A3C8C582C8CCC583E0
:10071600CCF0A3C8C582C8CCC583CCDFE9DEE780B0
:100726000D89828A83E493A3F608DFF9ECFAA9F02F
:10073600EDFB2289828A83ECFAE0A3C8C582C8CC85
:10074600C583CCF0A3C8C582C8CCC583CCDFEADE9E
:10075600E880DB89828A83E493A3F208DFF980CC00
:1007660088F0EF60010E4E60C388F0ED2402B404F9
:100776000050B9F582EB2402B4040050AF232345A0
:0607860082239006E673D9
:10078C00BB010689828A83E0225002E722BBFE026B
:09079C00E32289828A83E493229E
:1007A500BB010CE58229F582E5833AF583E0225009
:1007B50006E92582F8E622BBFE06E92582F8E22253
:0D07C500E58229F582E5833AF583E493226D
:1007D200BB010689828A83F0225002F722BBFE0106
:0207E200F32200
:1007E400F8BB010DE58229F582E5833AF583E8F04B
:1007F400225006E92582C8F622BBFE05E92582C8F7
:02080400F222DE
:10080600EF8DF0A4A8F0CF8CF0A428CE8DF0A42E06
:02081600FE22C0
:10081800BC000BBE0029EF8DF084FFADF022E4CCC4
:10082800F875F008EF2FFFEE33FEEC33FCEE9DEC8D
:10083800984005FCEE9DFE0FD5F0E9E4CEFD22EDD3
:10084800F8F5F0EE8420D21CFEADF075F008EF2F1D
:10085800FFED33FD4007985006D5F0F222C398FD0E
:050868000FD5F0EA22AB
:10086D00C2D5EC30E709B2D5E4C39DFDE49CFCEEA6
:10087D0030E715B2D5E4C39FFFE49EFE120818C3FE
:10088D00E49DFDE49CFC800312081830D507C3E4F9
:06089D009FFFE49EFE2215
:1008A300A3F8E0C5F025F0F0E58215827002158308
:0608B300E0C838F0E82265
:1008B900BB010A89828A83E0F5F0A3E0225006870A
:1008C900F009E71922BBFE07E3F5F009E3192289CC
:0B08D900828A83E493F5F074019322FF
:1008E400BB010789828A83020C92500B09C5F02749
:1008F400F7C5F01937F722BBFE0D09F8E325F0F32D
:10090400C5F019E338F322F889828A8374019325A8
:08091400F0C5F0F8E49338226D
:10091C00BB010A89828A83F0E5F0A3F0225006F726
:0F092C0009A7F01922BBFE06F3E5F009F3192223
:0E093B00C3E49FFFE49EFEE49DFDE49CFC22CD
:10094900EB9FF5F0EA9E42F0E99D42F0EC6480C825
:0609590064809845F022C5
:10095F00EB9FF5F0EA9E42F0E99D42F0E89C45F0EE
:01096F002265
:10097000E8600FEFC333FFEE33FEED33FDEC33FCE5
:03098000D8F12289
:10098300BB010789828A830209F95005E9F8020944
:10099300EDBBFE05E9F8020CA889828A83020A05E9
:1009A300BB010DE58229F582E5833AF5830209F956
:1009B3005007E92582F80209EDBBFE07E92582F815
:1009C300020CA8E58229F582E5833AF583020A053C
:1009D300BB010789828A83020A7A5005E9F8020A71
:0A09E3006EBBFE05E9F8020CC1220C
:0C09ED00E6FC08E6FD08E6FE08E6FF2236
:0C09F900E0FCA3E0FDA3E0FEA3E0FF2271
:100A0500E493FC740193FD740293FE740393FF2237
:0D0A1500E6FB08E6F908E6FA08E6CBF82251
:0C0A2200E0F8A3E0F9A3E0FAA3E0FB2257
:100A2E00E493F8740193F9740293FA740393FB221E
:100A3E00BB010DE58229F582E5833AF583020A2290
:100A4E005007E92582F8020A15BBFE07E92582F850
:100A5E00020CB4E58229F582E5833AF583020A2E6B
:0C0A6E00ECF608EDF608EEF608EFF622B4
:0C0A7A00ECF0A3EDF0A3EEF0A3EFF022EF
:100A8600D083D082E493F608740193F60874029337
:090A9600F608740393F67404736E
:100A9F00A8828583F0D083D082120AB6120AB612CA
:100AAF000AB6120AB6E473E493A3C583C5F0C583EF
:100ABF00C8C582C8F0A3C583C5F0C583C8C582C8A1
:010ACF002204
:100AD000BB010789828A83020A9F5005E9F8020A4E
:0A0AE00086BBFE05E9F8020CCD22EA
:100AEA00FAE6FB0808E6F925F0F618E6CA3AF6220D
:100AFA00BB010DE58229F582E5833AF583020CEF05
:100B0A005007E92582F8020CE6BBFE07E92582F8C0
:100B1A00020CF8E58229F582E5833AF583020D0194
:100B2A00D083D082F8E4937012740193700DA3A35A
:100B3A0093F8740193F5828883E47374029368606E
:060B4A00EFA3A3A380DF6E
:100B5000EC8EF0A4CCC5F0CCCDF8EFA4CEC5F02D32
:100B6000FDE43CFCE8A42EC8C5F03DFDE43CFCEFF0
:0D0B7000A4FFE5F028FEE43DFDE43CFC227E
:10C7790012078C601CFF09E970010AC0E0EAC0E0F9
:10C78900EBC0E012C95BD0E0FBD0E0FAD0E0F98061
:0AC79900DF7F0A12C95BE4FEFF22F5
:10C0F1008B458A4689478B4B8A4C894DAB45054711
:10C10100E547AA467002054614F912078C70ED74D2
:10C11100FF2547F54774FF3546F546AB48054AE527
:10C121004AAA497002054914F912078CFFAB45056B
:10C1310047E547AA467002054614F9EF1207D27087
:08C14100DAAB4BAA4CA94D2218
:100B7D00E709F60870FA8046E709F20870FA803E38
:100B8D0088828C83E709F0A370FA807EE309F6086A
:100B9D0070FA8076E309F20870FA806E88828C8391
:100BAD00E309F0A370FA806289828A83E0A3F608D4
:100BBD0070FA805689828A83E0A3F20870FA804A1F
:100BCD0080D280FA80C680D4806580F2803180101A
:100BDD0080A680EA809A80A880DA80E280CA80317F
:100BED0089828A83ECFAE493A3C8C582C8CCC583F5
:100BFD00CCF0A3C8C582C8CCC583CC70E9800D8963
:100C0D00828A83E493A3F60870F9ECFAA9F0EDFB60
:100C1D002289828A83ECFAE0A3C8C582C8CCC58339
:100C2D00CCF0A3C8C582C8CCC583CC70EA80DD8961
:100C3D00828A83E493A3F20870F980CE88F0ED24C4
:100C4D0002B4040050C4F582EB2402B4040050BA7F
:090C5D002323458223900BCD7383
:10C1F1008B458A468947E4F54DF54EE54C154CAE25
:10C201004B7002154B4E6033AB48AA49A94A12073D
:10C211008CFFAB45AA46A947054EE54EAC4D7002D1
:10C22100054D14F5828C83EF1207E4EF60CD7401A4
:10C23100254AF54AE43549F54980C0AB45AA46A9E6
:02C24100472292
:10C98600E4FFFE12078C600C0FEF70010E09E970D0
:05C99600F20A80EF220F
:10C8AC00E94A4B70012212078CFF6D700122EF7068
:0CC8BC0004FBFAF92209E970ED0A80EA99
:10C149008B478A4889498B4A8A4B894CAB4AAA4B07
:10C15900A94C12078C600D7401254CF54CE4354B44
:10C16900F54B80E8AB4AAA4BA94C12078C6D7001BC
:10C1790022E54C154CAA4B7002154BF9E547854849
:10C1890083854982654A7008E965827003EA658397
:06C1990070D2FBFAF9224E
:10B223008B458A468947AB45AA46A94712078CFF37
:10B2330012CA0E500D74012547F547E43546F5460D
:10B2430080E4D216AB45AA46A94712078CFF642BAC
:10B253006004EFB42D1BAB450547E547AA467002D2
:10B26300054614F912078C642D6003D38001C39241
:10B2730016E4F548F549AB45AA46A94712078CFFE2
:10B2830012CA435036AB45AA46A94712078CFF336F
:10B2930095E0FEEF24D0FBEE34FFFAAE48AF497CD5
:10B2A300007D0A120806EF2BF549EE3AF5487401C2
:10B2B3002547F547E43546F54680BB301606AE48CC
:0EB2C300AF498009C3E49549FFE49548FE2297
:100C6600EF4E6012EF60010EEDBB010B89828A83A5
:100C7600F0A3DFFCDEFA2289F05007F709DFFCA9B2
:0C0C8600F022BBFEFCF309DFFCA9F02209
:10BB1E0002C971E493A3F8E493A34003F68001F203
:10BB2E0008DFF48029E493A3F85407240CC8C33328
:10BB3E00C4540F4420C8834004F456800146F6DFF7
:10BB4E00E4800B010204081020408090C243E47E82
:10BB5E00019360BCA3FF543F30E509541FFEE493EC
:10BB6E00A360010ECF54C025E060A840B8E493A3B3
:10BB7E00FAE493A3F8E493A3C8C582C8CAC583CADE
:10BB8E00F0A3C8C582C8CAC583CADFE9DEE780BE96
:01C2930000AA
:100C9200C5F0F8A3E028F0C5F0F8E58215827002ED
:060CA2001583E038F0228A
:0C0CA800E2FC08E2FD08E2FE08E2FF2288
:0D0CB400E2FB08E2F908E2FA08E2CBF822C0
:0C0CC100ECF208EDF208EEF208EFF2226F
:100CCD00D083D082E493F208740193F208740293F6
:090CDD00F208740393F27404732D
:090CE600E6FB08E6FA08E6F92233
:090CEF00E0FBA3E0FAA3E0F92206
:090CF800E2FB08E2FA08E2F9222D
:0C0D0100E493FB740193FA740293F9224E
:0FCA4300EFC394304007EF943A50028001C322B2
:10CA0E00EFC394094005EF940E4003BF2003D3807B
:03CA1E0001C3222F
:00000001FF
